:020000040800F2
:10000000102D0020C503000885E1000841DA000832
:1000100081E10008B52E0008090F0108D703000888
:10002000000000000000000000000000D9030008EC
:100030000540000800000000AD0400085904000855
:10004000E1030008E1030008E1030008E103000800
:10005000E1030008E1030008E1030008E1030008F0
:10006000E1030008E1030008E1030008E1030008E0
:10007000E1030008E1030008E1030008E1030008D0
:10008000E1030008E1030008E1030008E1030008C0
:10009000E1030008E1030008E1030008E1030008B0
:1000A000E1030008E1030008E1030008E1030008A0
:1000B000E1030008E10300081140000821400008A6
:1000C00031400008E1030008E1030008E1030008F3
:1000D00000000000E1030008E1030008E10300085C
:1000E000E1030008E1030008E1030008E103000860
:1000F000E1030008CDE60008DDE60008E1030008A2
:10010000E1030008EDE60008E1030008E103000850
:10011000E1030008E1030008E1030008E10300082F
:10012000E1030008E1030008E1030008E90E01080B
:10013000F90E0108C9F80008E1030008E10300080E
:10014000E1030008E1030008E1030008E1030008FF
:10015000E1030008E1030008E1030008E1030008EF
:10016000E1030008E1030008E1030008E1030008DF
:10017000E1030008E1030008E1030008E1030008CF
:10018000E1030008E1030008E1030008E1030008BF
:10019000E1030008E1030008E1030008E1030008AF
:1001A000E1030008E1030008E1030008E10300089F
:1001B000E1030008E1030008E1030008E10300088F
:1001C000E1030008E1030008E1030008E10300087F
:1001D000E1030008E1030008E1030008E10300086F
:1001E000E1030008E1030008E1030008E10300085F
:1001F000E1030008E1030008E1030008E10300084F
:10020000E1030008E1030008E1030008000000002A
:1002100000000000E103000800000000E103000806
:10022000E1030008E1030008E1030008E10300081E
:10023000E1030008E1030008E1030008E10300080E
:10024000E1030008E1030008E103000800F002F800
:1002500000F0A8F814A696E8000CB244B344DA45BE
:1002600001D100F09FF8BAE80F000FA696E8300021
:10027000A5EB040504EB0607AAEB0704A7F10107A9
:100280004FEA15154FEA3414A4F10104AC4201D32E
:1002900000F088F813F0010F18BFFB1A43F00103B8
:1002A00000F001F8DBE71847CC470100EC470100FC
:1002B000103A24BF78C878C1FAD8520724BF30C892
:1002C00030C144BF04680C607047000070470000F4
:1002D0000023002400250026103A28BF78C1FBD84F
:1002E000520728BF30C148BF0B6070476E2900F02D
:1002F0006F83702900F0B184662914F0EA816529C2
:1003000014F0E781672914F0E481612914F0E38196
:1003100003681B0A28BF41F08001692900F01C8393
:10032000642900F01983752900F016836F2900F005
:100330003F84782900F07D84E92900F0D983E429FD
:1003400000F0D683F52900F0D383EF2900F03C8438
:10035000F82900F07C840368DB0928BF41F08001A4
:10036000632901F0E984732901F0EE84E32901F0A7
:10037000F984F32901F0FE84002070471FB514F0C2
:1003800093F902F0C5F904000020002113F084FF66
:10039000401C60600020002113F068FFE0601FBD7A
:1003A00010B510BD02F086F91146FFF7E7FF13F014
:1003B0005DF902F077FA03B4FFF7F2FF03BC02F035
:1003C000E3FC00000A4880470A480047FEE7FEE7D2
:1003D000FEE7FEE7FEE7FEE7FEE7FEE7FEE7FEE7F5
:1003E000FEE7000004480549054A064B7047000037
:1003F00095E500084D02000810270020102D002070
:10040000102900201029002072B64FF0E020174973
:10041000C0F8081D1648016841F001010160154847
:100420001249096801604FF0E020134941614FF023
:10043000070101614FF00001C0F8181D4FF07F4126
:10044000C0F81C1D0D49C0F8201D7047FFF7FEBF06
:1004500001B5BDE80140704701B500F099F8BDE86D
:1004600001407047FFF7FEBFFFF7FEBF0000000826
:10047000001000E0C80200209F2526000000FF4079
:100480004FF000002E4A1060EFF3148020F00400BB
:1004900080F3148862B64FF080504FF0E021C1F82D
:1004A000040DBFF34F8FBFF36F8FFEE72548264A39
:1004B0004FF00003016891B10360EFF3098C2CE960
:1004C000F00F1EF0100F01D12CED108A1F4C4CF8CC
:1004D00004EDC1F808C025680DB18D61236072B6C6
:1004E0001168D1B1016062B64F68184C8D6907F18F
:1004F00001074F602560D1F80CC08CF30B88D1F850
:1005000008C05CF804EB1EF0100F01D1BCEC108A9F
:10051000BCE8F00F8CF30988704772B6116801606F
:1005200009B962B6F9E74FF000674FF0E028C8F864
:10053000047D62B6D8E700BFB0EE400A7047000005
:100540004002002030020020340200202C0800204D
:10055000026922F00702A2F144026FF04303136024
:100560004FF0000353609360D36013615361936154
:10057000D361136253629362D362136353634FF088
:10058000FF339363D1634FF08073136482607047CD
:100590002249086800F101000860214B1A683AB14D
:1005A000A2F101021A601AB91E4B4FF00100186047
:1005B0001D490868026822B11C4B4FF001021A6005
:1005C00008E000F104001A4B1A68904201D1194B5F
:1005D00018680860134B1A6812B914490868C8B142
:1005E00001B51249086808B112F05AF90D4B1A68A2
:1005F00072B112F0C9F81048016849B90F48016892
:100600000F4A13680F484FF08052994200D00260A1
:10061000BDE80140BFF34F8F704700007803002012
:100620002C080020DC020020D4020020D802002088
:1006300064030020680300204002002030020020F4
:100640003402002004ED00E053EA020C00F069805F
:100650002DE9F04B4FF00006002B1FBFB3FA83F5D6
:1006600003FA05F424FA05F65E4012BF1643B2FA07
:1006700082F502FA05F4C5F120051EBF22FA05FC39
:1006800044EA0C04203556EA044C4FEA144418BFDF
:10069000641C4FF000084FF00009904271EB030C0E
:1006A00039D3002919BFB1FA81F701FA07F6B0FA78
:1006B00080F700FA07F6C7F120071EBF20FA07FCF3
:1006C00046EA0C062037B6FBF4FCA7EB0507103F03
:1006D00007F01F0BCBF120062CFA06F60CFA0BFBE9
:1006E00044BFB3460026202FA4BF5E464FF0000B48
:1006F0005BEA060C08BF4FF0010B19EB0B0948EB46
:100700000608ABFB027C06FB02CC0BFB03CCC01B38
:1007100071EB0C01C1E70B46024641464846BDE875
:10072000F08B13B5084318BF4FF0FF300146AFF30D
:100730000080BDE81C4070471CB50C46064B7B444E
:1007400069460090204600F05CF9044600206946A6
:1007500000F06AF920461CBDE70200000FB400B5A6
:100760008DB010A9099000910B904FF0FF300A90C6
:1007700000200C90064878440690064878446A4663
:1007800007900F9909A800F0FFFC0DB05DF814FB6D
:100790002F0A0000470A000010B5431C02E010F8C1
:1007A000011B71B18107FAD14FF0013202C88C1AD6
:1007B0008C4314EAC211F9D0C01A0A0603D0C01E35
:1007C00010BDC01A10BD0A0401D0801E10BD090260
:1007D000FCD0401E10BD02F0FF0343EA032242EAB0
:1007E000024200F002B84FF000020429C0F012806B
:1007F00010F0030C00F01B80CCF1040CBCF1020FD4
:1008000018BF00F8012BA8BF20F8022BA1EB0C01A8
:1008100000F00DB85FEAC17C24BF00F8012B00F89E
:10082000012B48BF00F8012B70474FF0000200B5C4
:10083000134694469646203922BFA0E80C50A0E803
:100840000C50B1F12001BFF4F7AF090728BFA0E8B1
:100850000C5048BF0CC05DF804EB890028BF40F87D
:10086000042B08BF704748BF20F8022B11F0804FBF
:1008700018BF00F8012B704770477047704710B5DC
:1008800000F018FE006810BD10B5044600F012FE1E
:10089000046010BD70B5044685690068C10601D5C5
:1008A000302600E02026C00707D070BDD4E9012122
:1008B00030469047206A401C20626D1EF6D570BD00
:1008C00070B5044685690078C00707D170BDD4E9CA
:1008D000012120209047206A401C20626D1EF6D521
:1008E00070BD09684A0501D540B27047C905FCD5FD
:1008F00000B2704709684A0501D5C0B27047C90502
:10090000FCD580B2704770B50C460546012A05D06B
:100910002878800600D5EA69002302E0012305E07B
:100920005B1C934202D2E05C0028F9D1A869E6186A
:10093000C01AA861286A184428622846FFF7AAFF4F
:1009400004E0D5E9012114F8010B9047B442F8D333
:100950002846FFF7B5FF70BD2DE9F041064600249B
:1009600010687529314616A510D0FFF7BAFF002888
:1009700002DA404213A507E031688A0701D512A5C3
:1009800002E0490704D511A5012401E0FFF7B2FFF9
:1009900000210A2206F1240709E0B0FBF2FCB0FBBB
:1009A000F2F302FB1C00303078541846491C002832
:1009B000F3D123462A463046BDE8F04100F0CCBDD5
:1009C000000000002D0000002B00000020000000AF
:1009D00011680268006A530501D508700AE0D30562
:1009E00001D5088006E0130603D5C217C1E900024D
:1009F00000E008600120704701694A1C0261087824
:100A0000704700B58FB0CDE901310021059105494E
:100A10007944CDE903101146684600F029F90FB07A
:100A200000BD0000E5FFFFFF0A6802F8010B0A6045
:100A3000704700002DE9FF5F15468A460446DFF83F
:100A4000AC80F8440027D8E900103E46CDE90010FC
:100A500010E03AF816106A4602A801F002FE411CA6
:100A600007D02178890603D5E269391891420DD85B
:100A70000744761C2078800602D5E069B84205DD7F
:100A8000AE42E6DB3AF816000028E2D1A069C01BAE
:100A9000A0612046FFF7FEFED8E90010CDE9001066
:100AA000002017E03AF818106A4602A801F0D9FDB4
:100AB000B0F1FF3F81460BD000250DF1080B05E09A
:100AC000D4E901211BF8050090476D1C4D45F7D373
:100AD00008F10100B0428046E4DB206A384420621D
:100AE0002046FFF7EDFEBDE8FF9F0000923D0100AC
:100AF0002DE9F0418046D21D22F007020025D2E9FF
:100B00000002F52915A614D0011E72F1000106DAC3
:100B10000023D0EB030063EB020211A608E0D8F833
:100B200000108B0701D50FA602E0490701D50EA6DC
:100B300001251146002408F1240704E000F0BEFC62
:100B400030323A55641C50EA0102F7D12B46324646
:100B500021464046BDE8F04100F0FEBC0000000028
:100B60002D0000002B0000002000000030B4002108
:100B700000F1240408E002F00705D208303542EA0B
:100B80004372DB086554491C52EA0305F3D104683B
:100B9000002310A2250708D504F020040C4304D03C
:100BA000C46901230CA2641EC46130BC00F0D4BC33
:100BB00010B5044621461068FFF79CFE0246204609
:100BC000BDE810400023D1E7D21D22F00701D1E992
:100BD0000023CBE70000000030000000F0B40D4619
:100BE0000188090502D5214C7C4402E01F4C7C445D
:100BF0000E34002100F1240608E002F00F0712096C
:100C0000E75D42EA03721B097754491C52EA030765
:100C1000F3D102780023120704D5702D06D009B154
:100C2000022311342246F0BC00F096BC012310349C
:100C3000F8E770B504460D4621461068FFF75AFEE6
:100C4000024629462046BDE870400023C6E7D21D73
:100C500022F00703D3E90023C0E70368126843F0DA
:100C6000200303600823C3610023B7E7F43B0100BE
:100C70002DE9F05F894604464FF0000ADFF874B1B1
:100C8000FB44C0F820A02046E1688847002874D0C3
:100C9000252806D0D4E901219047206A401C206213
:100CA000F1E700265F462046E16888472028054690
:100CB00007DB312D05D2781910F8200C08B1064356
:100CC000F1E7B00701D526F00406C4F81CA0002700
:100CD000C4F818A02A2D09D0284613F078FA38B3A2
:100CE00004EB8708303DC8F8185019E059F8041B88
:100CF000204604EB87029161E1688847012F054691
:100D000018D1E069002820DA26F020061DE0D8F886
:100D1000180000EB800005EB40003038C8F81800E0
:100D20002046E1688847054613F051FA0028EED1C5
:100D3000012F0AD02E2D08D12046E16888477F1C5C
:100D40000546022F46F02006C4DBA069002803DA1E
:100D5000404246F00106A061F00701D026F01006DF
:100D60006C2D0BD0682D09D04C2D39D06A2D35D083
:100D7000742D35D07A2D33D016E038E0E1682F4657
:100D800020468847B842054609D16C2F26D04FF43B
:100D90008060E168064320468847054604E06C2FE2
:100DA0001AD04FF4807006430DB3A5F14100192805
:100DB00002D8203546F400664A4629462046266079
:100DC0004E46FFF793FA80B101280BD0F61D26F0AE
:100DD000070000F1080956E74020E4E78020D8E743
:100DE0000020D6E706F104094DE7284652E7206ABD
:100DF000BDE8F09F843B01002DE9FF4F1C46914662
:100E00004FF0FF3581B000218A468846D4E901675A
:100E1000A16902986D1C8847216A8346884700288B
:100E2000F6D1BBF1FF3F0CD0002F26F4C0661ADDCF
:100E3000700615D5BBF12B0F0AD0BBF12D0F0FD1CA
:100E400004E04FF0FF3005B0BDE8F08F46F4806657
:100E5000A16902986D1C88477F1E8346002F02DD22
:100E6000BBF1300F03D0B9F1000F2AD025E0A16902
:100E70006D1C02987F1E46F400768847002F83463B
:100E800005DDBBF1780F06D0BBF1580F03D0B9F1E7
:100E9000000F10D011E0B9F1000F02D0B9F1100F1E
:100EA0000BD1A1696D1C02987F1E26F4007688473D
:100EB0008346102000E0082081464FEAE970009048
:100EC00017E00A20F8E74346AAFB0928DDF800C02E
:100ED0007F1E03FB098046F4007605F101050AFB3D
:100EE0000C0112EB0B0A029841EBEB78A1698847E1
:100EF0008346002F06DD4946584600F03FFF5FEA73
:100F0000000BE0D5E16902988847B00502D46FF084
:100F1000010098E7F00718D1700610D5514670050A
:100F200005D50023D1EB030163EB080200E0424644
:100F30002068031D23600068C0E9001205E02068F6
:100F4000011D21600068C0E900A828467BE72DE963
:100F5000FF5F1D464FF0FF3B91464FF000085F4694
:100F6000D5E90146A96901987F1C8847296A82460C
:100F700088470028F6D1BAF1FF3F0CD0002E24F4A8
:100F8000C06419DD600614D5BAF12B0F09D0BAF18F
:100F90002D0F0ED103E0584604B0BDE8F09F44F495
:100FA0008064A96901987F1C8847761E8246002EBE
:100FB00002DDBAF1300F03D0B9F1000F26D032E0D4
:100FC000A969761E01987F1C44F400748847002E9E
:100FD000824605DDBAF1780F06D0BAF1580F03D07A
:100FE000B9F1000F10D01EE0B9F1000F02D0B9F135
:100FF000100F18D1A969761E01987F1C24F4007483
:1010000088478246102002E0082000E00A2081463E
:1010100009E0A96908FB0908761E01987F1C44F4C1
:10102000007488478246002E05DD4946504600F090
:10103000A5FE0028EDDAE96901988847A00502D4E9
:101040006FF00100A8E7E00725D1600613D5600521
:1010500002D5C8F1000000E0404629680A1D2A6058
:101060000968220501D5087015E0220701D508801E
:1010700011E008600FE02868011D29600068210563
:1010800002D580F8008006E0210702D5A0F8008094
:1010900001E0C0F8008038467EE72DE9FF5F4FF0A1
:1010A00000089946144646469169D2E901A7DDF841
:1010B00038B001988847054659EA0B0005D009E089
:1010C000A1690198761C88470546216A2846884709
:1010D0000028F5D1681C03D05FEACA7005D015E07E
:1010E0004FF0FF3004B0BDE8F09F2068011D216083
:1010F000D0F800800AE05FEACA7001D108F8015B0D
:10110000A169761C01987F1E88470546002F1ADDCD
:10111000681C18D0B9F1000F0DD0E81705EBD060AE
:10112000421120F01F0059F822102A1A0120904085
:101130000142E0D107E0BBF1000FDCD12846216A73
:1011400088470028D7D0E16901988847BBF1000F94
:1011500007D1002E05DD5FEACA7002D1002188F8B0
:101160000010A068B84203DDBBF1000F03D017B137
:101170006FF00100B6E73046B4E7000002681144A2
:101180001378016018467047D16005497944516170
:1011900004497944116200211161114600F0FCBD3F
:1011A000EDFFFFFFB1030000426842B1016811F892
:1011B000013B23B1521EC0E90012184670470121BD
:1011C000C160881E704742685AB1C368016843B95C
:1011D00083688B4205D0491E521CC0E900120020D2
:1011E00070474FF0FF3070472DE9FF4F4FF0000878
:1011F0009A461446C146464683B0D2E901B7CDF8B7
:101200000080CDF8048091690498884710990546BC
:101210005AEA010005D009E0A1690498761C8847C4
:101220000546216A284688470028F5D1681C03D066
:101230005FEACB7005D02AE04FF0FF3007B0BDE881
:10124000F08F2068011D2160D0F800801FE002A807
:101250006A46E9B201F0E5F9411C07D0801C09D0CB
:101260004FF000095FEACB7007D00AE0E16904980B
:1012700088473EE04FF0010904E0BDF8081028F867
:10128000021B7F1EA1690498761C88470546002F23
:101290001ADD681C18D0BAF1000F0DD0E81705EB65
:1012A000D060421120F01F005AF822102A1A0120A3
:1012B00090400142CBD107E010980028C7D12846C2
:1012C000216A88470028C2D0E16904988847B9F1AB
:1012D000000F0ED1109830B9002E04DD5FEACB70FC
:1012E00001D1A8F80000A068B84202DD109818B13A
:1012F00017B16FF00100A1E730469FE72DE9FF4FDE
:101300004FF000089B461446454683B0D2E901964B
:10131000CDF80080CDF804809169DDF848A00498EC
:10132000884707465BEA0A0005D009E0A1690498EE
:101330006D1C88470746216A384688470028F5D142
:10134000781C03D05FEAC97005D01BE04FF0FF3076
:1013500007B0BDE8F08F2068011D2160D0F8008043
:1013600010E05FEAC97007D16A464046B9B201F0A1
:1013700078F9411C31D08044A1696D1C0498761E17
:1013800088470746002E14DD781C12D0BBF1000000
:1013900007D03B46DDE9101201F034F90028E0D116
:1013A00007E0BAF1000FDCD13846216A88470028EF
:1013B000D7D0E16904988847BAF1000F06D1002D13
:1013C00004DD5FEAC97001D188F80000A068B0426E
:1013D00003DDBAF1000F03D016B16FF00100B7E7DB
:1013E0002846B5E72DE9FF5F9B46144600273D469A
:1013F0009169D2E90196DDF840A0019888478046BE
:101400005BEA0A0005D009E0A16901986D1C8847D4
:101410008046216A404688470028F5D1B8F1FF3F51
:1014200003D05FEAC97005D014E04FF0FF3004B07C
:10143000BDE8F09F2068011D216007680AE05FEAAF
:10144000C97001D127F8028BA1696D1C0198761E25
:1014500088478046002E15DDB8F1FF3F12D0BBF162
:10146000000007D04346DDE90E1201F0CBF800285A
:10147000E5D107E0BAF1000FE1D14046216A884783
:101480000028DCD0E16901988847BAF1000F05D146
:10149000002D03DD5FEAC97000D13880A068B0423A
:1014A00003DDBAF1000F03D016B16FF00100BEE703
:1014B0002846BCE7004870471000002030B5B0F166
:1014C0000A0271F100034FEA900E4EEA817EB0EB02
:1014D0000E0061EB91014FEA101E4EEA017E10EB07
:1014E0000E0041EB11114FEA102E4EEA016E10EB87
:1014F0000E0041EB11214FEA104E4EEA014E10EB67
:101500000E0041EB1141401841F100014FEAD000BB
:1015100040EA41704FEAD1014FEA810444EA9074F5
:1015200010EB800544EB01046D1944EB0404521BDD
:10153000A3414FF0000348BF0A3200D530BD401C24
:1015400041F1000130BD10B5044601F0D9F8006842
:10155000005D00F0010010BD2DE9F0470D469946F1
:101560009246044600F124080168880604D5E06923
:1015700021F01001216000E00120A84201DD471B9D
:1015800000E00027A1697A1902EB0900081AA0619E
:101590002078C00602D42046FFF77CF9002608E038
:1015A000D4E901211AF806009047206A401C761CF5
:1015B00020624E45F4DB2078C0060AD52046FFF7AE
:1015C00069F906E0D4E9012130209047206A401CE7
:1015D0002062381EA7F10107F4DC07E0D4E90121FD
:1015E00018F805009047206A401C2062281EA5F1CB
:1015F0000105F3DC2046FFF763F92078000602D5E9
:101600000220BDE8F0870120FBE72DE9FF4F0C46E3
:101610001E464FF0FF378BB0D2E90001DDF8608045
:101620000A908A46C1F30A5505B93D46002108468D
:101630004FF00000BAF1000F00F4400005DA00EBB3
:1016400080004FF4400101EA50004FEA9059B9F18F
:10165000010F00DDB9460A9850EA4A000ED044F660
:101660001050A5F2FF3545432F14B8F1000F1ED0DE
:101670007542291E1EDDC9F100021CE0B8F1010F00
:101680004FF0000001D0302103E0F24305E0215487
:10169000401CB042FBDB30460022002121540B9954
:1016A000C1F80880C1E900200FB0BDE8F08FBD1B74
:1016B0006D1CDEE74A4600DA694206A801F080F8B0
:1016C00006AB93E8070003AB83E8070050460A998E
:1016D00012F018F88DE80700A0F500501F380090B0
:1016E0000398002D0ADD42F21F014A4608440023F8
:1016F00003A90390684612F0C3FA09E0A0F5005070
:101700004A461F38002303A90390684612F0E2FA04
:101710008DE807000004000C03D04FF0FF304108B3
:1017200000E01046B8F1000F03D0002200921546E9
:101730001EE0751E05D4FFF7C1FE303262556D1EE6
:10174000F9D5B3460122084302D000227F1C04E0F1
:101750002078302801D100227F1E002A099784D0EA
:101760001DE0112D07DAFFF7A9FE303262556D1C1E
:1017700050EA0102F5D1084302D00098C8B10EE04A
:101780000021681E05E0235C625C63542254401E05
:10179000491C8142F7DBAB46A81B401E0990002084
:1017A00004F80B000B98099AC0F80880C0E9002BD8
:1017B0007AE711264FF0000857E72DE9F04F8846E9
:1017C0000446D21D22F0070191B0D1E90001CDE914
:1017D0000A0112F0CBFB02460B98C00F01D02D205E
:1017E00007E02068810701D52B2002E0202101EAD3
:1017F000C000032A099001D0072A05DB03464146B1
:10180000204600F09DFF0BE12078800601D5E069BD
:1018100000E00620B8F1650F814606D0B8F1660FEA
:1018200018D0B8F1670F70D131E00020B9F1110F75
:10183000009001DB112301E009F101030AAA01A9CB
:101840000CA8FFF7E2FEDDE90C70002609F10105A6
:10185000834647E001204B4600904FF000470AAA1C
:1018600001A90CA8FFF7D1FEDDE90DB00C995D468A
:10187000002610B909F101000D18B9EB050003D4D9
:10188000C0F1FF3609F10105A5EB09002BE0B9F124
:10189000010F01DA4FF001090020B9F1110F00909A
:1018A000484601DD112300E003460AAA01A90CA85D
:1018B000FFF7ABFEDDE90C704D460026834620782D
:1018C00000070AD4AB4500DA5D4601A8012D04DD0E
:1018D000411911F8011C302907D04F4502DA17F1E0
:1018E000040F04DA012082460FE06D1EEEE7002FA0
:1018F00002DCED1B3E4403E0781CA84200DD7D1CA9
:10190000B81B00F1010A4FF000472078000703D40C
:10191000AA4501DB4FF0FF3A0021B7F1004F0DF16E
:1019200043088DF8431024D002202B23002F01DA26
:101930007F422D230A21021EA0F1010000DC5FB1CD
:1019400097FBF1FC97FBF1F201FB1C7C17460CF1B5
:10195000300C08F801CDEEE7A8F1010003702188F2
:10196000090501D5452100E06521A0F1010800F835
:10197000011C09980FA9A1EB0807FF1D00B1012068
:10198000411901EBEA70A1693844081A401EA061B0
:101990002078C00602D42046FEF77CFF099828B1C3
:1019A000D4E901219047206A401C20622078C006BB
:1019B00022D52046FEF76EFF1EE0002E04DBB34565
:1019C00002DD01A8805D00E03020D4E901219047CC
:1019D000206A401C2062761CAAF101005FEA000A1E
:1019E0000AD100F095FEC0680168405CD4E901218D
:1019F0009047206A401C2062281EA5F10105DCDC0E
:101A000007E0D4E9012118F8010B9047206A401C37
:101A10002062381EA7F10107F3DC2046FEF750FFD5
:101A2000032011B041E600002DE9F04F04460D46B9
:101A3000D21D22F0070089B0D0E900974846394608
:101A400012F094FA0246F80F01D02D2307E0206827
:101A5000810701D52B2302E0202101EAC0038DF884
:101A600020300BB1012000E00020032A824601D083
:101A7000072A04DB2946204600F062FE3FE1207879
:101A8000800601D40D2500E0E569C7F30A560D2D47
:101A900049DA00214FEA175B08464FF00000002F9B
:101AA00000F4400007DA00EB80004FF4400100EB47
:101AB000D07001EA60008115012901DD4FF0FF318E
:101AC00000224FEA850CBCF1180F06D31346ACF187
:101AD00018004FF08052C24003E04FF4801323FA05
:101AE0000CF30CF10C0CBCF1200F04D3ACF1200C66
:101AF00009FA0CF001E007FA0CF000294FF0004859
:101B000001DD18B90FE00ED140450CD319EB0209E5
:101B10005F4121B9404502D19F4329EA0209BBEB4D
:101B2000175F00D0761C2088000502D57B487844DA
:101B300002E07A487844193808AA302302F80A30BB
:101B4000037C0AF10101002E0AF1020A53546A468D
:101B500002DC4FF0300101E04FF031014FF001089D
:101B60008DF8001002D0A6F2FF3603E059EA4701D3
:101B700000D06B4E002D02DC2178090704D54FF010
:101B800002082E218DF80110C44600210BE0C7F396
:101B900003433F01C35C491C6D1E02F80830052950
:101BA00008F1010801DA002DF1DC00210CE000EB66
:101BB0001973491C1B786D1E082902F808304FEA7A
:101BC000091908F1010801DA002DF0DC21688B0603
:101BD00002D516E0A8F10108E04505DD02EB080397
:101BE00013F8013C302BF5D0B8F1000F09DD02EB02
:101BF000080313F8013C2E2B03D1090701D4A8F1E7
:101C00000108002D05DD3E2102F808106D1E08F1C7
:101C10000108407C002E02F8080008F1010804DAEF
:101C20002D20764202F8080002E02B2002F808007E
:101C30000A214FF47A70864208F101080BDB96FB0B
:101C4000F0F3303302F8083096FBF0F308F10108A6
:101C500000FB136601E0642E0CDB642096FBF0F3BE
:101C6000303302F8083096FBF0F308F1010800FB6E
:101C7000136601E00A2E06DB96FBF1F0303002F825
:101C8000080008F1010896FBF1F001FB106030300C
:101C900002F80800A16908F1010808EB050202EB4F
:101CA0000A00081AA0612078C00602D42046FEF778
:101CB000F1FD216A08AE01EB0A00206204E0D4E9DC
:101CC000012116F8010B9047BAF1010AF7D22078EA
:101CD000C00602D52046FEF7DDFD6E4609E016F887
:101CE000010B3E280FD0D4E901219047206A401C07
:101CF0002062B8F10108F2D22046FEF7E1FD09B0FA
:101D00000320BDE8F08F206A2844206203E0D4E974
:101D10000121302090476D1EEBD3F8E7FA2C01002B
:101D200002FCFFFF10B5436913B1AFF3008001E07F
:101D3000FEF7E9FD012010BD127800F124010A70C0
:101D400000224A700122EDE711684FF0FF32E9E707
:101D500010B5436913B1AFF3008001E0FEF76AFEEE
:101D6000012010BD128800F1240182840022C28467
:101D70000122EDE711684FF0FF32E9E73A2800D27F
:101D8000303820F02002412A01D3A2F137008842E6
:101D900001D34FF0FF3070472DE9F34F4FF0000AA9
:101DA0000C4656468DB001200C9001F10C000B90B2
:101DB00062690B9801219047051E2DD0252D2CD04E
:101DC000216A8847C0B162690B9801219047216A56
:101DD00088470028F7D16269411E0B98904700E0C0
:101DE000761CA1690D988847216A88470028F7D199
:101DF000E1690D988847DBE7A1690D988847A842FB
:101E0000074601D1761CD3E7E1690D9888477F1C0E
:101E100002D1BAF1000F6FD06BE162690B98002715
:101E20003D46394690472A2804D162690B98012122
:101E300090470125DFF8D08262690B980121904715
:101E4000A0F130010A290AD24745E5DC07EB8701FA
:101E500000EB4107303FDFD445F01005ECE7E90621
:101E600001D46FF000476C280AD04C2814D06828A1
:101E700015D06A280DD074281CD07A281AD01DE0FD
:101E800062690B98012190476C2802D045F0040547
:101E900014E045F002050DE045F020050AE0626916
:101EA0000B9801219047682802D045F0080505E00D
:101EB00045F4006562690B9801219047C4E9015718
:101EC00065283DD019DC58287AD00CDC452837D05D
:101ED00004DC252826D041289ED131E046282FD089
:101EE000472899D12CE05B2877D0612828D0632837
:101EF0007CD0642823D15AE0F6E06F2848D008DC73
:101F000066281DD067281BD0692821D06E2816D1DD
:101F100027E0702845D0732868D0752847D07828E6
:101F20000DD14DE0A1690D988847252805463FF45D
:101F300069AFE1690D9888476D1C3FF46AAFD8E03E
:101F40000D9923466A466FF0010012F026FCC5E0A9
:101F500045F0400023464FF000026060A80736D4E9
:101F60003EE0E8077FF447AF2068011D216000686C
:101F7000290501D506701BE7290701D5068017E75B
:101F8000A90703D5F117C0E9006111E706600FE763
:101F900045F0400023464FF008026060A80716D4C1
:101FA0001EE040F60E0125EA0100606016E045F0F3
:101FB000400023464FF00A026060A80707D40FE0F4
:101FC00045F040006060A80708D5234610220D990F
:101FD0006FF00100FEF710FF80E007E010222346BB
:101FE0000D996FF00100FEF7B2FF77E04FF00009A6
:101FF00063284F46C8464B46CB4602D05B2806D0E6
:1020000038E0E80601D40120A060012732E06269CF
:10201000D4F80CB00B98012190475E2807D14FF0FF
:10202000010949466269D4F80CB00B9890472169C0
:1020300039B900210A4603AB43F82120491C08297D
:10204000FADBD8B3216949B308F1010862690B983A
:10205000012190475D28F4D1B9F1000F09D000208B
:1020600003A951F82020D24341F82020401C082821
:10207000F7DB03AB2069002820794FEA40701ED0BF
:102080005B462246CDF80080CDE901970D990028E6
:102090006FF0010020DAFFF7A5F91FE0C11703AACE
:1020A00000EBD1614B1121F01F0102EB8302411AB9
:1020B00013680120884003431360C7E719E00D99B6
:1020C000224600286FF00100009702DAFFF78CF833
:1020D00004E0FEF7E2FF01E0FFF710F900280ADA5A
:1020E000401C06D10C9820B14FF0FF300FB0BDE876
:1020F000F08F5046FAE7E90701D10AF1010A0644D8
:1021000000200C9054E60000CCCCCC0C2DE9FF4F05
:1021100006468BB00878FF2806D0491C2D2805D02C
:1021200000244FF0000908E000200CE00124F8E74B
:1021300009EB8903491C00EB43090878FF28F7D114
:1021400014B1C9F100008146107800252C46AA463A
:1021500029462D2801D02B2804D1521C2D2813D01C
:10216000002082468B461078FF280FD04FF0000CDD
:102170000A21521CA5FB017804FB018105FB0C110F
:10218000C5194BEB0104EEE70120EAE70021084600
:102190004FF00000BAF1000F02D000EB80004008C1
:1021A000C0F38157012F01DD4FF0FF370E9955EA3B
:1021B000040009EB01080BD04FF0020918F5FA7F73
:1021C00016DA4FEACA70002F706008DD012007E0C0
:1021D0004FEACA70C6E900B00FB0BDE8F08F00202A
:1021E0003060FFF767F9C0F800901821084616E044
:1021F000B8F5FA7F18DD002F02DAF748784401E0DD
:10220000F6487844D0E90010C6E9001040EACA70E8
:102210007060FFF74FF9C0F80090142108460FB026
:10222000BDE8F04F12F052BA002108464FF000000E
:10223000B8F10001099002DAC7F1000200E03A4665
:1022400001DAC8F1000106A800F0BAFA06AB93E87B
:10225000070003AB83E8070044F23E005BEA040199
:102260000090584604D144F21E012C465D46009170
:10227000210C0904014306D10099240444EA1544C1
:102280002D041039009104F07F41014306D10099DB
:10229000240244EA15642D020839009104F07041CB
:1022A000014306D10099240144EA15742D01091F48
:1022B000009104F04041014306D10099A40044EA92
:1022C0009574AD00891E009104F00041084304D1CB
:1022D00000986D196441401E00904FF001033A468A
:1022E0006846B8F1000FCDE9014503A902DD11F000
:1022F00006FD01E011F0D9FCBAF1000F04460D46CD
:1023000001D084F00044002108464FF000000999F4
:1023100040F2FF77484010F00C0F07D124F0004046
:10232000284303D0C4F30A50B84212D1FFF7C2F8D1
:10233000C0F80090C4F30A50B8420AD1A8487844C3
:10234000D0E90010C6E9001004F0004108437060B5
:1023500042E7C6E900543FE72DE9FF4F1F464FF023
:10236000000A4FF0FF38454691B0D7E90146CDF855
:102370003CA000F0CDF9C0680168405C1090B969DC
:1023800012986D1C8847396A814688470028F6D123
:10239000B9F1FF3F0AD0002E24F4D06411DDB9F169
:1023A0002B0F08D0B9F12D0F0BD102E0404615B02C
:1023B00013E744F48064B96912986D1C8847761E4F
:1023C0008146600504A901D52D2000E02B20002EB8
:1023D00001F1010B0DF130088DF810003FDDB9F16E
:1023E000690F08D0B9F1490F05D0B9F16E0F02D0CD
:1023F000B9F14E0F1CD13B4601A8009580E8500270
:10240000DDE912126FF0020012F0CBF9C11CCED13F
:102410000EE0B96912986D1C884781461398761EA4
:1024200044F4007405600F98401C002E0F9016DDD8
:10243000B9F1300FEDD0B9F1780F02D0B9F1580FE2
:102440000DD10F9801280AD13B46CDE90054DDE9B2
:102450001212001F029612F0A2F9C11CA7D1109906
:1024600089453ED144F0800406E01399681CAAF126
:10247000010A44F400740860B9696D1C1298761E54
:10248000884730288146F0D02BE01099894505D146
:10249000200603D4761E44F0800418E0484611F06C
:1024A00096FE08B3761E0DF123029345A9F1300084
:1024B00044F4007406D20BF8010B200607D5AAF1EC
:1024C000010003E0200602D40AF101008246A005C3
:1024D00002D51399681C0860B96912986D1C884769
:1024E0008146002ED1DC53E0002E51DDB9F1650F9D
:1024F00002D0B9F1450F4BD1A00549D5B9696D1C82
:102500001298761E24F440748847002E81460CDD14
:102510002B2804D0B9F12D0F07D144F48074B96988
:1025200012986D1C8847761E8146E00501D52D2145
:1025300000E02B2108F8011BCDF8008021E0761E79
:102540000DF13901884544F400740CD2A9F1300032
:1025500010F0FF0088F8000002D10099884509D9E1
:1025600008F1010806E0E00501D51E4801E042F24D
:102570000F708246B96912986D1C8847814613987E
:102580000560002E04DD484611F021FE0028D6D15A
:10259000F96912988847FF2053468BF8000088F8A5
:1025A000000000200A900B9004AA0CA90AA8FFF7CB
:1025B000ADFDA00502D46FF00100F8E614F0240F81
:1025C00012D0E0071CD13868DDE90A12031D3B6018
:1025D0000068C0E9001213E09C2801008E28010069
:1025E00052270100F1D8FFFF0AA9684611F0DCFD6F
:1025F000E00705D13868009A011D39600068026063
:102600002846D4E610B508E030F8024B9C4204D1CD
:102610000AB1002010BD012010BD491EF4D21046A1
:1026200010BDF8B516460C46054600F069F803687B
:1026300093F80101012804D0185D78B101202C80A5
:10264000F8BDD3F803013246214603F20313C7183D
:1026500068460023B84700992980F8BD4FF0FF3045
:10266000F8BD2DE9F04116460C46054600F048F845
:10267000036893F80101012807D0FF2C12D8185DD8
:1026800080B101202C70BDE8F081D3F807013246FB
:10269000214603F20713C7182846BC46BDE8F0419F
:1026A000002360474FF0FF30EDE70000004870471F
:1026B000100000207546FFF7F9FFAE460500694699
:1026C000534620F00700854618B020B5FDF78AFE76
:1026D000BDE820404FF000064FF000074FF0000823
:1026E0004FF0000BAC46ACE8C009ACE8C009ACE860
:1026F000C009ACE8C00921F007018D467047000011
:1027000010B500F005F8001D10BD00BF8D1B0100C5
:102710000048704730000020B2F120030AD5C2F112
:10272000200301FA02F120FA03F341EA030100FA5F
:1027300002F0704700FA03F14FF00000704700000C
:102740002DE9F0411F46044603260168072A01F4DB
:10275000006004DB08B116A505E016A503E008B18A
:1027600015A500E015A521F010002060A069C01E8D
:10277000A0610FB1401EA0612046FEF78BF84FB15B
:10278000D4E9012138469047206A401C2062C01CD1
:10279000206206E0206AFAE7D4E9012115F8010B6E
:1027A0009047761EF8D22046FEF78AF8BDE8F08101
:1027B0004E414E006E616E00494E4600696E6600E5
:1027C0002DE9F047814616468AB0354878440DC851
:1027D0008DE80D0032487844801C03AC0DC884E8B5
:1027E0000D0041F69B300844372190FBF1F290FB3D
:1027F000F1F5A5F1800501FB12041B3C02D56442F2
:10280000012000E00020DFF898A080460027FA446D
:10281000AAF1BE0A0EE0E0070AD03246684607EB8E
:10282000470101230AEB810111F054FA8DE80700FA
:1028300064107F1C002CEED1194F7F44AE3F19E08D
:10284000E80715D007EB04100DF1180A90E80E0008
:102850008AE80E00C068F04201D19819089032460B
:10286000012306A903A811F035FA03AB83E807009A
:102870006D10641C002DE3D14FF001033246694610
:10288000B8F1000F03A802D011F0FAF901E011F03D
:1028900021FAC9E90001C9F808200AB0BDE8F087AB
:1028A000EC20010010B50446AFF300802046BDE8DF
:1028B0001040FDF780BD000030B44FF0013C50F8EF
:1028C000042B51F8043BCCFA52F4D51A20D1FCB9B0
:1028D00050F8042B51F8043BCCFA52F4D51A17D116
:1028E000B4B950F8042B51F8043BCCFA52F4D51A81
:1028F0000ED16CB950F8042B51F8043BCCFA52F4C9
:10290000D51A05D1002CDAD030BC4FF0000070474A
:1029100029BAB1FA81F111F01801D1F120008440F7
:10292000F2D1CA40CB4012F0FF0213F0FF0330BCDB
:10293000D01A70472DE9FF4F1F464FF03C0987B072
:102940004FF00042DDE9141001F10108DDF858A054
:1029500002EA405003900020059083460546044655
:102960000490B969461E08988847AAF1010A0290A6
:10297000BAF1000F3BDD02982E2815D01021FFF789
:10298000FDF900282EDB4FF0010B0599014317D00C
:10299000B9F1000F0BDB4A46C117FFF7BDFE054337
:1029A0000C43A9F1040905E0012004900BE008B1F3
:1029B00045F0010501200590049820B9361D02E07C
:1029C000049800B1361FB969089808F101088847D2
:1029D000BBF1000FAAF1010A0290C9D00999C1F810
:1029E0000080C5E70298702808D0502806D0F96901
:1029F00008988847BBF1000F14D04FE000200290E8
:102A00000120BBF1000F049009D0B969089808F1C2
:102A100001088847AAF10109B9F1000F07DCF9693B
:102A2000089888476FF001000BB0BDE8F08F2B28A5
:102A300004D02D280CD14FF0FF300490B9690898CC
:102A400008F101088847A9F10109B9F1000FE6DD95
:102A5000411CE4D00A21FFF791F90028DFDB02993D
:102A600008F1010801EB810100EB41000290B96916
:102A7000089888470A21FFF781F9099AA9F1010905
:102A8000B9F1000FC2F8008001DD0028E7DAF9692A
:102A9000089888470499029800FB016655EA0400EB
:102AA00004D004F04041090002D006E0039898E009
:102AB000A40044EA9574AD00B61E04F0004108007D
:102AC00002D16D196441761E159810F0240F03D0C1
:102AD0004FF00B095C4803E04FF028096FF07D00D0
:102AE0008246564507DAAAEB06018944B9F1410F3F
:102AF00001DD4FF0410901200021A9F10102FFF79A
:102B00000BFE024628400B462140084301D001211C
:102B100000E00021501E029143F1FF312840214086
:102B2000084301D0012000E000200299834651EAC9
:102B30000B014FD0002108464FF00000039900F42C
:102B4000400039B100EB80004FF4400100EBD07041
:102B500001EA60008015012802DD4FF0FF3000E03F
:102B600013D0401C36D0029860B3BBF1000F0CD1DB
:102B70004A4601200021FFF7CFFD284021400843AD
:102B800001D0012000E00020E0B101204A460021F0
:102B9000FFF7C2FD034640190A4661412D1A8C41D8
:102BA00011D3B9F1400F09DD159810F0240F02D0B0
:102BB000AAF1340603E0AAF1170600E0761C00250E
:102BC0004FF0004406E05B1E42F1FF3220EA0305AD
:102BD00021EA0204CAF10100B04206DA1B49039857
:102BE00008430190002000900EE0039AC4F3D32123
:102BF000E80A0A43164940EA44500A433146CDE9FF
:102C00000002684611F0D9FA159810F0240F0BD085
:102C10001598C00715D13868DDE90012031D3B6027
:102C20000068C0E900120CE002A8694611F0BCFA85
:102C30001598C00705D13868029A011D39600068EF
:102C400002604046F0E6000002FCFFFF0000F07F5B
:102C50000000F03F2DE9FF4F92461D4685B04FF032
:102C60000041DDE9124BDDE914727F1E01EA4B5091
:102C7000414940F0FF4940EA0108002122F02000CC
:102C80004928049102D04E2828D04CE03BA00126D0
:102C900007C88DE80700A9690698641C88477F1E4D
:102CA000014606D41DF8060018B121F0200181422A
:102CB0000BD0E96906988847032E34D0082E32D00D
:102CC0006FF0010009B0BDE8F08F761C032E01D033
:102CD000082EE0D1601CCAF80000DCE7A96906985C
:102CE000641C88477F1E2AD420F02000412826D16A
:102CF000A9690698641C88477F1E20D420F0200014
:102D00004E281CD1A9690698641C88477F1E48F488
:102D1000002849F48009CAF8004001D4282806D0C8
:102D2000E969069888475FEACB7012D022E0A9696A
:102D30000698641C88477F1E01D4002803DAE969DD
:102D400006988847BCE72928F1D1641CCAF80040DE
:102D5000E9E71BF0240F07D028680499031D2B60B6
:102D60000068C0E9001805E02868021D2A600068B4
:102D7000C0F800902046A5E70000F07F494E464984
:102D80004E4954590000000001491820ABBEFEE72F
:102D9000260002007047000080B58AB0089044F613
:102DA0007810C0F601000AF029FE6946B02088615B
:102DB0000120486100230B610A20C86088604FF43D
:102DC0000060486040F65810C2F20000086041F20E
:102DD0005810C2F2000044F6C111C0F6010143F2DE
:102DE0000562C0F6010210F0D9FA0790079818B1F1
:102DF000FFE70798099059E06946B02088610120F3
:102E0000486100230B610A20C86088604FF40060AD
:102E1000486041F2C040C2F20000086041F6C04084
:102E2000C2F2000044F6CF11C0F6010143F23D6248
:102E3000C0F6010210F0B2FA0790079850B1FFE710
:102E4000079944F61410C0F601000AF0D7FD079860
:102E500009902BE06946382048604FF420700860E4
:102E600041F20820C2F2000044F6DD11C0F6010173
:102E700041F24023C2F20003102210F069F90790DA
:102E8000079850B1FFE7079944F64310C0F60100D8
:102E90000AF0B4FD0798099008E044F69210C0F6D5
:102EA00001000AF0ABFD00200990FFE709980AB085
:102EB00080BD0000FFE7FEE785B004900498006A3B
:102EC000039004980068406920F443000399084384
:102ED000049909684861049B1A6958699969DB6912
:102EE00018431043084303900498016801205022BE
:102EF000C4F202029142029000F06781FFE7049859
:102F0000016801205022C5F202029142029000F0B5
:102F10005C81FFE7049801680120D022C4F202021C
:102F20009142029000F05181FFE70498016801206E
:102F3000D022C5F202029142029000F04681FFE7E2
:102F400004980168012040F25012C4F2020291423A
:102F5000029000F03A81FFE704980168012040F2F6
:102F60005012C5F202029142029000F02E81FFE75A
:102F700004980168012040F2D012C4F2020291428A
:102F8000029000F02281FFE704980168012040F2DE
:102F9000D012C5F202029142029000F01681FFE7C2
:102FA00004980168012040F25022C4F202029142CA
:102FB000029000F00A81FFE704980168012040F2C6
:102FC0005022C5F202029142029000F0FE80FFE71B
:102FD00004980168012040F2D022C4F2020291421A
:102FE000029000F0F280FFE704980168012040F2AF
:102FF000D022C5F202029142029000F0E680FFE783
:1030000004980168012040F25032C4F20202914259
:10301000029000F0DA80FFE704980168012040F296
:103020005032C5F202029142029000F0CE80FFE7DA
:1030300004980168012040F2D032C4F202029142A9
:10304000029000F0C280FFE704980168012040F27E
:10305000D032C5F202029142029000F0B680FFE742
:1030600004980168012041F25002C4F20202914228
:10307000029000F0AA80FFE704980168012041F265
:103080005002C5F202029142029000F09E80FFE7DA
:1030900004980168012041F2D002C4F20202914278
:1030A000029000F09280FFE704980168012041F24D
:1030B000D002C5F202029142029000F08680FFE742
:1030C00004980168012041F25012C4F202029142B8
:1030D00002907AD0FFE704980168012041F2501273
:1030E000C5F20202914202906FD0FFE70498016896
:1030F000012041F2D012C4F202029142029064D047
:10310000FFE704980168012041F2D012C5F20202E3
:103110009142029059D0FFE704980168012041F2E2
:103120005022C4F20202914202904ED0FFE704986E
:103130000168012041F25022C5F202029142029040
:1031400043D0FFE704980168012041F2D022C4F285
:1031500002029142029038D0FFE7049801680120F2
:1031600041F2D022C5F20202914202902DD0FFE737
:1031700004980168012041F25032C4F202029142E7
:10318000029022D0FFE704980168012041F25032FA
:10319000C5F202029142029017D0FFE7049801683D
:1031A000012041F2D032C4F20202914202900CD0CE
:1031B000FFE7049800684EF63041CAF6FD710844F6
:1031C000B0FA80F040090290FFE70298C007B8B15A
:1031D000FFE70498426A836AC06A0021CFF6F07163
:1031E00001EB035101F07C7108436FF00F0101EB1B
:1031F000021101F47C710143039808430390FFE737
:1032000004980068006C00F080200399084304993A
:1032100009680864049988680A791043096B0843AF
:1032200003900498C068B0F5806F40F07C81FFE7A0
:103230000498016801205022C4F2020291420190D8
:1032400000F06781FFE70498016801205022C5F271
:1032500002029142019000F05C81FFE7049801684E
:103260000120D022C4F202029142019000F051816B
:10327000FFE7049801680120D022C5F202029142C2
:10328000019000F04681FFE704980168012040F2B8
:103290005012C4F202029142019000F03A81FFE71D
:1032A00004980168012040F25012C5F202029142D6
:1032B000019000F02E81FFE704980168012040F2A0
:1032C000D012C4F202029142019000F02281FFE785
:1032D00004980168012040F2D012C5F20202914226
:1032E000019000F01681FFE704980168012040F288
:1032F0005022C4F202029142019000F00A81FFE7DD
:1033000004980168012040F25022C5F20202914265
:10331000019000F0FE80FFE704980168012040F270
:10332000D022C4F202029142019000F0F280FFE745
:1033300004980168012040F2D022C5F202029142B5
:10334000019000F0E680FFE704980168012040F258
:103350005032C4F202029142019000F0DA80FFE79D
:1033600004980168012040F25032C5F202029142F5
:10337000019000F0CE80FFE704980168012040F240
:10338000D032C4F202029142019000F0C280FFE705
:1033900004980168012040F2D032C5F20202914245
:1033A000019000F0B680FFE704980168012041F227
:1033B0005002C4F202029142019000F0AA80FFE79D
:1033C00004980168012041F25002C5F202029142C4
:1033D000019000F09E80FFE704980168012041F20F
:1033E000D002C4F202029142019000F09280FFE705
:1033F00004980168012041F2D002C5F20202914214
:10340000019000F08680FFE704980168012041F2F6
:103410005012C4F20202914201907AD0FFE7049860
:103420000168012041F25012C5F20202914201905E
:103430006FD0FFE704980168012041F2D012C4F276
:1034400002029142019064D0FFE7049801680120D4
:1034500041F2D012C5F202029142019059D0FFE729
:1034600004980168012041F25022C4F20202914204
:1034700001904ED0FFE704980168012041F25022EC
:10348000C5F202029142019043D0FFE7049801681F
:10349000012041F2D022C4F202029142019038D0C0
:1034A000FFE704980168012041F2D022C5F2020230
:1034B000914201902DD0FFE704980168012041F26C
:1034C0005032C4F202029142019022D0FFE70498E8
:1034D0000168012041F25032C5F20202914201908E
:1034E00017D0FFE704980168012041F2D032C4F2FE
:1034F0000202914201900CD0FFE7049800684EF65A
:103500003041CAF6FD710844B0FA80F040090190DC
:10351000FFE70198C00728B1FFE7039840F48060F7
:103520000390FFE70CE00498C068B0F5007F05D178
:10353000FFE7039840F40070039000E0FFE7FFE727
:103540000498416B03980843039004980068406C0A
:1035500042F20011C3F6C0410840039908430499A0
:103560000968486404980168002088640498016828
:10357000012040F25032C4F20202914200904ED03B
:10358000FFE704980168012040F25032C5F20202C0
:103590009142009043D0FFE704980168012040F277
:1035A000D032C4F202029142009038D0FFE7049872
:1035B0000168012040F2D032C5F20202914200902F
:1035C0002DD0FFE704980168012041F25032C4F287
:1035D00002029142009022D0FFE704980168012086
:1035E00041F25032C5F202029142009017D0FFE73B
:1035F00004980168012041F2D032C4F202029142E3
:1036000000900CD0FFE7049800684EF63041CAF6EF
:10361000FD710844B0FA80F040090090FFE700987F
:10362000C00740B1FFE7049801680020486504998D
:1036300009688865FFE7049801680020C86705B03D
:103640007047000083B002900191029B1A6958698B
:103650009969D3F81CC040EA0C00DB6B1843104397
:1036600008430199086002980078800600281BD55D
:10367000FFE702994A6A8B6AC86A896B084300218E
:10368000CFF6F07101EB035101F07C7108436FF04C
:103690000F0101EB021101F47C7140EA0102019972
:1036A000086810430860FFE702984168006B40F229
:1036B000FF2211400843019948600298C068B0F5A4
:1036C000806F0DD1FFE7029800788006002806D5AC
:1036D000FFE70199486840F480604860FFE70DE02B
:1036E0000298C068B0F5007F06D1FFE701994868ED
:1036F00040F40070486000E0FFE7FFE70298426B8B
:1037000001994868104348600298406C70B1FFE727
:103710000299086C4A6C896C104301F03F0140EA41
:1037200001420199486810434860FFE70298B0F8E9
:10373000680001998860029800788007002859D5B0
:10374000FFE70298C16C0020CFF6FF7000EB01404C
:103750000021C0F2FF7100EA01020199886810435C
:1037600088600298006DB0F1FF3F06DCFFE7019929
:10377000886840F08050886005E00199886820F0F2
:1037800080508860FFE70298406DB0F1FF3F06DC93
:10379000FFE70199886840F00050886005E00199D2
:1037A000886820F000508860FFE70298806DB0F1D3
:1037B000FF3F06DCFFE70199886840F080408860A1
:1037C00005E00199886820F080408860FFE7029852
:1037D000C06DB0F1FF3F06DCFFE70199886840F05B
:1037E0000040886005E00199886820F0004088600A
:1037F000FFE7FFE70298006E0199C8600298406EEB
:103800000199086102980078800700286AD5FFE7CF
:103810000298006DB0F1FF3F0ADCFFE70298006DEF
:103820004042009000986FF35F300199486106E0D4
:103830000298006D6FF35F3001994861FFE70298CD
:10384000406DB0F1FF3F0FDCFFE70298406D404252
:10385000009000990020C1F6FF7000EA0142019932
:103860004869104348610BE00298416D0020C1F6A1
:10387000FF7000EA01420199486910434861FFE77F
:103880000298806DB0F1FF3F09DCFFE70298806D80
:1038900040420090BDF800000199886105E002985F
:1038A000B0F8580001998861FFE70298C06DB0F147
:1038B000FF3F0BDCFFE70298C06D40420090009A8A
:1038C0000199886940EA0240886107E00298C26D68
:1038D0000199886940EA02408861FFE70199002068
:1038E000C86103E0019900204861FFE70298006881
:1038F00001990862029800788007002806D5FFE742
:103900000199086A40F4E060086205E00199086ADC
:1039100040F4A0600862FFE703B0704786B00490EF
:1039200003910292049803990843029908434FF6C1
:10393000FF718843019000200090049818B1FFE7C0
:10394000049800900EE0039818B1FFE703980090E8
:1039500007E0029818B1FFE70298009000E0FFE747
:10396000FFE7FFE70198BDF80210B0EB014F03D06D
:10397000FFE70120059002E000200590FFE7059891
:1039800006B0704785B0039002910192002000902C
:10399000039828B1FFE7039890F82000009012E008
:1039A000029828B1FFE7029890F82000009009E003
:1039B000019828B1FFE7019890F82000009000E0FE
:1039C000FFE7FFE7FFE7029858B1FFE70098029989
:1039D00091F82010884203D0FFE70220049011E004
:1039E000FFE7019858B1FFE70098019991F820107E
:1039F000884203D0FFE70320049003E0FFE70020A4
:103A00000490FFE7049805B07047000089B0079064
:103A1000069105920020049003900290059800689A
:103A20000190069828BBFFE7FFE70498079989688B
:103A300088421DD2FFE7049838B9FFE7079800686D
:103A40004FF6FC71084003900EE003980290039833
:103A50000799498800EB0140019950F821004FF681
:103A6000FC7108400390FFE7049801300490DCE704
:103A700034E0FFE7049907988268002091420090A3
:103A80000AD2FFE7039806994FF6FC721140401ADC
:103A900018BF01200090FFE70098C007E8B1FFE7DA
:103AA000049838B9FFE7079800684FF6FC710840A2
:103AB00003900EE00398029003980799498800EB61
:103AC0000140019950F821004FF6FC710840039025
:103AD000FFE7049801300490CCE7FFE7069860B157
:103AE000FFE7039806994FF6FC721140884203D015
:103AF000FFE70120089029E0FFE704980599886016
:103B000002980799498840EA01400599486003985E
:103B10000799498840EA01400599C8600598C0683E
:103B2000019950F8210070B1FFE70599C868019A22
:103B300050F822004FF6FC721040079A528840EA73
:103B400002400861FFE700200890FFE7089809B0ED
:103B50007047000083B0029001910092029890F8A3
:103B600020008007002811D5FFE7019830B1FFE75A
:103B700001990020CFF601600860FFE7009820B1AE
:103B8000FFE7009907200860FFE710E0019830B1D7
:103B9000FFE701990020CFF601000860FFE70098D9
:103BA00020B1FFE7009905200860FFE7FFE703B0B9
:103BB0007047000084B003900399886BC96B084379
:103BC00002900398016801205022C4F2020291423F
:103BD000019000F06781FFE70398016801205022FF
:103BE000C5F202029142019000F05C81FFE7039868
:103BF00001680120D022C4F202029142019000F03B
:103C00005181FFE7039801680120D022C5F202022A
:103C10009142019000F04681FFE70398016801207E
:103C200040F25012C4F202029142019000F03A8137
:103C3000FFE703980168012040F25012C5F202022A
:103C40009142019000F02E81FFE703980168012066
:103C500040F2D012C4F202029142019000F022819F
:103C6000FFE703980168012040F2D012C5F202027A
:103C70009142019000F01681FFE70398016801204E
:103C800040F25022C4F202029142019000F00A81F7
:103C9000FFE703980168012040F25022C5F20202BA
:103CA0009142019000F0FE80FFE703980168012037
:103CB00040F2D022C4F202029142019000F0F28060
:103CC000FFE703980168012040F2D022C5F202020A
:103CD0009142019000F0E680FFE70398016801201F
:103CE00040F25032C4F202029142019000F0DA80B8
:103CF000FFE703980168012040F25032C5F202024A
:103D00009142019000F0CE80FFE703980168012006
:103D100040F2D032C4F202029142019000F0C2801F
:103D2000FFE703980168012040F2D032C5F2020299
:103D30009142019000F0B680FFE7039801680120EE
:103D400041F25002C4F202029142019000F0AA80B6
:103D5000FFE703980168012041F25002C5F2020218
:103D60009142019000F09E80FFE7039801680120D6
:103D700041F2D002C4F202029142019000F092801E
:103D8000FFE703980168012041F2D002C5F2020268
:103D90009142019000F08680FFE7039801680120BE
:103DA00041F25012C4F20202914201907AD0FFE730
:103DB00003980168012041F25012C5F202029142BB
:103DC00001906FD0FFE703980168012041F2D01203
:103DD000C4F202029142019064D0FFE703980168A7
:103DE000012041F2D012C5F202029142019059D055
:103DF000FFE703980168012041F25022C4F2020259
:103E0000914201904ED0FFE703980168012041F2F2
:103E10005022C5F202029142019043D0FFE703987D
:103E20000168012041F2D022C4F2020291420190C5
:103E300038D0FFE703980168012041F2D022C5F293
:103E40000202914201902DD0FFE703980168012002
:103E500041F25032C4F202029142019022D0FFE7B7
:103E600003980168012041F25032C5F202029142EA
:103E7000019017D0FFE703980168012041F2D0328A
:103E8000C4F20202914201900CD0FFE7039800684F
:103E90004EF63041CAF6FD710844B0FA80F0400990
:103EA0000190FFE70198C00730B1FFE70398016C6C
:103EB000029808430290FFE703980068406920F4E5
:103EC000430002990843039909684861039801680F
:103ED0000020086403990A68496C516403990968D1
:103EE000886403990968C864039909680865039898
:103EF0000168012040F25032C4F202029142009067
:103F00004ED0FFE703980168012040F25032C5F21D
:103F100002029142009043D0FFE70398016801201C
:103F200040F2D032C4F202029142009038D0FFE752
:103F300003980168012040F2D032C5F2020291429A
:103F400000902DD0FFE703980168012041F2503224
:103F5000C4F202029142009022D0FFE70398016868
:103F6000012041F25032C5F202029142009017D076
:103F7000FFE703980168012041F2D032C4F2020247
:103F8000914200900CD0FFE7039800684EF6304154
:103F9000CAF6FD710844B0FA80F040090090FFE7CE
:103FA0000098C00740B1FFE703980168002048650A
:103FB000039909688865FFE7039801680020C867CE
:103FC00004B0704784B0039002910192009303986B
:103FD0000068806C4FF6FF718843BDF800100844FC
:103FE000039909688864039801684FF4FE40C8602B
:103FF000029803990968C8640198039909680865DB
:1040000004B070477047000072B6FFE7FEE700009B
:1040100080B541F67C50C2F2000000F09BFD80BDEF
:1040200080B541F6F450C2F2000000F093FD80BD6F
:1040300080B541F66C60C2F2000000F08BFD80BDDF
:1040400080B584B002900191029818B1FFE7019801
:1040500020B9FFE701208DF80F001AE002980078E0
:104060008006002801D5FFE7FFE70298406C08B101
:10407000FFE7FFE7029800788007002801D5FFE7F7
:10408000FFE702980199FFF7DDFA00208DF80F0095
:10409000FFE79DF80F0004B080BD000080B584B03C
:1040A000029001F09FFA0190029820B9FFE70120E9
:1040B0008DF80F00AFE10298016801205022C4F290
:1040C00002029142009000F06781FFE702980168C8
:1040D00001205022C5F202029142009000F05C8162
:1040E000FFE7029801680120D022C4F20202914247
:1040F000009000F05181FFE7029801680120D02272
:10410000C5F202029142009000F04681FFE702985A
:104110000168012040F25012C4F202029142009064
:1041200000F03A81FFE702980168012040F2501246
:10413000C5F202029142009000F02E81FFE7029842
:104140000168012040F2D012C4F2020291420090B4
:1041500000F02281FFE702980168012040F2D012AE
:10416000C5F202029142009000F01681FFE702982A
:104170000168012040F25022C4F2020291420090F4
:1041800000F00A81FFE702980168012040F2502206
:10419000C5F202029142009000F0FE80FFE7029813
:1041A0000168012040F2D022C4F202029142009044
:1041B00000F0F280FFE702980168012040F2D0226F
:1041C000C5F202029142009000F0E680FFE70298FB
:1041D0000168012040F25032C4F202029142009084
:1041E00000F0DA80FFE702980168012040F25032C7
:1041F000C5F202029142009000F0CE80FFE70298E3
:104200000168012040F2D032C4F2020291420090D3
:1042100000F0C280FFE702980168012040F2D0322E
:10422000C5F202029142009000F0B680FFE70298CA
:104230000168012041F25002C4F202029142009052
:1042400000F0AA80FFE702980168012041F25002C5
:10425000C5F202029142009000F09E80FFE70298B2
:104260000168012041F2D002C4F2020291420090A2
:1042700000F09280FFE702980168012041F2D0022D
:10428000C5F202029142009000F08680FFE702989A
:104290000168012041F25012C4F2020291420090E2
:1042A0007AD0FFE702980168012041F25012C5F26E
:1042B0000202914200906FD0FFE70298016801204E
:1042C00041F2D012C4F202029142009064D0FFE7A2
:1042D00002980168012041F2D012C5F20202914217
:1042E000009059D0FFE702980168012041F2502266
:1042F000C4F20202914200904ED0FFE7029801689A
:10430000012041F25022C5F202029142009043D0B6
:10431000FFE702980168012041F2D022C4F20202B4
:104320009142009038D0FFE702980168012041F2E5
:10433000D022C5F20202914200902DD0FFE70298F0
:104340000168012041F25032C4F202029142009011
:1043500022D0FFE702980168012041F25032C5F2F5
:1043600002029142009017D0FFE7029801680120F5
:1043700041F2D032C4F20202914200900CD0FFE729
:10438000029800684EF63041CAF6FD710844B0FA52
:1043900080F040090090FFE70098C00708B1FFE7F0
:1043A000FFE7FFE70299002081F84C00FFE7029940
:1043B000022081F8540002980168486940F0060024
:1043C0004861FFE7029800684069C00798B1FFE7BD
:1043D00001F008F90199401A06280BD3FFE702996A
:1043E000102088650299032081F8540001208DF87F
:1043F0000F0010E0E6E70298FFF7DCFB0299886CFB
:104400000865029900208865029A012182F85410FB
:104410008DF80F00FFE79DF80F0004B080BD00008D
:1044200080B58CB00A90099108920A9818B1FFE7FC
:10443000089820B9FFE701208DF82F00B9E00A980D
:104440004069012807D1FFE70A990420086101208B
:104450008DF82F00ADE00A9800680999089AFFF7D7
:104460005DFA38B1FFE70A990520086101208DF84F
:104470002F009EE00A9800680999089AFFF782FACF
:1044800038B1FFE70A990420086101208DF82F0058
:104490008FE00A99022008730A99002008610898A1
:1044A00007A906AAFFF756FB0A980068E0B9FFE7DC
:1044B000099838B9FFE708980A9908600A99012015
:1044C000886010E009980A99086008984FF6FC7116
:1044D0000840079908430999069A41F822000A9969
:1044E00002208860FFE75BE0099878B9FFE70A9847
:1044F00000684FF6FC710840079908430899069A2E
:1045000041F8220008980A99086044E00698019052
:104510000A98099901AAFFF779FAA0BBFFE7039867
:104520000A99896888421BD1FFE70A98406860B100
:10453000FFE70A9840684FF6FC7108400799084366
:104540000899069A41F82200FFE708984FF6FC7197
:104550000840079908430999069A41F8220011E09A
:104560000998069A50F82200089941F82200089804
:104570004FF6FC710840079908430999069A41F8DB
:104580002200FFE706E00A990620086101208DF865
:104590002F000EE0FFE70A99886801308860FFE786
:1045A0000A99002008610A9A012111738DF82F00E1
:1045B000FFE79DF82F000CB080BD000085B0039090
:1045C0000291039818B1FFE7029820B9FFE7012094
:1045D0008DF81300BFE00398006D20B9FFE70120BC
:1045E0008DF81300B7E0039890F854008DF8070099
:1045F000039890F85400022805D0FFE79DF80700C3
:1046000005280DD1FFE7039940208865FFE703994E
:10461000002081F84C00FFE701208DF813009AE09C
:104620000298007B022806D1FFE702990120086169
:104630008DF813008FE003980168012040F250329A
:10464000C4F20202914200904ED0FFE70398016845
:10465000012040F25032C5F202029142009043D054
:10466000FFE703980168012040F2D032C4F2020251
:104670009142009038D0FFE703980168012040F292
:10468000D032C5F20202914200902DD0FFE703988C
:104690000168012041F25032C4F2020291420090BE
:1046A00022D0FFE703980168012041F25032C5F2A1
:1046B00002029142009017D0FFE7039801680120A1
:1046C00041F2D032C4F20202914200900CD0FFE7D6
:1046D000039800684EF63041CAF6FD710844B0FAFE
:1046E00080F040090090FFE70098C00778B9FFE725
:1046F0000298006890F820008007002807D5FFE79F
:1047000002990320086101208DF8130023E003982B
:10471000006D81280CD1FFE70298406838B9FFE7A7
:1047200002990420086101208DF8130013E00BE0CA
:104730000298406838B1FFE702990420086101201F
:104740008DF8130007E0FFE70298039948670020FF
:104750008DF81300FFE79DF8130005B070470000C7
:1047600080B58AB00890089820B9FFE701208DF83D
:10477000270056E00898006838B9FFE7089902203A
:10478000086101208DF827004BE00898406888B147
:10479000FFE7089801684068884204D1FFE70020DD
:1047A0008DF827003DE008990420086101208DF86C
:1047B000270036E008984069012807D1FFE70899EB
:1047C0000420086101208DF827002AE008990220C2
:1047D000087308990020009008610898006807A9EC
:1047E00006AAFFF7B7F9009906980190089801AA60
:1047F000FFF70CF90098089909684FF6FC72114010
:10480000079A1143049A069B42F82310089A1168EC
:10481000516008990861089A012111738DF82700E9
:10482000FFE79DF827000AB080BD000080B586B084
:104830000490049820B1FFE70498406F20B9FFE787
:1048400001208DF8170090E00498006D20B9FFE773
:1048500001208DF8170088E0049890F854008DF836
:104860000F0004980068406900F4803002909DF8C1
:104870000F00012809D0FFE79DF80F00022863D13F
:10488000FFE7029800285FD0FFE7049890F85400F3
:10489000012852D1FFE7FFE7049890F84C00012867
:1048A00004D1FFE702208DF817005EE00499012093
:1048B00081F84C00FFE7FFE70499022081F85400DB
:1048C0000499496F08730499002088650499496F19
:1048D000086104980168486940F4BA404861049846
:1048E000406E38B1FFE704980168486940F40070F1
:1048F0004861FFE70498006F38B1FFE7049801684A
:10490000486940F400504861FFE70498406F006830
:1049100001A90022FFF71EF904980168406F408842
:104920000004086004980168406F00684FF6FC724C
:104930001040019A1043C867FFE70498016848696E
:1049400040F0010048610CE0049940208865FFE7D1
:104950000499002081F84C00FFE701208DF8170032
:1049600003E000208DF81700FFE79DF8170006B060
:1049700080BD000080B584B0029000F033FE01904D
:10498000029820B9FFE701208DF80F0079E0029826
:1049900090F8540002280DD0FFE702992020886586
:1049A000FFE70299002081F84C00FFE701208DF815
:1049B0000F0066E002980168486940F00400486111
:1049C0000299052081F85400FFE702980068006909
:1049D0008004002827D4FFE700F004FE0199401A64
:1049E00006281FD3FFE70299886D40F01000886504
:1049F0000299032081F85400029890F850000006B4
:104A0000002805D5FFE70298416F01200873FFE7F2
:104A1000FFE70299002081F84C00FFE701208DF8A4
:104A20000F002EE0D1E702980168486940F00200CB
:104A300048610299042081F85400029801684FF4FB
:104A4000FE40C8600299012081F85400029890F855
:104A500050000006002809D5FFE70298416F0120A9
:104A600008730298016800208864FFE7FFE7029955
:104A7000002081F84C00FFE7FFE700208DF80F00D1
:104A8000FFE79DF80F0004B080BD000082B00090E9
:104A9000009820B9FFE701208DF807001CE000987E
:104AA00090F85400022807D0FFE70099202088657D
:104AB00001208DF807000FE00099042081F85400D0
:104AC00000980168486942F2040210434861FFE718
:104AD00000208DF80700FFE79DF8070002B070473F
:104AE00085B003900291039820B9FFE701208DF86B
:104AF00013002AE00398006840F6FF718843019094
:104B0000039800685038C0F3C41101208840009019
:104B10009DF80800C006002813D5FFE7029800F0B2
:104B20001100112806D1FFE7009A01994868104347
:104B3000486005E0009A0199486890434860FFE7A3
:104B4000FFE700208DF81300FFE79DF8130005B084
:104B50007047000080B584B003900398006840F669
:104B6000FF7188430290039800685038C0F3C41165
:104B70000120884001900298C06801990840009087
:104B8000009808B9FFE74DE1039800680069400507
:104B9000002813D5FFE70398006840694005002806
:104BA0000BD5FFE7039801684FF48060C860039954
:104BB000886D40F001008865FFE7FFE70398006813
:104BC00000690005002813D5FFE7039800684069D5
:104BD000000500280BD5FFE7039801684FF400603B
:104BE000C8600399886D40F002008865FFE7FFE721
:104BF000039800680069C004002813D5FFE70398F4
:104C000000684069C00400280BD5FFE703980168DD
:104C10004FF48050C8600399886D40F004008865A7
:104C2000FFE7FFE70398006800694004002813D5F8
:104C3000FFE7039800684069400400280BD5FFE7B0
:104C4000039801684FF48040C8600399886D40F074
:104C500008008865FFE7FFE70398006800698005A2
:104C6000002816D5FFE703980068406980050028F2
:104C70000ED5FFE7039801684FF40070C8600398F1
:104C8000406E20B1FFE70398416E8847FFE7FFE7DA
:104C9000FFE70398006800698004002850D5FFE70B
:104CA0000398006840698004002848D5FFE703980E
:104CB00001684FF40050C860039890F8540004282D
:104CC0002FD1FFE703980168486920F4005048613C
:104CD00003980168486940F0020048610399012087
:104CE00081F85400039890F850000006002809D578
:104CF000FFE70398416F01200873039801680020C3
:104D00008864FFE7FFE70399002081F84C00FFE784
:104D10000398C06E20B1FFE70398C16E8847FFE794
:104D200080E00399052081F854000398006F20B1BA
:104D3000FFE70398016F8847FFE7FFE7FFE7FFE71B
:104D4000039800680069C005002842D5FFE7039872
:104D500000684069C00500283AD5FFE7039890F83D
:104D600050000006002814D5FFE703980068C06FC4
:104D700070B9FFE703980068806C40B9FFE70399BA
:104D8000012081F854000399496F0873FFE7FFE79A
:104D90000AE003980068806C28B9FFE703990120B6
:104DA00081F85400FFE7FFE7039801684FF4407073
:104DB000C860FFE70399002081F84C00FFE70398E3
:104DC000006E20B1FFE70398016E8847FFE7FFE719
:104DD000FFE70398806D28B3FFE7039801684869EF
:104DE00040F0020048610399012081F854000398C3
:104DF00090F850000006002805D5FFE70398416FA2
:104E000001200873FFE7FFE70399002081F84C00B9
:104E1000FFE70398806E20B1FFE70398816E884713
:104E2000FFE7FFE704B080BD80B584B0029000F0DA
:104E3000D9FB0190029820B9FFE701208DF80F00FF
:104E4000CEE10298C068B0F5007F01D0FFE7FFE730
:104E50000298406BB0F5805F01D1FFE7FFE7029851
:104E6000016801205022C4F202029142009000F039
:104E70006781FFE70298016801205022C5F2020213
:104E80009142009000F05C81FFE7029801680120E8
:104E9000D022C4F202029142009000F05181FFE75B
:104EA000029801680120D022C5F2020291420090CE
:104EB00000F04681FFE702980168012040F250129D
:104EC000C4F202029142009000F03A81FFE702989A
:104ED0000168012040F25012C5F202029142009096
:104EE00000F02E81FFE702980168012040F2D01205
:104EF000C4F202029142009000F02281FFE7029882
:104F00000168012040F2D012C5F2020291420090E5
:104F100000F01681FFE702980168012040F250225C
:104F2000C4F202029142009000F00A81FFE7029869
:104F30000168012040F25022C5F202029142009025
:104F400000F0FE80FFE702980168012040F2D022C5
:104F5000C4F202029142009000F0F280FFE7029852
:104F60000168012040F2D022C5F202029142009075
:104F700000F0E680FFE702980168012040F250321D
:104F8000C4F202029142009000F0DA80FFE702983A
:104F90000168012040F25032C5F2020291420090B5
:104FA00000F0CE80FFE702980168012040F2D03285
:104FB000C4F202029142009000F0C280FFE7029822
:104FC0000168012040F2D032C5F202029142009005
:104FD00000F0B680FFE702980168012041F250021C
:104FE000C4F202029142009000F0AA80FFE702980A
:104FF0000168012041F25002C5F202029142009084
:1050000000F09E80FFE702980168012041F2D00283
:10501000C4F202029142009000F09280FFE70298F1
:105020000168012041F2D002C5F2020291420090D3
:1050300000F08680FFE702980168012041F25012DB
:10504000C4F20202914200907AD0FFE70298016810
:10505000012041F25012C5F20202914200906FD03D
:10506000FFE702980168012041F2D012C4F2020267
:105070009142009064D0FFE702980168012041F25C
:10508000D012C5F202029142009059D0FFE7029877
:105090000168012041F25022C4F2020291420090C4
:1050A0004ED0FFE702980168012041F25022C5F27C
:1050B00002029142009043D0FFE70298016801206C
:1050C00041F2D022C4F202029142009038D0FFE7B0
:1050D00002980168012041F2D022C5F202029142F9
:1050E00000902DD0FFE702980168012041F2503274
:1050F000C4F202029142009022D0FFE702980168B8
:10510000012041F25032C5F202029142009017D0C4
:10511000FFE702980168012041F2D032C4F2020296
:10512000914200900CD0FFE7029800684EF63041A3
:10513000CAF6FD710844B0FA80F040090090FFE71C
:105140000098C00708B1FFE7FFE7FFE702990020DA
:1051500081F84C00FFE7029890F8540060B9FFE72F
:1051600002990020086602994866029988660299A9
:10517000C86602990867FFE70299022081F8540087
:1051800002980168486940F006004861FFE702980C
:1051900000684069C00798B1FFE700F023FA019961
:1051A000401A06280BD3FFE7029910208865029960
:1051B000032081F8540001208DF80F0010E0E6E78D
:1051C0000298FDF779FE0299486B08650299002064
:1051D0008865029A012182F854108DF80F00FFE7CC
:1051E0009DF80F0004B080BD80B586B00490039197
:1051F00002920193049820B9FFE701208DF817006F
:105200005FE00498006D20B1FFE701208DF81700E2
:1052100057E0FFE7049890F84C00012804D1FFE71D
:1052200002208DF817004CE00499012081F84C0011
:10523000FFE7FFE7049890F85400012830D1FFE71A
:105240000499022081F8540004990020886504988C
:105250000399029A019BFEF7B5FE0498016848691C
:1052600040F4BA4048610498406E38B1FFE70498B2
:105270000168486940F400704861FFE70498006FD6
:1052800038B1FFE704980168486940F4005048616C
:10529000FFE704980168486940F0010048610CE0AC
:1052A000049940208865FFE70499002081F84C00AC
:1052B000FFE701208DF8170003E000208DF81700AC
:1052C000FFE79DF8170006B080BD000085B0049090
:1052D000039100200090FFE7039800680099C84000
:1052E000002800F06681FFE703980068009A01211A
:1052F0009140084001900198002800F05681FFE796
:1053000003984068022805D0FFE7039840681228F8
:1053100028D1FFE7049800996FF0030202EA5101D7
:105320000844006A0290009800F0070081000F20F6
:1053300000FA01F10298884302900398006900F096
:105340000F00009901F00701890000FA01F10298AD
:105350000843029002980499009B02EA5302114408
:105360000862FFE70498006802900098410003205B
:1053700000FA01F10298884302900398406800F017
:1053800003000099490000FA01F1029808430290D5
:105390000298049908600398406801280FD0FFE73D
:1053A0000398406802280AD0FFE703984068112854
:1053B00005D0FFE70398406812282FD1FFE7049833
:1053C0008068029000984100032000FA01F10298E1
:1053D000884302900398C0680099490000FA01F1DF
:1053E00002980843029002980499886004984068E3
:1053F00002900099012000FA01F10298884302907E
:1054000003984068C0F30010009900FA01F1029877
:1054100008430290029804994860FFE703984068A7
:1054200000F0030003280CD1FFE70398406800F068
:10543000030003281DD1FFE703988068012818D0D6
:10544000FFE70498C068029000984100032000FA2A
:1054500001F10298884302900398806800994900FE
:1054600000FA01F102980843029002980499C8607A
:10547000FFE70398C079C006002840F19580FFE758
:10548000009820F0030042F26002C4F20242805809
:105490000290009800F00300C1000F2000FA01F113
:1054A00002988843029004984FF60041CBF6FD51D4
:1054B0000840800A009901F00301C90000FA01F1D7
:1054C0000298084302900298009921F00301885045
:1054D00042F20000C4F20240006802900199029872
:1054E0008843029003988079C006002805D5FFE71D
:1054F0000199029808430290FFE7029842F20001E6
:10550000C4F20241086042F20400C4F202400068A2
:10551000029001990298884302900398807980064E
:10552000002805D5FFE70199029808430290FFE79C
:10553000029842F20401C4F20241086042F284007F
:10554000C4F20240006802900199029888430290D8
:10555000039880798007002805D5FFE70199029814
:1055600008430290FFE7029842F28401C4F202412C
:10557000086042F28000C4F2024000680290019983
:1055800002988843029003988079C00728B1FFE70A
:105590000199029808430290FFE7029842F28001C5
:1055A000C4F202410860FFE7FFE700980130009075
:1055B00092E605B07047000082B00190ADF802108D
:1055C0008DF801209DF8010028B1FFE7BDF8020029
:1055D0000199886104E0BDF8020001998862FFE743
:1055E00002B0704742F20C70C2F2000000687047CF
:1055F00040F20800C2F20000027842F20C71C2F2DE
:1056000000010868104408607047000080B582B04F
:10561000032000F0C1F805F005F940F62041C4F27E
:105620000241096801F00F0244F6D401C0F60101FD
:10563000895CC84040F20001C2F200010860042009
:1056400005F054FF0F2000F011F820B1FFE7012012
:105650008DF8070005E000F07BF800208DF80700CA
:10566000FFE79DF8070002B080BD000080B58EB056
:105670000D90FFE740F69C40C4F20240016841F003
:1056800010010160006800F0100001900198FFE730
:1056900007A803A905F03AF80A980590059820B9DB
:1056A000FFE705F083F8069004E005F07FF840007E
:1056B0000690FFE70698400945F6C521C0F67C2113
:1056C000A0FB01014FF0FF3000EBD110049042F23B
:1056D0001400C2F2000041F20001C4F200010160B6
:1056E0006321C1600499416000210161816006F07D
:1056F00071F88DF80B009DF80B0010BBFFE742F22C
:105700001400C2F2000006F041F98DF80B009DF87C
:105710000B00A8B9FFE70D980F280CD8FFE70D99EB
:105720003120002200F020F80D9840F20C01C2F266
:105730000001086003E001208DF80B00FFE7FFE7A0
:10574000FFE7312000F006F89DF80B000EB080BD99
:105750007047000080B582B0ADF80600BDF90600C4
:105760000BF0D4FB02B080BD80B586B0ADF816005A
:10577000049103920BF0E2FB0290BDF91600019038
:1057800002980499039A08F0FFFC014601980BF077
:10579000DDFB06B080BD000080B582B001900198AD
:1057A0000BF0F6FB02B080BD89B0089040F63440A3
:1057B000C4F2024000686FF35F20059040F6284075
:1057C000C4F20240016801F0030107910168C1F3CE
:1057D000052106910068C0F300100490049840F67B
:1057E0003841C4F20241096889B2C90800FB01F0DE
:1057F00000EE100AB8EE400A8DED020A0698002865
:1058000000F03D81FFE707980090012808D0FFE7EE
:105810000098022830D0FFE70098032849D065E0BF
:1058200040F60040C4F202400068C0F3C10149F2F2
:105830000000C0F2D030C84003909DED030AB8EEDE
:10584000400A9DED061AB8EE411A80EE010A9DED60
:10585000051AB8EE411A9DED022A9FED8F3A82EEAD
:10586000032A31EE021AB7EE002A31EE021A20EEB8
:10587000010A8DED010A65E09DED060AB8EE401AB9
:105880009FED860A80EE010A9DED051AB8EE411AD9
:105890009DED022A9FED803A82EE032A31EE021A34
:1058A000B7EE002A31EE021A20EE010A8DED010A50
:1058B00048E09DED060AB8EE401A9FED760A80EEAC
:1058C000010A9DED051AB8EE411A9DED022A9FEDE1
:1058D000723A82EE032A31EE021AB7EE002A31EE56
:1058E000021A20EE010A8DED010A2BE040F600407D
:1058F000C4F202400068C0F3C10149F20000C0F2E6
:10590000D030C84003909DED030AB8EE400A9DEDEB
:10591000061AB8EE411A80EE010A9DED051AB8EE9E
:10592000411A9DED022A9FED5C3A82EE032A31EE88
:10593000021AB7EE002A31EE021A20EE010A8DEDAE
:10594000010AFFE740F60040C4F20240006880010F
:10595000002827D5FFE740F62840C4F2024000683F
:10596000C003002819D5FFE79DED010A40F6344039
:10597000C4F20240006880B2400A01EE100AB8EE9C
:10598000411AB7EE002A31EE021A80EE010A089899
:10599000BCEEC00A80ED000A03E008990020086010
:1059A000FFE703E0089900200860FFE740F60040A9
:1059B000C4F2024000688001002827D5FFE740F6C6
:1059C0002840C4F2024000688003002819D5FFE790
:1059D0009DED010A40F63440C4F202400068C0F375
:1059E000064001EE100AB8EE411AB7EE002A31EE79
:1059F000021A80EE010A0898BCEEC00A80ED010A86
:105A000003E0089900204860FFE703E008990020C0
:105A10004860FFE740F60040C4F2024000688001A1
:105A2000002827D5FFE740F62840C4F2024000686E
:105A30004003002819D5FFE79DED010A40F63440E8
:105A4000C4F202400068C0F3066001EE100AB8EE2E
:105A5000411AB7EE002A31EE021A80EE010A0898C8
:105A6000BCEEC00A80ED020A03E0089900208860BD
:105A7000FFE703E0089900208860FFE707E0089946
:105A8000002008600899486008998860FFE709B01D
:105A9000704700BF20BCBE4B000000460024744A83
:105AA00089B0089040F63C40C4F2024000686FF3B1
:105AB0005F20059040F62C40C4F20240016801F0DE
:105AC000030107910168C1F3052106910068C0F345
:105AD00000100490049840F64041C4F20241096865
:105AE00089B2C90800FB01F000EE100AB8EE400AC6
:105AF0008DED020A0698002800F03D81FFE7079827
:105B00000090012808D0FFE70098022830D0FFE776
:105B10000098032849D065E040F60040C4F20240F6
:105B20000068C0F3C10149F20000C0F2D030C840A3
:105B300003909DED030AB8EE400A9DED061AB8EEFB
:105B4000411A80EE010A9DED051AB8EE411A9DED4D
:105B5000022A9FED8F3A82EE032A31EE021AB7EE47
:105B6000002A31EE021A20EE010A8DED010A65E0ED
:105B70009DED060AB8EE401A9FED860A80EE010AF6
:105B80009DED051AB8EE411A9DED022A9FED803A6F
:105B900082EE032A31EE021AB7EE002A31EE021A23
:105BA00020EE010A8DED010A48E09DED060AB8EEEF
:105BB000401A9FED760A80EE010A9DED051AB8EEB7
:105BC000411A9DED022A9FED723A82EE032A31EED0
:105BD000021AB7EE002A31EE021A20EE010A8DED0C
:105BE000010A2BE040F60040C4F202400068C0F316
:105BF000C10149F20000C0F2D030C84003909DEDD1
:105C0000030AB8EE400A9DED061AB8EE411A80EE7E
:105C1000010A9DED051AB8EE411A9DED022A9FED8D
:105C20005C3A82EE032A31EE021AB7EE002A31EE18
:105C3000021A20EE010A8DED010AFFE740F600404E
:105C4000C4F2024000680001002827D5FFE740F6B3
:105C50002C40C4F202400068C003002819D5FFE7B9
:105C60009DED010A40F63C40C4F20240006880B25B
:105C7000400A01EE100AB8EE411AB7EE002A31EEE2
:105C8000021A80EE010A0898BCEEC00A80ED000AF4
:105C900003E0089900200860FFE703E0089900206E
:105CA0000860FFE740F60040C4F2024000680001CF
:105CB000002827D5FFE740F62C40C4F202400068D8
:105CC0008003002819D5FFE79DED010A40F63C400E
:105CD000C4F202400068C0F3064001EE100AB8EEBC
:105CE000411AB7EE002A31EE021A80EE010A089836
:105CF000BCEEC00A80ED010A03E00899002048606C
:105D0000FFE703E0089900204860FFE740F6004005
:105D1000C4F2024000680001002827D5FFE740F6E2
:105D20002C40C4F2024000684003002819D5FFE768
:105D30009DED010A40F63C40C4F202400068C0F309
:105D4000066001EE100AB8EE411AB7EE002A31EEF5
:105D5000021A80EE010A0898BCEEC00A80ED020A21
:105D600003E0089900208860FFE703E0089900201D
:105D70008860FFE707E008990020086008994860FC
:105D800008998860FFE709B0704700BF20BCBE4B90
:105D9000000000460024744A89B0089040F6444050
:105DA000C4F2024000686FF35F20059040F6304077
:105DB000C4F20240016801F0030107910168C1F3D8
:105DC000052106910068C0F300100490049840F685
:105DD0004841C4F20241096889B2C90800FB01F0D8
:105DE00000EE100AB8EE400A8DED020A069800286F
:105DF00000F03D81FFE707980090012808D0FFE7F9
:105E00000098022830D0FFE70098032849D065E0C9
:105E100040F60040C4F202400068C0F3C10149F2FC
:105E20000000C0F2D030C84003909DED030AB8EEE8
:105E3000400A9DED061AB8EE411A80EE010A9DED6A
:105E4000051AB8EE411A9DED022A9FED8F3A82EEB7
:105E5000032A31EE021AB7EE002A31EE021A20EEC2
:105E6000010A8DED010A65E09DED060AB8EE401AC3
:105E70009FED860A80EE010A9DED051AB8EE411AE3
:105E80009DED022A9FED803A82EE032A31EE021A3E
:105E9000B7EE002A31EE021A20EE010A8DED010A5A
:105EA00048E09DED060AB8EE401A9FED760A80EEB6
:105EB000010A9DED051AB8EE411A9DED022A9FEDEB
:105EC000723A82EE032A31EE021AB7EE002A31EE60
:105ED000021A20EE010A8DED010A2BE040F6004087
:105EE000C4F202400068C0F3C10149F20000C0F2F0
:105EF000D030C84003909DED030AB8EE400A9DEDF6
:105F0000061AB8EE411A80EE010A9DED051AB8EEA8
:105F1000411A9DED022A9FED5C3A82EE032A31EE92
:105F2000021AB7EE002A31EE021A20EE010A8DEDB8
:105F3000010AFFE740F60040C4F20240006880001A
:105F4000002827D5FFE740F63040C4F20240006841
:105F5000C003002819D5FFE79DED010A40F6444033
:105F6000C4F20240006880B2400A01EE100AB8EEA6
:105F7000411AB7EE002A31EE021A80EE010A0898A3
:105F8000BCEEC00A80ED000A03E00899002008601A
:105F9000FFE703E0089900200860FFE740F60040B3
:105FA000C4F2024000688000002827D5FFE740F6D1
:105FB0003040C4F2024000688003002819D5FFE792
:105FC0009DED010A40F64440C4F202400068C0F36F
:105FD000064001EE100AB8EE411AB7EE002A31EE83
:105FE000021A80EE010A0898BCEEC00A80ED010A90
:105FF00003E0089900204860FFE703E008990020CB
:106000004860FFE740F60040C4F2024000688000AC
:10601000002827D5FFE740F63040C4F20240006870
:106020004003002819D5FFE79DED010A40F64440E2
:10603000C4F202400068C0F3066001EE100AB8EE38
:10604000411AB7EE002A31EE021A80EE010A0898D2
:10605000BCEEC00A80ED020A03E0089900208860C7
:10606000FFE703E0089900208860FFE707E0089950
:10607000002008600899486008998860FFE709B027
:10608000704700BF20BCBE4B000000460024744A8D
:1060900080B59CB01B911A901A981B9980F00070E3
:1060A000084300285BD1FFE740F6F040C4F202400D
:1060B000016801F440710E9100688007002809D53D
:1060C000FFE70E98B0F5807F04D1FFE74FF4004062
:1060D000109042E040F6F040C4F202400068000137
:1060E000002809D5FFE70E98B0F5007F04D1FFE73F
:1060F0004FF4FA4010902FE040F60040C4F2024006
:1061000000688003002823D5FFE70E98B0F5407F94
:106110001ED1FFE740F61C40C4F20240006800F4C4
:106120007C50B0F5007F0FD3FFE740F61C40C4F26F
:1061300002400068C0F3052147F64000C0F27D1020
:10614000B0FBF1F0109002E000201090FFE702E0B9
:1061500000201090FFE7FFE7FFE702F012BC1A985B
:106160000C901B990D9180F001000843002800F06D
:10617000C682FFE70D990C9880F0020008430028C2
:1061800000F03B83FFE70D990C9880F00400084372
:10619000002800F0A783FFE70D990C9880F0080015
:1061A0000843002800F01E84FFE70D990C9880F04A
:1061B00010000843002800F09884FFE70D990C9820
:1061C00080F020000843002800F01285FFE70D99B9
:1061D0000C9880F040000843002800F08C85FFE711
:1061E0000D990C9880F080000843002800F0068686
:1061F000FFE70D990C9880F480700843002800F0A8
:106200008086FFE70D990C9880F400700843002801
:1062100000F0FA86FFE70D990C9880F4806008433F
:10622000002800F07487FFE70D990C9880F4006057
:106230000843002800F0E987FFE70D990C9880F4E7
:1062400080500843002801F05E80FFE70D990C980C
:1062500080F400500843002801F06181FFE70D99A8
:106260000C9880F480400843002801F0AA81FFE7E1
:106270000D990C9880F400400843002801F0F38148
:10628000FFE70D990C9880F480300843002801F056
:106290008E82FFE70D990C9880F4003008430028A7
:1062A00001F0C282FFE70D990C9880F4802008432A
:1062B000002801F06583FFE70D990C9880F4002019
:1062C0000843002800F0BF80FFE70D990C9880F488
:1062D00080100843002800F04381FFE70D990C98D7
:1062E00080F400100843002801F07E80FFE70D993C
:1062F0000C9880F480000843002800F0BE81FFE77E
:106300000D990C9880F400000843002800F0D68115
:10631000FFE70D990C9880F080600843002802F098
:106320009882FFE70D990C9880F0006008430028E0
:1063300001F0B986FFE70D990C9880F08050084372
:10634000002801F02F87FFE70D990C9880F000508E
:106350000843002801F0B387FFE70D990C9880F0FF
:1063600080400843002802F03380FFE70D990C9825
:1063700080F000400843002802F0AE80FFE70C9850
:106380000D9981F001010843002802F02981FFE7FF
:106390000C980D9981F002010843002802F0A481B5
:1063A000FFE70C980D9981F004010843002801F0E3
:1063B0004386FFE70C980D9981F0080108430028F7
:1063C00002F00782FFE70C980D9981F01001084355
:1063D000002802F09482FFE70C980D9981F02001CB
:1063E0000843002801F07883FFE70C980D9981F0AD
:1063F00040010843002801F01B84FFE70C980D9929
:1064000081F080010843002801F0BE84FFE70C986A
:106410000D9981F480710843002801F06185FFE740
:106420000C980D9981F400710843002801F0488010
:10643000FFE70C980D9981F480610843002801F072
:10644000648102F09ABA40F6E840C4F20240006863
:1064500000F4E0200E900E980B90A0B1FFE70B988F
:10646000B0F5803F15D0FFE70B98B0F5003F16D090
:10647000FFE70B98B0F5403F17D0FFE70B98B0F55A
:10648000802F18D067E017A8FFF78EF918981090A2
:1064900064E014A8FFF704FB149810905EE011A8C4
:1064A000FFF77AFC1198109058E048F20000C0F213
:1064B000BB00109052E040F6E840C4F20240006891
:1064C00000F040400F9040F60040C4F202400068E7
:1064D0008007002811D5FFE70F9870B9FFE740F655
:1064E0000040C4F202400068C0F3C10149F200005C
:1064F000C0F2D030C84010902CE040F60040C4F20A
:1065000002400068800500280BD5FFE70F98B0F126
:10651000804F06D1FFE740F60010C0F23D0010901A
:1065200017E040F60040C4F20240006880030028F3
:106530000BD5FFE70F98B0F1004F06D1FFE747F604
:106540004000C0F27D10109002E000201090FFE7A4
:10655000FFE7FFE702E000201090FFE702F010BA2B
:1065600040F6E840C4F20240006800F460100E906B
:106570000E980A90A0B1FFE70A98B0F5002F15D049
:10658000FFE70A98B0F5801F16D0FFE70A98B0F52C
:10659000C01F17D0FFE70A98B0F5001F18D067E0BA
:1065A00017A8FFF701F91898109064E014A8FFF7F6
:1065B00077FA149810905EE011A8FFF7EDFB1198A0
:1065C000109058E048F20000C0F2BB00109052E07A
:1065D00040F6E840C4F20240006800F040400F90EE
:1065E00040F60040C4F2024000688007002811D540
:1065F000FFE70F9870B9FFE740F60040C4F2024091
:106600000068C0F3C10149F20000C0F2D030C840B8
:1066100010902CE040F60040C4F202400068800573
:1066200000280BD5FFE70F98B0F1804F06D1FFE7A8
:1066300040F60010C0F23D00109017E040F6004018
:10664000C4F202400068800300280BD5FFE70F98D2
:10665000B0F1004F06D1FFE747F64000C0F27D10D1
:10666000109002E000201090FFE7FFE7FFE702E054
:1066700000201090FFE702F083B940F6E440C4F236
:106680000240006800F040000E900E9830B9FFE71D
:1066900017A8FFF789F8189810900DE00E98402879
:1066A00006D1FFE714A8FFF7FBF91698109002E057
:1066B00000201090FFE7FFE702F062B940F6E440E7
:1066C000C4F20240006800F080000E900E9830B9CD
:1066D000FFE717A8FFF768F8189810900DE00E98DC
:1066E000802806D1FFE714A8FFF7DAF91698109072
:1066F00002E000201090FFE7FFE702F041B940F60A
:10670000D840C4F20240006800F007000E900E98D6
:1067100020B9FFE704F05EF810906CE040F600400E
:10672000C4F202400068000100280AD5FFE70E9875
:10673000012806D1FFE714A8FFF7B2F915981090C9
:1067400058E040F60040C4F2024000688000002893
:106750000AD5FFE70E98022806D1FFE711A8FFF738
:106760001BFB1298109044E040F60040C4F2024037
:1067700000688007002812D5FFE70E9803280ED185
:10678000FFE740F60040C4F202400068C0F3C101D8
:1067900049F20000C0F2D030C840109028E040F626
:1067A0000040C4F202400068800500280AD5FFE7D7
:1067B0000E98042806D1FFE740F60010C0F23D0015
:1067C000109014E040F6F040C4F2024000688007E8
:1067D000002808D5FFE70E98052804D1FFE74FF4FD
:1067E0000040109002E000201090FFE7FFE7FFE775
:1067F000FFE7FFE7FFE702F0C3B840F6D840C4F276
:106800000240006800F038000E900E9820B9FFE7B3
:1068100003F0CCFF109063E040F60040C4F2024069
:106820000068000100280AD5FFE70E98082806D165
:10683000FFE714A8FFF734F9159810904FE00E9871
:10684000102806D1FFE711A8FFF7A6FA12981090BA
:1068500044E040F60040C4F202400068800700288F
:1068600012D5FFE70E9818280ED1FFE740F600403A
:10687000C4F202400068C0F3C10149F20000C0F256
:10688000D030C840109028E040F60040C4F20240EA
:106890000068800500280AD5FFE70E98202806D159
:1068A000FFE740F60010C0F23D00109014E040F603
:1068B000F040C4F2024000688007002808D5FFE7D6
:1068C0000E98282804D1FFE74FF40040109002E012
:1068D00000201090FFE7FFE7FFE7FFE7FFE7FFE794
:1068E00002F04EB840F6D840C4F20240006800F40E
:1068F000E0700E900E9820B9FFE703F057FF10905C
:106900006EE040F60040C4F202400068000100283A
:106910000AD5FFE70E98402806D1FFE714A8FFF735
:10692000BFF8159810905AE040F60040C4F20240BB
:106930000068800000280AD5FFE70E98802806D15D
:10694000FFE711A8FFF728FA1298109046E040F6EA
:106950000040C4F2024000688007002812D5FFE71B
:106960000E98C0280ED1FFE740F60040C4F2024066
:106970000068C0F3C10149F20000C0F2D030C84045
:1069800010902AE040F60040C4F202400068800502
:1069900000280BD5FFE70E98B0F5807F06D1FFE702
:1069A00040F60010C0F23D00109015E040F6F040B7
:1069B000C4F2024000688007002809D5FFE70E985E
:1069C000B0F5A07F04D1FFE74FF40040109002E043
:1069D00000201090FFE7FFE7FFE7FFE7FFE7FFE793
:1069E00001F0CEBF40F6D840C4F20240006800F487
:1069F00060600E900E9820B9FFE703F0D7FE10906C
:106A000071E040F60040C4F2024000680001002836
:106A10000BD5FFE70E98B0F5007F06D1FFE714A86D
:106A2000FFF73EF8159810905CE040F60040C4F285
:106A300002400068800000280BD5FFE70E98B0F5F3
:106A4000806F06D1FFE711A8FFF7A6F91298109002
:106A500047E040F60040C4F202400068800700288A
:106A600013D5FFE70E98B0F5C06F0ED1FFE740F6E3
:106A70000040C4F202400068C0F3C10149F20000C6
:106A8000C0F2D030C84010902AE040F60040C4F276
:106A900002400068800500280BD5FFE70E98B0F58E
:106AA000006F06D1FFE740F60010C0F23D001090E5
:106AB00015E040F6F040C4F202400068800700286C
:106AC00009D5FFE70E98B0F5206F04D1FFE74FF42A
:106AD0000040109002E000201090FFE7FFE7FFE782
:106AE000FFE7FFE7FFE701F04BBF40F6D840C4F2F5
:106AF0000240006800F4E0400E900E9820B9FFE7D5
:106B000003F054FE109071E040F60040C4F20240E1
:106B10000068000100280BD5FFE70E98B0F5805FF4
:106B200006D1FFE714A8FEF7BBFF159810905CE0B4
:106B300040F60040C4F202400068800000280BD5F7
:106B4000FFE70E98B0F5005F06D1FFE711A8FFF749
:106B500023F91298109047E040F60040C4F202403A
:106B600000688007002813D5FFE70E98B0F5405F56
:106B70000ED1FFE740F60040C4F202400068C0F3C7
:106B8000C10149F20000C0F2D030C84010902AE0A4
:106B900040F60040C4F202400068800500280BD592
:106BA000FFE70E98B0F5804F06D1FFE740F60010E2
:106BB000C0F23D00109015E040F6F040C4F20240F3
:106BC00000688007002809D5FFE70E98B0F5A04FB0
:106BD00004D1FFE74FF40040109002E00020109035
:106BE000FFE7FFE7FFE7FFE7FFE7FFE701F0C8BECA
:106BF00040F6D840C4F20240006800F460300E90C5
:106C00000E9820B9FFE703F0D1FD109071E040F637
:106C10000040C4F202400068000100280BD5FFE7E5
:106C20000E98B0F5004F06D1FFE714A8FEF738FF25
:106C3000159810905CE040F60040C4F202400068F5
:106C4000800000280BD5FFE70E98B0F5803F06D1F5
:106C5000FFE711A8FFF7A0F81298109047E040F660
:106C60000040C4F2024000688007002813D5FFE707
:106C70000E98B0F5C03F0ED1FFE740F60040C4F2D9
:106C800002400068C0F3C10149F20000C0F2D030F8
:106C9000C84010902AE040F60040C4F2024000686C
:106CA000800500280BD5FFE70E98B0F5003F06D110
:106CB000FFE740F60010C0F23D00109015E040F6EE
:106CC000F040C4F2024000688007002809D5FFE7C1
:106CD0000E98B0F5203F04D1FFE74FF4004010902C
:106CE00002E000201090FFE7FFE7FFE7FFE7FFE784
:106CF000FFE701F045BE40F6D840C4F2024000680C
:106D000000F4E0100E900E9820B9FFE703F04EFD5E
:106D1000109071E040F60040C4F2024000680001AB
:106D200000280BD5FFE70E98B0F5802F06D1FFE7BE
:106D300014A8FEF7B5FE159810905CE040F60040F0
:106D4000C4F202400068800000280BD5FFE70E98CF
:106D5000B0F5002F06D1FFE711A8FFF71DF8129834
:106D6000109047E040F60040C4F2024000688007FF
:106D7000002813D5FFE70E98B0F5402F0ED1FFE79E
:106D800040F60040C4F202400068C0F3C10149F27D
:106D90000000C0F2D030C84010902AE040F6004019
:106DA000C4F202400068800500280BD5FFE70E986A
:106DB000B0F5801F06D1FFE740F60010C0F23D009D
:106DC000109015E040F6F040C4F2024000688007E1
:106DD000002809D5FFE70E98B0F5A01F04D1FFE702
:106DE0004FF40040109002E000201090FFE7FFE712
:106DF000FFE7FFE7FFE7FFE701F0C2BD40F6D8403D
:106E0000C4F20240006800F460000E900E9820B9B1
:106E1000FFE703F0CBFC109071E040F60040C4F2B5
:106E200002400068000100280BD5FFE70E98B0F57E
:106E3000001F06D1FFE714A8FEF732FE1598109048
:106E40005CE040F60040C4F2024000688000002888
:106E50000BD5FFE70E98B0F5800F06D1FFE711A81C
:106E6000FEF79AFF1298109047E040F60040C4F2F7
:106E7000024000688007002813D5FFE70E98B0F5A0
:106E8000C00F0ED1FFE740F60040C4F20240006898
:106E9000C0F3C10149F20000C0F2D030C8401090E8
:106EA0002AE040F60040C4F2024000688005002855
:106EB0000BD5FFE70E98B0F5000F06D1FFE740F6BF
:106EC0000010C0F23D00109015E040F6F040C4F212
:106ED000024000688007002809D5FFE70E98B0F54A
:106EE000200F04D1FFE74FF40040109002E0002093
:106EF0001090FFE7FFE7FFE7FFE7FFE7FFE701F09D
:106F00003FBD40F6D840C4F20240006800F0E060A7
:106F10000E900E9820B9FFE703F048FC109071E046
:106F200040F60040C4F202400068000100280BD582
:106F3000FFE70E98B0F1807F06D1FFE714A8FEF7B7
:106F4000AFFD159810905CE040F60040C4F202409E
:106F50000068800000280BD5FFE70E98B0F1007F95
:106F600006D1FFE711A8FEF717FF1298109047E02F
:106F700040F60040C4F2024000688007002813D5A4
:106F8000FFE70E98B0F1407F0ED1FFE740F60040DA
:106F9000C4F202400068C0F3C10149F20000C0F22F
:106FA000D030C84010902AE040F60040C4F20240C1
:106FB0000068800500280BD5FFE70E98B0F1806FC0
:106FC00006D1FFE740F60010C0F23D00109015E03A
:106FD00040F6F040C4F2024000688007002809D55E
:106FE000FFE70E98B0F1A06F04D1FFE74FF4004027
:106FF000109002E000201090FFE7FFE7FFE7FFE7B7
:10700000FFE7FFE701F0BCBC40F6D840C4F2024005
:10701000006800F060500E900E9820B9FFE703F072
:10702000C5FB109071E040F60040C4F202400068D9
:10703000000100280BD5FFE70E98B0F1006F06D1D4
:10704000FFE714A8FEF72CFD159810905CE040F6C1
:107050000040C4F202400068800000280BD5FFE722
:107060000E98B0F1805F06D1FFE711A8FEF794FEFD
:107070001298109047E040F60040C4F202400068C9
:107080008007002813D5FFE70E98B0F1C05F0ED13E
:10709000FFE740F60040C4F202400068C0F3C101BF
:1070A00049F20000C0F2D030C84010902AE040F60B
:1070B0000040C4F202400068800500280BD5FFE7BD
:1070C0000E98B0F1005F06D1FFE740F60010C0F265
:1070D0003D00109015E040F6F040C4F20240006818
:1070E0008007002809D5FFE70E98B0F1205F04D192
:1070F000FFE74FF40040109002E000201090FFE7FF
:10710000FFE7FFE7FFE7FFE7FFE701F039BC40F6E5
:10711000DC40C4F20240006800F007000E900E98B8
:1071200020B9FFE703F042FB10906CE040F600400E
:10713000C4F202400068000100280AD5FFE70E985B
:10714000012806D1FFE714A8FEF7AAFC15981090B5
:1071500058E040F60040C4F2024000688000002879
:107160000AD5FFE70E98022806D1FFE711A8FEF71F
:1071700013FE1298109044E040F60040C4F2024022
:1071800000688007002812D5FFE70E9803280ED16B
:10719000FFE740F60040C4F202400068C0F3C101BE
:1071A00049F20000C0F2D030C840109028E040F60C
:1071B0000040C4F202400068800500280AD5FFE7BD
:1071C0000E98042806D1FFE740F60010C0F23D00FB
:1071D000109014E040F6F040C4F2024000688007CE
:1071E000002808D5FFE70E98052804D1FFE74FF4E3
:1071F0000040109002E000201090FFE7FFE7FFE75B
:10720000FFE7FFE7FFE701F0BBBB40F6DC40C4F25D
:107210000240006800F070000E900E9820B9FFE761
:1072200003F0C4FA10906CE040F60040C4F2024053
:107230000068000100280AD5FFE70E98102806D143
:10724000FFE714A8FEF72CFC1598109058E040F6C4
:107250000040C4F202400068800000280AD5FFE721
:107260000E98202806D1FFE711A8FEF795FD129889
:10727000109044E040F60040C4F2024000688007ED
:10728000002812D5FFE70E9830280ED1FFE740F610
:107290000040C4F202400068C0F3C10149F200009E
:1072A000C0F2D030C840109028E040F60040C4F250
:1072B00002400068800500280AD5FFE70E984028A4
:1072C00006D1FFE740F60010C0F23D00109014E038
:1072D00040F6F040C4F2024000688007002808D55C
:1072E000FFE70E98502804D1FFE74FF400401090BC
:1072F00002E000201090FFE7FFE7FFE7FFE7FFE76E
:10730000FFE701F03DBB40F6E040C4F202400068F8
:1073100000F0E0600E900E9820B9FFE703F06EFADF
:1073200010905FE00E98B0F1807F06D1FFE714A8BF
:10733000FEF7B6FB1598109053E00E98B0F1007F61
:1073400006D1FFE711A8FEF727FD1298109047E03D
:1073500040F60040C4F2024000688007002813D5C0
:10736000FFE70E98B0F1407F0ED1FFE740F60040F6
:10737000C4F202400068C0F3C10149F20000C0F24B
:10738000D030C84010902AE040F60040C4F20240DD
:107390000068800500280BD5FFE70E98B0F1806FDC
:1073A00006D1FFE740F60010C0F23D00109015E056
:1073B00040F6F040C4F2024000688007002809D57A
:1073C000FFE70E98B0F1A06F04D1FFE74FF4004043
:1073D000109002E000201090FFE7FFE7FFE7FFE7D3
:1073E000FFE7FFE701F0CCBA40F6E840C4F2024004
:1073F000006800F007000E900E9820B9FFE703F038
:10740000BBF910905AE00E98012804D1FFE703F071
:1074100009FA109051E00E98022806D1FFE714A84F
:10742000FEF73EFB1698109046E040F60040C4F28E
:1074300002400068800300280AD5FFE70E98032861
:1074400006D1FFE747F64000C0F27D10109032E011
:1074500040F60040C4F2024000688007002812D5C0
:10746000FFE70E9804280ED1FFE740F60040C4F273
:1074700002400068C0F3C10149F20000C0F2D03000
:10748000C840109016E040F60040C4F20240006888
:10749000800500280AD5FFE70E98052806D1FFE7EA
:1074A00040F60010C0F23D00109002E00020109065
:1074B000FFE7FFE7FFE7FFE7FFE7FFE701F060BA5D
:1074C00040F6E840C4F20240006800F008000E9068
:1074D00040F6F040C4F2024000688007002807D55B
:1074E000FFE70E9820B9FFE74FF40040109014E03A
:1074F00040F6F040C4F2024000680001002808D5C0
:10750000FFE70E98082804D1FFE74FF4FA401090E7
:1075100002E000201090FFE7FFE701F031BA40F6EB
:10752000E440C4F20240006800F440300E900E982F
:1075300020B9FFE703F03AF9109040E00E98B0F55B
:10754000803F06D1FFE711A8FEF726FC13981090A4
:1075500034E040F60040C4F2024000688007002892
:1075600013D5FFE70E98B0F5003F0ED1FFE740F6C8
:107570000040C4F202400068C0F3C10149F20000BB
:10758000C0F2D030C840109017E040F60040C4F27E
:1075900002400068800500280BD5FFE70E98B0F583
:1075A000403F06D1FFE740F60010C0F23D001090CA
:1075B00002E000201090FFE7FFE7FFE7FFE701F0A0
:1075C000DFB940F6E440C4F20240006800F4402015
:1075D0000E900E9820B9FFE703F0E8F8109040E015
:1075E0000E98B0F5802F06D1FFE711A8FEF7D4FB67
:1075F0001398109034E040F60040C4F20240006856
:107600008007002813D5FFE70E98B0F5002F0ED1A4
:10761000FFE740F60040C4F202400068C0F3C10139
:1076200049F20000C0F2D030C840109017E040F698
:107630000040C4F202400068800500280BD5FFE737
:107640000E98B0F5402F06D1FFE740F60010C0F2CB
:107650003D00109002E000201090FFE7FFE7FFE7F9
:10766000FFE701F08DB940F6E440C4F20240006843
:1076700000F440100E900E9820B9FFE703F0BEF81A
:10768000109040E00E98B0F5801F06D1FFE711A8DA
:10769000FEF782FB1398109034E040F60040C4F2ED
:1076A000024000688007002813D5FFE70E98B0F568
:1076B000001F0ED1FFE740F60040C4F20240006810
:1076C000C0F3C10149F20000C0F2D030C8401090B0
:1076D00017E040F60040C4F2024000688005002830
:1076E0000BD5FFE70E98B0F5401F06D1FFE740F637
:1076F0000010C0F23D00109002E000201090FFE763
:10770000FFE7FFE7FFE701F03BB940F6E440C4F2D2
:107710000240006800F440000E900E9820B9FFE788
:1077200003F06CF8109040E00E98B0F5800F06D191
:10773000FFE711A8FEF730FB1398109034E040F6F5
:107740000040C4F2024000688007002813D5FFE71C
:107750000E98B0F5000F0ED1FFE740F60040C4F2DE
:1077600002400068C0F3C10149F20000C0F2D0300D
:10777000C840109017E040F60040C4F20240006894
:10778000800500280BD5FFE70E98B0F5400F06D115
:10779000FFE740F60010C0F23D00109002E000202C
:1077A0001090FFE7FFE7FFE7FFE701F0E9B840F6D9
:1077B000E440C4F20240006800F040700E900E9861
:1077C00020B9FFE702F0F2FF10902BE00E98B0F125
:1077D000807F06D1FFE711A8FEF7DEFA139810901C
:1077E0001FE040F60040C4F2024000688007002815
:1077F00013D5FFE70E98B0F1007F0ED1FFE740F6FA
:107800000040C4F202400068C0F3C10149F2000028
:10781000C0F2D030C840109002E000201090FFE786
:10782000FFE7FFE701F0ACB840F6DC40C4F20240ED
:10783000006800F4E0600E900E980990C8B1FFE770
:107840000998B0F5807F18D0FFE70998B0F5007F60
:1078500019D0FFE70998B0F5407F1AD0FFE70998E3
:10786000B0F5806F26D0FFE70998B0F5A06F32D051
:1078700081E002F0C3FF109080E014A8FEF710F939
:10788000149810907AE011A8FEF786FA13981090D9
:1078900074E040F6F040C4F202400068800700281F
:1078A00004D5FFE74FF40040109002E00020109054
:1078B000FFE763E040F6F040C4F2024000680001D8
:1078C000002804D5FFE74FF4FA40109002E00020B2
:1078D0001090FFE752E040F6E840C4F20240006832
:1078E00000F040400F9040F60040C4F202400068B3
:1078F0008007002811D5FFE70F9870B9FFE740F621
:107900000040C4F202400068C0F3C10149F2000027
:10791000C0F2D030C84010902CE040F60040C4F2D5
:1079200002400068800500280BD5FFE70F98B0F1F2
:10793000804F06D1FFE740F60010C0F23D001090E6
:1079400017E040F60040C4F20240006880030028BF
:107950000BD5FFE70F98B0F1004F06D1FFE747F6D0
:107960004000C0F27D10109002E000201090FFE770
:10797000FFE7FFE702E000201090FFE701F000B80A
:1079800040F6DC40C4F20240006800F4E0400E9093
:107990000E980890C8B1FFE70898B0F5805F18D03E
:1079A000FFE70898B0F5005F19D0FFE70898B0F539
:1079B000405F1AD0FFE70898B0F5804F26D0FFE768
:1079C0000898B0F5A04F32D081E002F0EFFE1090A1
:1079D00080E014A8FEF764F8149810907AE011A8DB
:1079E000FEF7DAF91398109074E040F6F040C4F214
:1079F000024000688007002804D5FFE74FF40040EC
:107A0000109002E000201090FFE763E040F6F040A5
:107A1000C4F2024000680001002804D5FFE74FF4DB
:107A2000FA40109002E000201090FFE752E040F68C
:107A3000E840C4F20240006800F040400F9040F679
:107A40000040C4F2024000688007002811D5FFE71B
:107A50000F9870B9FFE740F60040C4F2024000689A
:107A6000C0F3C10149F20000C0F2D030C84010900C
:107A70002CE040F60040C4F2024000688005002877
:107A80000BD5FFE70F98B0F1804F06D1FFE740F626
:107A90000010C0F23D00109017E040F60040C4F224
:107AA00002400068800300280BD5FFE70F98B0F173
:107AB000004F06D1FFE747F64000C0F27D1010905E
:107AC00002E000201090FFE7FFE7FFE702E0002060
:107AD0001090FFE700F054BF40F6DC40C4F20240D3
:107AE000006800F4E0200E900E980790C8B1FFE700
:107AF0000798B0F5803F18D0FFE70798B0F5003F32
:107B000019D0FFE70798B0F5403F1AD0FFE7079874
:107B1000B0F5802F26D0FFE70798B0F5A02F32D020
:107B200081E002F06BFE109080E014A8FDF7B8FF32
:107B3000149810907AE011A8FEF72EF9139810907F
:107B400074E040F6F040C4F202400068800700286C
:107B500004D5FFE74FF40040109002E000201090A1
:107B6000FFE763E040F6F040C4F202400068000125
:107B7000002804D5FFE74FF4FA40109002E00020FF
:107B80001090FFE752E040F6E840C4F2024000687F
:107B900000F040400F9040F60040C4F20240006800
:107BA0008007002811D5FFE70F9870B9FFE740F66E
:107BB0000040C4F202400068C0F3C10149F2000075
:107BC000C0F2D030C84010902CE040F60040C4F223
:107BD00002400068800500280BD5FFE70F98B0F140
:107BE000804F06D1FFE740F60010C0F23D00109034
:107BF00017E040F60040C4F202400068800300280D
:107C00000BD5FFE70F98B0F1004F06D1FFE747F61D
:107C10004000C0F27D10109002E000201090FFE7BD
:107C2000FFE7FFE702E000201090FFE700F0A8BEAA
:107C300040F6DC40C4F20240006800F4E0000E9020
:107C40000E980690C8B1FFE70698B0F5801F18D0CF
:107C5000FFE70698B0F5001F19D0FFE70698B0F5CA
:107C6000401F1AD0FFE70698B0F5800F26D0FFE737
:107C70000698B0F5A00F32D081E002F0BFFD109061
:107C800080E014A8FDF70CFF149810907AE011A87A
:107C9000FEF782F81398109074E040F6F040C4F2BA
:107CA000024000688007002804D5FFE74FF4004039
:107CB000109002E000201090FFE763E040F6F040F3
:107CC000C4F2024000680001002804D5FFE74FF429
:107CD000FA40109002E000201090FFE752E040F6DA
:107CE000E840C4F20240006800F040400F9040F6C7
:107CF0000040C4F2024000688007002811D5FFE769
:107D00000F9870B9FFE740F60040C4F202400068E7
:107D1000C0F3C10149F20000C0F2D030C840109059
:107D20002CE040F60040C4F20240006880050028C4
:107D30000BD5FFE70F98B0F1804F06D1FFE740F673
:107D40000010C0F23D00109017E040F60040C4F271
:107D500002400068800300280BD5FFE70F98B0F1C0
:107D6000004F06D1FFE747F64000C0F27D101090AB
:107D700002E000201090FFE7FFE7FFE702E00020AD
:107D80001090FFE700F0FCBD40F6DC40C4F202407A
:107D9000006800F0E0600E900E980590C8B1FFE713
:107DA0000598B0F1807F18D0FFE70598B0F1007F0B
:107DB00019D0FFE70598B0F1407F1AD0FFE705988A
:107DC000B0F1806F26D0FFE70598B0F1A06F32D0F8
:107DD00081E002F013FD109080E014A8FDF760FE32
:107DE000149810907AE011A8FDF7D6FF1398109020
:107DF00074E040F6F040C4F20240006880070028BA
:107E000004D5FFE74FF40040109002E000201090EE
:107E1000FFE763E040F6F040C4F202400068000172
:107E2000002804D5FFE74FF4FA40109002E000204C
:107E30001090FFE752E040F6E840C4F202400068CC
:107E400000F040400F9040F60040C4F2024000684D
:107E50008007002811D5FFE70F9870B9FFE740F6BB
:107E60000040C4F202400068C0F3C10149F20000C2
:107E7000C0F2D030C84010902CE040F60040C4F270
:107E800002400068800500280BD5FFE70F98B0F18D
:107E9000804F06D1FFE740F60010C0F23D00109081
:107EA00017E040F60040C4F202400068800300285A
:107EB0000BD5FFE70F98B0F1004F06D1FFE747F66B
:107EC0004000C0F27D10109002E000201090FFE70B
:107ED000FFE7FFE702E000201090FFE700F050BD51
:107EE00040F6DC40C4F20240006800F0E0400E9032
:107EF0000E980490C8B1FFE70498B0F1805F18D0E5
:107F0000FFE70498B0F1005F19D0FFE70498B0F1E3
:107F1000405F1AD0FFE70498B0F1804F26D0FFE70A
:107F20000498B0F1A04F32D081E002F067FC1090CD
:107F300080E014A8FDF7B4FD149810907AE011A821
:107F4000FDF72AFF1398109074E040F6F040C4F259
:107F5000024000688007002804D5FFE74FF4004086
:107F6000109002E000201090FFE763E040F6F04040
:107F7000C4F2024000680001002804D5FFE74FF476
:107F8000FA40109002E000201090FFE752E040F627
:107F9000E840C4F20240006800F040400F9040F614
:107FA0000040C4F2024000688007002811D5FFE7B6
:107FB0000F9870B9FFE740F60040C4F20240006835
:107FC000C0F3C10149F20000C0F2D030C8401090A7
:107FD0002CE040F60040C4F2024000688005002812
:107FE0000BD5FFE70F98B0F1804F06D1FFE740F6C1
:107FF0000010C0F23D00109017E040F60040C4F2BF
:1080000002400068800300280BD5FFE70F98B0F10D
:10801000004F06D1FFE747F64000C0F27D101090F8
:1080200002E000201090FFE7FFE7FFE702E00020FA
:108030001090FFE700F0A4BC40F6E840C4F2024014
:10804000006800F440700E9040F60040C4F2024018
:1080500000688003002809D5FFE70E9830B9FFE7D4
:1080600047F64000C0F27D1010901AE00E98B0F56F
:10807000807F06D1FFE717A8FDF796FB18981090B0
:108080000EE00E98B0F5007F06D1FFE714A8FDF7CB
:1080900007FD1598109002E000201090FFE7FFE721
:1080A000FFE700F06DBC40F6E040C4F2024000681B
:1080B00000F007000E900E98039004286DD80399E5
:1080C000DFE801F003090F151B0017A8FDF76CFB93
:1080D0001898109064E014A8FDF7E2FC1498109032
:1080E0005EE011A8FDF758FE1198109058E048F294
:1080F0000000C0F2BB00109052E040F6E840C4F22D
:108100000240006800F040400F9040F60040C4F28A
:10811000024000688007002811D5FFE70F9870B96A
:10812000FFE740F60040C4F202400068C0F3C1011E
:1081300049F20000C0F2D030C84010902CE040F668
:108140000040C4F202400068800500280BD5FFE71C
:108150000F98B0F1804F06D1FFE740F60010C0F253
:108160003D00109017E040F60040C4F20240006865
:10817000800300280BD5FFE70F98B0F1004F06D120
:10818000FFE747F64000C0F27D10109002E00020AB
:108190001090FFE7FFE7FFE702E000201090FFE705
:1081A00000F0EEBB40F6E040C4F20240006800F090
:1081B00038000E900E980290202800F27C800299E0
:1081C000DFE801F011797979797979791779797915
:1081D000797979791D7979797979797923797979C1
:1081E00079797979290017A8FDF7DEFA18981090A7
:1081F00064E014A8FDF754FC149810905EE011A8F8
:10820000FDF7CAFD1198109058E048F20000C0F246
:10821000BB00109052E040F6E840C4F20240006813
:1082200000F040400F9040F60040C4F20240006869
:108230008007002811D5FFE70F9870B9FFE740F6D7
:108240000040C4F202400068C0F3C10149F20000DE
:10825000C0F2D030C84010902CE040F60040C4F28C
:1082600002400068800500280BD5FFE70F98B0F1A9
:10827000804F06D1FFE740F60010C0F23D0010909D
:1082800017E040F60040C4F2024000688003002876
:108290000BD5FFE70F98B0F1004F06D1FFE747F687
:1082A0004000C0F27D10109002E000201090FFE727
:1082B000FFE7FFE702E000201090FFE760E340F6F1
:1082C000E040C4F20240006800F4E0700E900E98A6
:1082D000019088B1FFE70198402813D0FFE701988B
:1082E000802815D0FFE70198C02817D0FFE7019834
:1082F000B0F5807F18D067E017A8FDF755FA1898F9
:10830000109064E014A8FDF7CBFB149810905EE089
:1083100011A8FDF741FD1198109058E048F20000B7
:10832000C0F2BB00109052E040F6E840C4F20240B8
:10833000006800F040400F9040F60040C4F2024058
:1083400000688007002811D5FFE70F9870B9FFE794
:1083500040F60040C4F202400068C0F3C10149F297
:108360000000C0F2D030C84010902CE040F6004031
:10837000C4F202400068800500280BD5FFE70F9883
:10838000B0F1804F06D1FFE740F60010C0F23D008B
:10839000109017E040F60040C4F2024000688003ED
:1083A00000280BD5FFE70F98B0F1004F06D1FFE78B
:1083B00047F64000C0F27D10109002E000201090BF
:1083C000FFE7FFE7FFE702E000201090FFE7D7E2BA
:1083D00040F6E040C4F20240006800F460600E9095
:1083E0000E9820B9FFE702F0F5F9109073E040F61F
:1083F0000040C4F202400068000100280BD5FFE7EE
:108400000E98B0F5007F06D1FFE714A8FDF748FBF2
:10841000159810905EE040F60040C4F202400068FB
:10842000800000280BD5FFE70E98B0F5806F06D1CD
:10843000FFE711A8FDF7B0FC1298109049E040F654
:108440000040C4F2024000688007002813D5FFE70F
:108450000E98B0F5C06F0ED1FFE740F60040C4F2B1
:1084600002400068C0F3C10149F20000C0F2D03000
:10847000C84010902CE040F60040C4F20240006872
:10848000800500280BD5FFE70E98B0F5006F06D1E8
:10849000FFE740F60010C0F23D00109017E040F6F4
:1084A0000040C4F202400068800300280BD5FFE7BB
:1084B0000E98B0F5206F06D1FFE747F64000C0F2F6
:1084C0007D10109002E000201090FFE7FFE7FFE72B
:1084D000FFE7FFE7FFE753E240F6E040C4F2024067
:1084E000006800F4E0400E900E9820B9FFE702F01B
:1084F00085F9109073E040F60040C4F20240006835
:10850000000100280BD5FFE70E98B0F5805F06D17B
:10851000FFE714A8FDF7C4FA159810905EE040F646
:108520000040C4F202400068800000280BD5FFE73D
:108530000E98B0F5005F06D1FFE711A8FDF72CFCFF
:108540001298109049E040F60040C4F202400068E2
:108550008007002813D5FFE70E98B0F5405F0ED1D5
:10856000FFE740F60040C4F202400068C0F3C101DA
:1085700049F20000C0F2D030C84010902CE040F624
:108580000040C4F202400068800500280BD5FFE7D8
:108590000E98B0F5804F06D1FFE740F60010C0F20C
:1085A0003D00109017E040F60040C4F20240006821
:1085B000800300280BD5FFE70E98B0F5A04F06D139
:1085C000FFE747F64000C0F27D10109002E0002067
:1085D0001090FFE7FFE7FFE7FFE7FFE7FFE7CFE1E7
:1085E00040F6E040C4F20240006800F460300E90B3
:1085F0000E9820B9FFE702F0EDF8109073E040F616
:108600000040C4F202400068000100280BD5FFE7DB
:108610000E98B0F5004F06D1FFE714A8FDF740FA19
:10862000159810905EE040F60040C4F202400068E9
:10863000800000280BD5FFE70E98B0F5803F06D1EB
:10864000FFE711A8FDF7A8FB1298109049E040F64B
:108650000040C4F2024000688007002813D5FFE7FD
:108660000E98B0F5C03F0ED1FFE740F60040C4F2CF
:1086700002400068C0F3C10149F20000C0F2D030EE
:10868000C84010902CE040F60040C4F20240006860
:10869000800500280BD5FFE70E98B0F5003F06D106
:1086A000FFE740F60010C0F23D00109017E040F6E2
:1086B0000040C4F202400068800300280BD5FFE7A9
:1086C0000E98B0F5203F06D1FFE747F64000C0F214
:1086D0007D10109002E000201090FFE7FFE7FFE719
:1086E000FFE7FFE7FFE74BE140F6E440C4F202405A
:1086F000006800F003000E900E980090032864D8E4
:108700000099DFE801F002060C1202F035F8109033
:108710005EE017A8FDF748F81898109058E014A8E4
:10872000FDF7BEF91698109052E040F6E840C4F20A
:108730000240006800F040400F9040F60040C4F254
:10874000024000688007002811D5FFE70F9870B934
:10875000FFE740F60040C4F202400068C0F3C101E8
:1087600049F20000C0F2D030C84010902CE040F632
:108770000040C4F202400068800500280BD5FFE7E6
:108780000F98B0F1804F06D1FFE740F60010C0F21D
:108790003D00109017E040F60040C4F2024000682F
:1087A000800300280BD5FFE70F98B0F1004F06D1EA
:1087B000FFE747F64000C0F27D10109002E0002075
:1087C0001090FFE7FFE7FFE702E000201090FFE7CF
:1087D000D6E040F6E840C4F20240006800F0C00075
:1087E0000E9040F6F040C4F2024000688007002876
:1087F00007D5FFE70E9820B9FFE74FF4004010902F
:1088000026E040F6F040C4F2024000680001002873
:1088100008D5FFE70E98402804D1FFE74FF4FA404F
:10882000109014E040F60040C4F202400068800559
:10883000002808D5FFE70E98802804D1FFE748F20A
:108840001200109002E000201090FFE7FFE7FFE722
:1088500096E040F6E840C4F20240006800F03000C4
:108860000E9040F60040C4F20240006880040028E8
:1088700009D5FFE70E9830B9FFE746F60040C0F291
:10888000DC2010903AE040F60040C4F2024000685C
:10889000800100280AD5FFE70E98102806D1FFE7CF
:1088A00017A8FCF781FF1898109026E040F6F040DA
:1088B000C4F2024000688007002808D5FFE70E9840
:1088C000202804D1FFE74FF40040109014E040F658
:1088D000F040C4F2024000680001002808D5FFE71C
:1088E0000E98302804D1FFE74FF4FA40109002E0D0
:1088F00000201090FFE7FFE7FFE7FFE740E040F6CA
:10890000E440C4F20240006800F030000E900E987F
:10891000102806D1FFE717A8FCF746FF189810901B
:108920002EE040F60040C4F20240006880000028BB
:108930000AD5FFE70E98202806D1FFE711A8FDF71A
:108940002BFA1298109016E040F60040C4F2024054
:108950000068800400280AD5FFE70E98302806D169
:10896000FFE746F60040C0F2DC20109002E0002055
:108970001090FFE7FFE7FFE702E000201090FFE71D
:10898000FFE710981CB080BD80B5ACB02B900020E4
:108990008DF8A3008DF8A2002B98C078C00760B1B5
:1089A000FFE740F6E841C4F20241086820F0404089
:1089B0002B9A926D10430860FFE72B980068C00760
:1089C000002837D0FFE72B98C06D2790052817D8CF
:1089D0002799DFE801F003040B12131414E02B981D
:1089E000083005F007FC8DF8A3000DE02B9830301F
:1089F00005F0B6FC8DF8A30006E005E004E003E016
:108A000001208DF8A300FFE79DF8A30060B9FFE700
:108A100040F6D841C4F20241086820F007002B9AC2
:108A2000D26D1043086004E09DF8A3008DF8A20009
:108A3000FFE7FFE72B9800788007002840F14A8085
:108A4000FFE72B98006E2690282829D82699DFE882
:108A500001F0152727272727272716272727272726
:108A600027271D27272727272727242727272727A3
:108A700027272527272727272727260014E02B9895
:108A8000083005F0B7FB8DF8A3000DE02B983030CF
:108A900005F066FC8DF8A30006E005E004E003E0C5
:108AA00001208DF8A300FFE79DF8A30060B9FFE760
:108AB00040F6D841C4F20241086820F038002B9AF1
:108AC000126E1043086004E09DF8A3008DF8A20028
:108AD000FFE7FFE72B9800784007002847D5FFE71E
:108AE0002B98406E2590B0B1FFE72598402813D011
:108AF000FFE72598802816D0FFE72598C02819D0D1
:108B0000FFE72598B0F5807F15D0FFE72598B0F5F1
:108B1000A07F11D011E014E02B98083005F06AFB1B
:108B20008DF8A3000DE02B98303005F019FC8DF87E
:108B3000A30006E005E004E003E001208DF8A300B7
:108B4000FFE79DF8A30060B9FFE740F6D841C4F203
:108B50000241086820F4E0702B9A526E10430860BE
:108B600004E09DF8A3008DF8A200FFE7FFE72B9833
:108B70000078000700284AD5FFE72B98806E2490E4
:108B8000C8B1FFE72498B0F5007F15D0FFE724981F
:108B9000B0F5806F17D0FFE72498B0F5C06F19D0FB
:108BA000FFE72498B0F5006F15D0FFE72498B0F5E3
:108BB000206F11D011E014E02B98083005F01AFB5B
:108BC0008DF8A3000DE02B98303005F0C9FB8DF82F
:108BD000A30006E005E004E003E001208DF8A30017
:108BE000FFE79DF8A30060B9FFE740F6D841C4F263
:108BF0000241086820F460602B9A926E104308606E
:108C000004E09DF8A3008DF8A200FFE7FFE72B9892
:108C10000078C00600284AD5FFE72B98C06E239045
:108C2000C8B1FFE72398B0F5805F15D0FFE7239820
:108C3000B0F5005F17D0FFE72398B0F5405F19D07B
:108C4000FFE72398B0F5804F15D0FFE72398B0F5E4
:108C5000A04F11D011E014E02B98083005F0CAFAAB
:108C60008DF8A3000DE02B98303005F079FB8DF8DE
:108C7000A30006E005E004E003E001208DF8A30076
:108C8000FFE79DF8A30060B9FFE740F6D841C4F2C2
:108C90000241086820F4E0402B9AD26E104308602D
:108CA00004E09DF8A3008DF8A200FFE7FFE72B98F2
:108CB0000078800600284AD5FFE72B98006F2290A5
:108CC000C8B1FFE72298B0F5004F15D0FFE7229812
:108CD000B0F5803F17D0FFE72298B0F5C03F19D01C
:108CE000FFE72298B0F5003F15D0FFE72298B0F5D6
:108CF000203F11D011E014E02B98083005F07AFAEB
:108D00008DF8A3000DE02B98303005F029FB8DF88D
:108D1000A30006E005E004E003E001208DF8A300D5
:108D2000FFE79DF8A30060B9FFE740F6D841C4F221
:108D30000241086820F460302B9A126F10430860DB
:108D400004E09DF8A3008DF8A200FFE7FFE72B9851
:108D50000078400600284AD5FFE72B98406F219005
:108D6000C8B1FFE72198B0F5802F15D0FFE7219813
:108D7000B0F5002F17D0FFE72198B0F5402F19D09C
:108D8000FFE72198B0F5801F15D0FFE72198B0F5D7
:108D9000A01F11D011E014E02B98083005F02AFA3A
:108DA0008DF8A3000DE02B98303005F0D9FA8DF83E
:108DB000A30006E005E004E003E001208DF8A30035
:108DC000FFE79DF8A30060B9FFE740F6D841C4F281
:108DD0000241086820F4E0102B9A526F104308609B
:108DE00004E09DF8A3008DF8A200FFE7FFE72B98B1
:108DF0000078000600284AD5FFE72B98806F209066
:108E0000C8B1FFE72098B0F5001F15D0FFE7209804
:108E1000B0F5800F17D0FFE72098B0F5C00F19D03C
:108E2000FFE72098B0F5000F15D0FFE72098B0F5C8
:108E3000200F11D011E014E02B98083005F0DAF97A
:108E40008DF8A3000DE02B98303005F089FA8DF8ED
:108E5000A30006E005E004E003E001208DF8A30094
:108E6000FFE79DF8A30060B9FFE740F6D841C4F2E0
:108E70000241086820F460002B9A926F104308604A
:108E800004E09DF8A3008DF8A200FFE7FFE72B9810
:108E90004078C00700284AD0FFE72B98C06F1F908A
:108EA000C8B1FFE71F98B0F1807F15D0FFE71F988A
:108EB000B0F1007F17D0FFE71F98B0F1407F19D0C5
:108EC000FFE71F98B0F1806F15D0FFE71F98B0F152
:108ED000A06F11D011E014E02B98083005F08AF94A
:108EE0008DF8A3000DE02B98303005F039FA8DF89D
:108EF000A30006E005E004E003E001208DF8A300F4
:108F0000FFE79DF8A30060B9FFE740F6D841C4F23F
:108F10000241086820F0E0602B9AD26F104308608D
:108F200004E09DF8A3008DF8A200FFE7FFE72B986F
:108F30004078800700284CD5FFE72B98D0F88000B8
:108F40001E90C8B1FFE71E98B0F1006F15D0FFE783
:108F50001E98B0F1805F17D0FFE71E98B0F1C05F98
:108F600019D0FFE71E98B0F1005F15D0FFE71E98FB
:108F7000B0F1205F11D011E014E02B98083005F01B
:108F800039F98DF8A3000DE02B98303005F0E8F9A1
:108F90008DF8A30006E005E004E003E001208DF871
:108FA000A300FFE79DF8A30068B9FFE740F6D841AA
:108FB000C4F20241086820F060502B9AD2F8802059
:108FC0001043086004E09DF8A3008DF8A200FFE7BD
:108FD000FFE72B9840784007002839D5FFE72B980A
:108FE000D0F884001D90052817D81D99DFE801F0FE
:108FF00003040B12131414E02B98083005F0FAF850
:109000008DF8A3000DE02B98303005F0A9F98DF80C
:10901000A30006E005E004E003E001208DF8A300D2
:10902000FFE79DF8A30068B9FFE740F6DC41C4F212
:109030000241086820F007002B9AD2F884201043E0
:10904000086004E09DF8A3008DF8A200FFE7FFE7A9
:109050002B9840780007002847D5FFE72B98D0F8D9
:1090600088001C90A0B1FFE71C98102811D0FFE7E2
:109070001C98202814D0FFE71C98302817D0FFE751
:109080001C98402814D0FFE71C98502811D011E0FC
:1090900014E02B98083005F0ADF88DF8A3000DE032
:1090A0002B98303005F05CF98DF8A30006E005E060
:1090B00004E003E001208DF8A300FFE79DF8A30082
:1090C00068B9FFE740F6DC41C4F20241086820F0CD
:1090D00070002B9AD2F888201043086004E09DF8B5
:1090E000A3008DF8A200FFE7FFE72B984078C006A9
:1090F00000284CD5FFE72B98D0F88C001B90C8B106
:10910000FFE71B98B0F1807F15D0FFE71B98B0F107
:10911000007F17D0FFE71B98B0F1407F19D0FFE721
:109120001B98B0F1806F15D0FFE71B98B0F1A06FCE
:1091300011D011E014E02B98083005F05BF88DF8A1
:10914000A3000DE02B98303005F00AF98DF8A3004C
:1091500006E005E004E003E001208DF8A300FFE74E
:109160009DF8A30068B9FFE740F6E041C4F2024170
:10917000086820F0E0602B9AD2F88C201043086039
:1091800004E09DF8A3008DF8A200FFE7FFE72B980D
:109190004078800600283AD5FFE72B98D0F8900059
:1091A0001A9078B1FFE71A98B0F5803F0BD0FFE72F
:1091B0001A98B0F5003F0DD0FFE71A98B0F5403F80
:1091C00009D009E00CE02B98303005F0C9F88DF893
:1091D000A30005E004E003E001208DF8A300FFE711
:1091E0009DF8A30068B9FFE740F6E441C4F20241EC
:1091F000086820F440302B9AD2F890201043086081
:1092000004E09DF8A3008DF8A200FFE7FFE72B988C
:109210004078400600283AD5FFE72B98D0F8940014
:10922000199078B1FFE71998B0F5802F0BD0FFE7C0
:109230001998B0F5002F0DD0FFE71998B0F5402F21
:1092400009D009E00CE02B98303005F089F88DF852
:10925000A30005E004E003E001208DF8A300FFE790
:109260009DF8A30068B9FFE740F6E441C4F202416B
:10927000086820F440202B9AD2F89420104308600C
:1092800004E09DF8A3008DF8A200FFE7FFE72B980C
:109290004078000600283AD5FFE72B98D0F89800D0
:1092A000189078B1FFE71898B0F5801F0BD0FFE752
:1092B0001898B0F5001F0DD0FFE71898B0F5401FC3
:1092C00009D009E00CE02B98303005F049F88DF812
:1092D000A30005E004E003E001208DF8A300FFE710
:1092E0009DF8A30068B9FFE740F6E441C4F20241EB
:1092F000086820F440102B9AD2F898201043086098
:1093000004E09DF8A3008DF8A200FFE7FFE72B988B
:109310004079400700283AD5FFE72B98D0F89C0009
:10932000179078B1FFE71798B0F5800F0BD0FFE7E3
:109330001798B0F5000F0DD0FFE71798B0F5400F64
:1093400009D009E00CE02B98303005F009F88DF8D1
:10935000A30005E004E003E001208DF8A300FFE78F
:109360009DF8A30068B9FFE740F6E441C4F202416A
:10937000086820F440002B9AD2F89C201043086023
:1093800004E09DF8A3008DF8A200FFE7FFE72B980B
:109390008078C007A0B3FFE72B98D0F8A000169004
:1093A00050B1FFE71698B0F1807F06D0FFE716981E
:1093B000B0F1007F08D008E00BE02B98303004F0CB
:1093C000CFFF8DF8A30004E003E001208DF8A30097
:1093D000FFE79DF8A30068B9FFE740F6E441C4F257
:1093E0000241086820F040702B9AD2F8A020104368
:1093F000086004E09DF8A3008DF8A200FFE7FFE7F6
:109400002B9840790007002811D5FFE7FFE740F6C9
:109410001C41C4F20241086820F4004008602B9807
:10942000D0F80421086810430860FFE7FFE72B9895
:109430008078800700284CD5FFE72B98D0F8A4004F
:109440001590C8B1FFE71598B0F5807F15D0FFE7FC
:109450001598B0F5007F17D0FFE71598B0F5407F5D
:1094600019D0FFE71598B0F5806F15D0FFE7159874
:10947000B0F5A06F11D011E014E02B98083004F083
:10948000B9FE8DF8A3000DE02B98303004F068FF92
:109490008DF8A30006E005E004E003E001208DF86C
:1094A000A300FFE79DF8A30068B9FFE740F6DC41A1
:1094B000C4F20241086820F4E0602B9AD2F8A4209C
:1094C0001043086004E09DF8A3008DF8A200FFE7B8
:1094D000FFE72B988078400700284CD5FFE72B98B2
:1094E000D0F8A8001490C8B1FFE71498B0F5805FD9
:1094F00015D0FFE71498B0F5005F17D0FFE7149878
:10950000B0F5405F19D0FFE71498B0F5804F15D043
:10951000FFE71498B0F5A04F11D011E014E02B989C
:10952000083004F067FE8DF8A3000DE02B98303072
:1095300004F016FF8DF8A30006E005E004E003E068
:1095400001208DF8A300FFE79DF8A30068B9FFE7AD
:1095500040F6DC41C4F20241086820F4E0402B9A56
:10956000D2F8A8201043086004E09DF8A3008DF80D
:10957000A200FFE7FFE72B980079800600284CD572
:10958000FFE72B98D0F8AC001390C8B1FFE7139811
:10959000B0F5803F15D0FFE71398B0F5003F17D026
:1095A000FFE71398B0F5403F19D0FFE71398B0F5E7
:1095B000802F15D0FFE71398B0F5A02F11D011E040
:1095C00014E02B98083004F015FE8DF8A3000DE090
:1095D0002B98303004F0C4FE8DF8A30006E005E0BF
:1095E00004E003E001208DF8A300FFE79DF8A3004D
:1095F00068B9FFE740F6DC41C4F20241086820F494
:10960000E0202B9AD2F8AC201043086004E09DF8CB
:10961000A3008DF8A200FFE7FFE72B980079400632
:1096200000284CD5FFE72B98D0F8B0001290C8B1B5
:10963000FFE71298B0F5801F15D0FFE71298B0F53C
:10964000001F17D0FFE71298B0F5401F19D0FFE7B1
:109650001298B0F5800F15D0FFE71298B0F5A00F63
:1096600011D011E014E02B98083004F0C3FD8DF800
:10967000A3000DE02B98303004F072FE8DF8A300AB
:1096800006E005E004E003E001208DF8A300FFE719
:109690009DF8A30068B9FFE740F6DC41C4F202413F
:1096A000086820F4E0002B9AD2F8B020104308603C
:1096B00004E09DF8A3008DF8A200FFE7FFE72B98D8
:1096C0000079000600284CD5FFE72B98D0F8B400AD
:1096D0001190C8B1FFE71198B0F1807F15D0FFE776
:1096E0001198B0F1007F17D0FFE71198B0F1407FDB
:1096F00019D0FFE71198B0F1806F15D0FFE71198EE
:10970000B0F1A06F11D011E014E02B98083004F0F4
:1097100071FD8DF8A3000DE02B98303004F020FE91
:109720008DF8A30006E005E004E003E001208DF8D9
:10973000A300FFE79DF8A30068B9FFE740F6DC410E
:10974000C4F20241086820F0E0602B9AD2F8B420FD
:109750001043086004E09DF8A3008DF8A200FFE725
:10976000FFE72B984079C00700284CD0FFE72B98E3
:10977000D0F8B8001090C8B1FFE71098B0F1805F42
:1097800015D0FFE71098B0F1005F17D0FFE71098F1
:10979000B0F1405F19D0FFE71098B0F1804F15D0BD
:1097A000FFE71098B0F1A04F11D011E014E02B9812
:1097B000083004F01FFD8DF8A3000DE02B98303029
:1097C00004F0CEFD8DF8A30006E005E004E003E020
:1097D00001208DF8A300FFE79DF8A30068B9FFE71B
:1097E00040F6DC41C4F20241086820F0E0402B9AC8
:1097F000D2F8B8201043086004E09DF8A3008DF86B
:10980000A200FFE7FFE72B988078000700284ED5DD
:10981000FFE72B98D0F8C0000F90A0B1FFE70F989A
:10982000B0F5803F18D0FFE70F98B0F5003F1AD091
:10983000FFE70F98B0F5403F1CD0FFE70F98B0F559
:10984000802F18D018E040F62841C4F20241086881
:1098500040F40030086013E02B98083004F0CAFC94
:109860008DF8A3000CE02B98303004F079FD8DF8D2
:10987000A30005E004E003E001208DF8A300FFE76A
:109880009DF8A30068B9FFE740F6E841C4F2024141
:10989000086820F4E0202B9AD2F8C020104308601A
:1098A00004E09DF8A3008DF8A200FFE7FFE72B98E6
:1098B0008078C00600284DD5FFE72B98D0F8C4006B
:1098C0000E90A0B1FFE70E98B0F5002F18D0FFE77B
:1098D0000E98B0F5801F1AD0FFE70E98B0F5C01FA4
:1098E0001CD0FFE70E98B0F5001F17D017E040F628
:1098F0002841C4F20241086840F40030086012E0D8
:109900002B98083004F076FC8DF8A3000BE02B9820
:10991000303004F025FD8DF8A30004E003E00120C1
:109920008DF8A300FFE79DF8A30068B9FFE740F6B4
:10993000E841C4F20241086820F460102B9AD2F882
:10994000C4201043086004E09DF8A3008DF8A20035
:10995000FFE7FFE72B9880788006002834D5FFE7E3
:109960002B98D0F8D4000D90022809D3FFE70D986A
:10997000022806D0FFE70D980338032808D308E033
:109980000BE02B98083004F035FC8DF8A30004E0C0
:1099900003E001208DF8A300FFE79DF8A30068B95C
:1099A000FFE740F6E841C4F20241086820F00700F2
:1099B0002B9AD2F8D4201043086004E09DF8A3004D
:1099C0008DF8A200FFE7FFE72B9840798007002879
:1099D00027D5FFE72B98D0F8D8000C9020B1FFE7EF
:1099E0000C98082801D001E004E003E001208DF884
:1099F000A300FFE79DF8A30068B9FFE740F6E84140
:109A0000C4F20241086820F008002B9AD2F8D8204E
:109A10001043086004E09DF8A3008DF8A200FFE762
:109A2000FFE72B98C0788007002840F1B580FFE75A
:109A300040F62401C4F20241086840F001000860C9
:109A4000FBF7D0FD2990FFE740F62400C4F2024066
:109A50000068C00760B9FFE7FBF7C4FD2999401A09
:109A6000032804D3FFE703208DF8A30000E0EBE711
:109A70009DF8A300002840F08980FFE740F6F04001
:109A8000C4F20240006800F440702A902A98D0B1D5
:109A9000FFE72A982B99D1F8F810884213D0FFE7F6
:109AA00040F6F041C4F20241086820F440702A9068
:109AB000086840F480300860086820F4803008604E
:109AC0002A980860FFE79DF8A800C007E0B1FFE70B
:109AD000FBF788FD2990FFE740F6F040C4F2024012
:109AE0000068800700280ED4FFE7FBF77BFD29996B
:109AF000401A41F28931884204D3FFE703208DF8F0
:109B0000A30000E0E8E7FFE79DF8A300C0BBFFE784
:109B1000FFE72B98D0F8F80000F44070B0F5407FD4
:109B200013D1FFE740F61C41C4F20241086820F45B
:109B30007C502B9AD2F8F8204FF6F043C0F6FF7312
:109B40001A4040EA1210086008E040F61C41C4F2D6
:109B50000241086820F47C500860FFE740F6F041BD
:109B6000C4F20241086820F4407008602B98D0F8D5
:109B7000F8206FF31F32086810430860FFE704E025
:109B80009DF8A3008DF8A200FFE704E09DF8A30074
:109B90008DF8A200FFE7FFE72B98C0784007002868
:109BA00039D5FFE72B98D0F8C8000B9060B1FFE7DC
:109BB0000B98102809D0FFE70B9820280ED0FFE75C
:109BC0000B9830280BD00BE00EE040F62841C4F291
:109BD0000241086840F40030086005E004E003E05A
:109BE00001208DF8A300FFE79DF8A30068B9FFE707
:109BF00040F6E841C4F20241086820F030002B9A98
:109C0000D2F8C8201043086004E09DF8A3008DF846
:109C1000A200FFE7FFE72B9880784006002835D5A3
:109C2000FFE72B98D0F8CC000A9020B1FFE70A9804
:109C3000402809D00FE040F62841C4F202410868EC
:109C400040F4003008600AE02B98083004F0D2FAA3
:109C50008DF8A30003E001208DF8A300FFE79DF835
:109C6000A30068B9FFE740F6E441C4F20241086886
:109C700020F040002B9AD2F8CC201043086004E07A
:109C80009DF8A3008DF8A200FFE7FFE72B988078EE
:109C90000006002835D5FFE72B98D0F8D0000990B2
:109CA00020B1FFE70998802809D00FE040F628414D
:109CB000C4F20241086840F4003008600AE02B98C2
:109CC000083004F097FA8DF8A30003E001208DF826
:109CD000A300FFE79DF8A30068B9FFE740F6E44161
:109CE000C4F20241086820F080002B9AD2F8D020FC
:109CF0001043086004E09DF8A3008DF8A200FFE780
:109D0000FFE72B98C0780007002840D5FFE72B9885
:109D1000D0F8E000089004281ED80899DFE801F088
:109D2000030C131A1B0040F62841C4F202410868D4
:109D300040F40030086013E02B98083004F05AFA21
:109D40008DF8A3000CE02B98303004F009FB8DF85F
:109D5000A30005E004E003E001208DF8A300FFE785
:109D60009DF8A30068B9FFE740F6E041C4F2024164
:109D7000086820F007002B9AD2F8E0201043086012
:109D800004E09DF8A3008DF8A200FFE7FFE72B9801
:109D9000C078C006002840F14F80FFE72B98D0F82C
:109DA000E400079020282CD80799DFE801F0112A59
:109DB0002A2A2A2A2A2A1A2A2A2A2A2A2A2A212A1C
:109DC0002A2A2A2A2A2A282A2A2A2A2A2A2A290020
:109DD00040F62841C4F20241086840F400300860AF
:109DE00013E02B98083004F005FA8DF8A3000CE07E
:109DF0002B98303004F0B4FA8DF8A30005E004E0AD
:109E000003E001208DF8A300FFE79DF8A30068B9E7
:109E1000FFE740F6E041C4F20241086820F0380054
:109E20002B9AD2F8E4201043086004E09DF8A300C8
:109E30008DF8A200FFE7FFE72B98C0788006002886
:109E40004BD5FFE72B98D0F8E800069088B1FFE7E4
:109E50000698402816D0FFE70698802819D0FFE71B
:109E60000698C0281CD0FFE70698B0F5807F18D070
:109E700018E040F62841C4F20241086840F400307E
:109E8000086013E02B98083004F0B4F98DF8A300B3
:109E90000CE02B98303004F063FA8DF8A30005E055
:109EA00004E003E001208DF8A300FFE79DF8A30084
:109EB00068B9FFE740F6E041C4F20241086820F4C7
:109EC000E0702B9AD2F8E8201043086004E09DF877
:109ED000A3008DF8A200FFE7FFE72B98C0784006AB
:109EE00000284CD5FFE72B98D0F8EC000590C8B1BE
:109EF000FFE70598B0F5007F15D0FFE70598B0F5AE
:109F0000806F17D0FFE70598B0F5C06F19D0FFE755
:109F10000598B0F5006F15D0FFE70598B0F5206FF4
:109F200011D011E014E02B98083004F063F98DF89B
:109F3000A3000DE02B98303004F012FA8DF8A30046
:109F400006E005E004E003E001208DF8A300FFE750
:109F50009DF8A30068B9FFE740F6E041C4F2024172
:109F6000086820F460602B9AD2F8EC201043086057
:109F700004E09DF8A3008DF8A200FFE7FFE72B980F
:109F8000C078000600284CD5FFE72B98D0F8F000E9
:109F90000490C8B1FFE70498B0F5805F15D0FFE7E3
:109FA0000498B0F5005F17D0FFE70498B0F5405F64
:109FB00019D0FFE70498B0F5804F15D0FFE704985B
:109FC000B0F5A04F11D011E014E02B98083004F048
:109FD00011F98DF8A3000DE02B98303004F0C0F992
:109FE0008DF8A30006E005E004E003E001208DF811
:109FF000A300FFE79DF8A30068B9FFE740F6E04142
:10A00000C4F20241086820F4E0402B9AD2F8F02014
:10A010001043086004E09DF8A3008DF8A200FFE75C
:10A02000FFE72B980079C00700284CD0FFE72B985A
:10A03000D0F8F4000390C8B1FFE70398B0F5004FE3
:10A0400015D0FFE70398B0F5803F17D0FFE70398DE
:10A05000B0F5C03F19D0FFE70398B0F5003F15D029
:10A06000FFE70398B0F5203F11D011E014E02B98E2
:10A07000083004F0BFF88DF8A3000DE02B983030C5
:10A0800004F06EF98DF8A30006E005E004E003E0BB
:10A0900001208DF8A300FFE79DF8A30068B9FFE752
:10A0A00040F6E041C4F20241086820F460302B9A87
:10A0B000D2F8F4201043086004E09DF8A3008DF866
:10A0C000A200FFE7FFE72B9800798007002838D52A
:10A0D000FFE72B98D0F8DC000290032816D80299ED
:10A0E000DFE801F002030C1314E040F62841C4F24B
:10A0F0000241086840F4003008600BE02B980830FB
:10A1000004F078F88DF8A30004E003E001208DF856
:10A11000A300FFE79DF8A30068B9FFE740F6E4411C
:10A12000C4F20241086820F003002B9AD2F8DC2028
:10A130001043086004E09DF8A3008DF8A200FFE73B
:10A14000FFE72B980079400700283CD5FFE72B98C4
:10A15000D0F8BC00019050B1FFE70198B0F5807FC6
:10A1600006D0FFE70198B0F5007F0AD010E013E0B9
:10A1700040F62841C4F20241086840F4003008600B
:10A180000AE02B98083004F035F88DF8A30003E0BE
:10A1900001208DF8A300FFE79DF8A30068B9FFE751
:10A1A00040F6E841C4F20241086820F440702B9A5E
:10A1B000D2F8BC201043086004E09DF8A3008DF89D
:10A1C000A200FFE7FFE72B980079C00600283BD5E7
:10A1D000FFE72B98D0F800010090102808D0FFE787
:10A1E000009820280DD0FFE70098302810D010E00C
:10A1F00040F62841C4F20241086840F4003008608B
:10A200000BE02B98303004F0ABF88DF8A30004E09D
:10A2100003E001208DF8A300FFE79DF8A30068B9D3
:10A22000FFE740F6E441C4F20241086820F0300044
:10A230002B9AD2F800211043086004E09DF8A30097
:10A240008DF8A200FFE7FFE72B98007900070028B0
:10A250000DD5FFE740F6E841C4F20241086820F05E
:10A26000C0002B9AD2F8FC2010430860FFE79DF84D
:10A27000A2002CB080BD000080B586B00490039190
:10A28000049820B9FFE701208DF817003AE20398FF
:10A2900042F20001C4F20201096801F00F01884294
:10A2A00016D9FFE742F20000C4F20200016821F073
:10A2B0000F01039A11430160006800F00F00039939
:10A2C000884204D0FFE701208DF817001AE2FFE76B
:10A2D00004980078C00600281BD5FFE70498406961
:10A2E00040F62041C4F20241096801F4E041B0EBBC
:10A2F000112F0DD9FFE740F62041C4F20241086852
:10A3000020F4E040049A526940EA02200860FFE726
:10A31000FFE704980078000700281BD5FFE70498A2
:10A32000006940F62041C4F20241096801F4E0618D
:10A33000B0EB111F0DD9FFE740F62041C4F20241F6
:10A34000086820F4E060049A126940EA021008608C
:10A35000FFE7FFE7049800784007002819D5FFE7DA
:10A360000498C06840F62041C4F20241096801F037
:10A37000700188420CD9FFE740F62041C4F2024147
:10A38000086820F07000049AD26810430860FFE764
:10A39000FFE7049800788007002819D5FFE70498A4
:10A3A000806840F62041C4F20241096801F00F01C3
:10A3B00088420CD9FFE740F62041C4F20241086808
:10A3C00020F00F00049A926810430860FFE7FFE74F
:10A3D00004980078C007002800F0D180FFE70498B7
:10A3E000406803280ED1FFE740F60040C4F2024067
:10A3F00000688001002804D4FFE701208DF81700D1
:10A4000080E135E00498406802280ED1FFE740F66D
:10A410000040C4F2024000688003002804D4FFE733
:10A4200001208DF817006DE121E0049840680128B3
:10A430000ED1FFE740F60040C4F2024000688005FC
:10A44000002804D4FFE701208DF817005AE10DE041
:10A4500040F60040C4F2024000688007002804D49F
:10A46000FFE701208DF817004CE1FFE7FFE7FFE76A
:10A4700040F61C41C4F20241086820F00300049A2F
:10A48000526810430860FBF7ADF8019004984068EB
:10A4900003281AD1FFE7FFE740F61C40C4F2024050
:10A4A000006800F0180018280ED0FFE7FBF79AF8B4
:10A4B0000199401A41F28931884204D3FFE7032011
:10A4C0008DF817001EE1E7E758E00498406802287D
:10A4D0001AD1FFE7FFE740F61C40C4F202400068D3
:10A4E00000F0180010280ED0FFE7FBF77BF8019969
:10A4F000401A41F28931884204D3FFE703208DF8E6
:10A500001700FFE0E7E738E00498406801281AD117
:10A51000FFE7FFE740F61C40C4F20240006800F08D
:10A52000180008280ED0FFE7FBF75CF80199401AE5
:10A5300041F28931884204D3FFE703208DF81700E8
:10A54000E0E0E7E718E0FFE740F61C40C4F2024015
:10A55000006810F0180F0ED0FFE7FBF743F80199E1
:10A56000401A41F28931884204D3FFE703208DF875
:10A570001700C7E0E8E7FFE7FFE7FFE7FFE704981A
:10A5800000788007002819D5FFE70498806840F616
:10A590002041C4F20241096801F00F0188420CD247
:10A5A000FFE740F62041C4F20241086820F00F00A6
:10A5B000049A926810430860FFE7FFE7039842F2AD
:10A5C0000001C4F20201096801F00F01884216D2AD
:10A5D000FFE742F20000C4F20200016821F00F011F
:10A5E000039A11430160006800F00F00039988424C
:10A5F00004D0FFE701208DF8170083E0FFE70498FF
:10A6000000784007002819D5FFE70498C06840F695
:10A610002041C4F20241096801F0700188420CD265
:10A62000FFE740F62041C4F20241086820F07000C4
:10A63000049AD26810430860FFE7FFE704980078A7
:10A64000000700281BD5FFE70498006940F6204169
:10A65000C4F20241096801F4E061B0EB111F0DD2B0
:10A66000FFE740F62041C4F20241086820F4E060B0
:10A67000049A126940EA02100860FFE7FFE70498B5
:10A680000078C00600281BD5FFE70498406940F613
:10A690002041C4F20241096801F4E041B0EB112FFE
:10A6A0000DD2FFE740F62041C4F20241086820F4D1
:10A6B000E040049A526940EA02200860FFE7FFE7A1
:10A6C00000F0B0F840F62041C4F20241096801F000
:10A6D0000F0244F6D401C0F60101895CC84040F283
:10A6E0000001C2F20001086040F20C00C2F200005A
:10A6F0000068FAF7BBFF8DF80B009DF80B008DF892
:10A700001700FFE79DF8170006B080BD83B00290E8
:10A71000019102991F20086040F61C40C4F20240DB
:10A72000006800F003000299486040F62040C4F23F
:10A73000024000680090009800F00F0002998860C5
:10A74000009800F070000299C860009800F4E06082
:10A75000000902990861009800F4E040000A02999B
:10A76000486142F20000C4F20200006800F00F00ED
:10A770000199086003B0704780B500F053F840F6C7
:10A780002041C4F20241096801F00F0244F6D401ED
:10A79000C0F60101895C01F01F0120FA01F140F2CD
:10A7A0000000C2F200000160006880BD80B5FFF7C4
:10A7B000E3FF40F62041C4F202410968C1F30212EE
:10A7C00044F6E401C0F60101895C01F01F01C840B4
:10A7D00080BD000080B5FFF7CFFF40F62041C4F2F6
:10A7E00002410968C1F3022244F6E401C0F6010106
:10A7F000895C01F01F01C84080BD000080B5FFF7F3
:10A80000BBFF40F62041C4F202410968C1F30232A5
:10A8100044F6E401C0F60101895C01F01F01C84063
:10A8200080BD000089B040F61C40C4F202400068C0
:10A8300000F01800082806D1FFE740F60010C0F22B
:10A840003D00049048E140F61C40C4F2024000681C
:10A8500010F0180F21D1FFE740F60040C4F202408B
:10A86000006800F020010020B0EB511F0ED0FFE780
:10A8700040F60040C4F202400068C0F3C10149F252
:10A880000000C0F2D030C840049005E049F200005A
:10A89000C0F2D0300490FFE71DE140F61C40C4F246
:10A8A0000240006800F01800102806D1FFE747F6C4
:10A8B0004000C0F27D1004900CE140F61C40C4F250
:10A8C0000240006800F01800182840F0FC80FFE704
:10A8D00040F62840C4F20240016801F003010891EB
:10A8E0000168C1F3052106910068C0F300100590CE
:10A8F000059840F63841C4F20241096889B2C90896
:10A9000000FB01F000EE100AB8EE400A8DED020ADD
:10A910000698002800F0D380FFE7089800900128EF
:10A9200009D0FFE70098022800F08D80FFE700982B
:10A93000032864D088E040F60040C4F2024000687A
:10A9400000F020010020B0EB511F33D0FFE740F6AC
:10A950000040C4F202400068C0F3C10149F20000A7
:10A96000C0F2D030C84003909DED030AB8EE400A13
:10A970009DED061AB8EE411A80EE010A40F6344009
:10A98000C4F2024000686FF35F2001EE100AB8EED7
:10A99000411A9DED022A9FED533A82EE032A31EED1
:10A9A000021AB7EE002A31EE021A20EE010A8DEDEE
:10A9B000010A23E09DED060AB8EE401A9FED4A0A0F
:10A9C00080EE010A40F63440C4F2024000686FF3A2
:10A9D0005F2001EE100AB8EE411A9DED022A9FEDAC
:10A9E000413A82EE032A31EE021AB7EE002A31EE26
:10A9F000021A20EE010A8DED010AFFE748E09DED05
:10AA0000060AB8EE401A9FED360A80EE010A40F6BB
:10AA10003440C4F2024000686FF35F2001EE100A78
:10AA2000B8EE411A9DED022A9FED2E3A82EE032ADE
:10AA300031EE021AB7EE002A31EE021A20EE010AB8
:10AA40008DED010A24E0FFE79DED060AB8EE401AFD
:10AA50009FED260A80EE010A40F63440C4F202401F
:10AA600000686FF35F2001EE100AB8EE411A9DED09
:10AA7000022A9FED1C3A82EE032A31EE021AB7EE4B
:10AA8000002A31EE021A20EE010A8DED010AFFE7DD
:10AA900040F63440C4F20240006881B2012000EB6D
:10AAA000512007909DED010A9DED071AB8EE411A5D
:10AAB00080EE010ABCEEC00A8DED040A02E000201F
:10AAC0000490FFE705E049F20000C0F2D0300490A6
:10AAD000FFE7FFE7FFE7FFE7049809B0704700BF13
:10AAE00020BCBE4B000000460024744C0024744A75
:10AAF00080B588B00690069828B9FFE701208DF848
:10AB00001F0000F0EFBC40F61C40C4F20240006899
:10AB100000F01800049040F62840C4F2024000689B
:10AB200000F00300039006980078C006002840F16A
:10AB30008080FFE70498082808D0FFE704981828C9
:10AB40001DD1FFE70398022819D1FFE70698C069D5
:10AB500028B9FFE701208DF81F0000F0C3BCFFE714
:10AB600040F61841C4F20241086820F47C10069AAD
:10AB7000126A40EA02400860FFE7FFE758E00698E3
:10AB8000C06988B3FFE740F60041C4F2024108689B
:10AB900040F480700860FAF725FD0590FFE740F665
:10ABA0000040C4F202400068800500280DD4FFE791
:10ABB000FAF718FD0599401A032805D3FFE703208B
:10ABC0008DF81F0000F08EBCE9E7FFE740F6184162
:10ABD000C4F20241086820F47C10069A126A40EA26
:10ABE00002400860FFE722E040F60041C4F2024163
:10ABF000086820F480700860FAF7F4FC0590FFE71D
:10AC000040F60040C4F202400068800500280DD5DF
:10AC1000FFE7FAF7E7FC0599401A032805D3FFE799
:10AC200003208DF81F0000F05DBCE9E7FFE7FFE7B8
:10AC3000FFE706980078C007002800F0B980FFE71A
:10AC40000498102808D0FFE7049818280ED1FFE7D1
:10AC5000039803280AD1FFE70698406828B9FFE760
:10AC600001208DF81F0000F03DBCA0E0FFE7069832
:10AC70004068B0F5803F09D1FFE740F60041C4F2DB
:10AC80000241086840F48030086056E00698406849
:10AC900088B9FFE740F60041C4F20241086820F499
:10ACA00080300860086820F480100860086820F48C
:10ACB0008020086040E006984068B0F5A02F11D1D0
:10ACC000FFE740F60041C4F20241086840F48020EA
:10ACD0000860086820F480100860086840F480303C
:10ACE000086028E006984068B0F5A81F11D1FFE77A
:10ACF00040F60041C4F20241086840F48020086038
:10AD0000086840F480100860086840F480300860EB
:10AD100010E040F60041C4F20241086820F480309F
:10AD20000860086820F480200860086820F480101B
:10AD30000860FFE7FFE7FFE7FFE7FFE706984068E7
:10AD4000D0B1FFE7FAF74EFC0590FFE740F6004070
:10AD5000C4F202400068800300280CD4FFE7FAF731
:10AD600041FC0599401A652804D3FFE703208DF8BC
:10AD70001F00B7E3EAE719E0FAF734FC0590FFE7B4
:10AD800040F60040C4F202400068800300280CD561
:10AD9000FFE7FAF727FC0599401A652804D3FFE777
:10ADA00003208DF81F009DE3EAE7FFE7FFE7FFE7D9
:10ADB000069800788007002840F1C380FFE70498D8
:10ADC00040B1FFE7049818285ED1FFE703980128F7
:10ADD0005AD1FFE70698C06820B9FFE701208DF837
:10ADE0001F007FE3049840BBFFE740F60040C4F239
:10ADF0000240006800F018000699096988421BD0DB
:10AE0000FFE740F60041C4F20241086820F0180054
:10AE1000069A126910430860FFF7AEFC40F20C007E
:10AE2000C2F200000068FAF721FC20B1FFE7012020
:10AE30008DF81F0056E3FFE7FFE7FAF7D3FB059015
:10AE4000FFE740F60040C4F2024000688007002897
:10AE50000CD4FFE7FAF7C6FB0599401A032804D380
:10AE6000FFE703208DF81F003CE3EAE740F61041BE
:10AE7000C4F20241086820F4FE00069A526940EAD2
:10AE800002400860FFE75BE00698C068A8B3FFE7F0
:10AE900040F60041C4F20241086820F01800069A0A
:10AEA000126910430860086840F001000860FAF772
:10AEB00099FB0590FFE740F60040C4F202400068AD
:10AEC000800700280CD4FFE7FAF78CFB0599401A9D
:10AED000032804D3FFE703208DF81F0002E3EAE70D
:10AEE00040F61041C4F20241086820F4FE00069AC0
:10AEF000526940EA0240086021E040F60041C4F295
:10AF00000241086820F001000860FAF76BFB059029
:10AF1000FFE740F60040C4F20240006880070028C6
:10AF20000CD5FFE7FAF75EFB0599401A032804D316
:10AF3000FFE703208DF81F00D4E2EAE7FFE7FFE711
:10AF4000FFE7069800780007002849D5FFE7069834
:10AF5000806910B3FFE740F6F041C4F2024108688F
:10AF600040F080600860FAF73DFB0590FFE740F68F
:10AF7000F040C4F202400068000100280CD4FFE752
:10AF8000FAF730FB0599401A032804D3FFE70320A2
:10AF90008DF81F00A6E2EAE721E040F6F041C4F296
:10AFA0000241086820F080600860FAF71BFB0590FA
:10AFB000FFE740F6F040C4F20240006800010028BC
:10AFC0000CD5FFE7FAF70EFB0599401A032804D3C6
:10AFD000FFE703208DF81F0084E2EAE7FFE7FFE7C1
:10AFE000069800784007002840F1CC80FFE740F643
:10AFF0002400C4F202400068C00708BBFFE740F627
:10B000002401C4F20241086840F001000860FAF728
:10B01000E9FA0590FFE740F62400C4F20240006818
:10B02000C00760B9FFE7FAF7DDFA0599401A03286F
:10B0300004D3FFE703208DF81F0053E2EBE7FFE79F
:10B04000FFE706988068012809D1FFE740F6F04144
:10B05000C4F20241086840F00100086054E006981C
:10B06000806888B9FFE740F6F041C4F20241086801
:10B0700020F001000860086820F08000086008687F
:10B0800020F0040008603EE006988068052811D191
:10B09000FFE740F6F041C4F20241086840F00400C6
:10B0A0000860086820F080000860086840F001002F
:10B0B000086027E006988068852811D1FFE740F6F0
:10B0C000F041C4F20241086840F0040008600868DA
:10B0D00040F080000860086840F00100086010E05F
:10B0E00040F6F041C4F20241086820F00100086017
:10B0F000086820F004000860086820F080000860FC
:10B10000FFE7FFE7FFE7FFE7FFE706988068E0B1AA
:10B11000FFE7FAF767FA0590FFE740F6F040C4F260
:10B1200002400068800700280ED4FFE7FAF75AFAB9
:10B130000599401A41F28931884204D3FFE7032080
:10B140008DF81F00CEE1E8E71BE0FAF74BFA059017
:10B15000FFE740F6F040C4F2024000688007002894
:10B160000ED5FFE7FAF73EFA0599401A41F2893108
:10B17000884204D3FFE703208DF81F00B2E1E8E71F
:10B18000FFE7FFE7069800788006002849D5FFE72B
:10B190000698406A10B3FFE740F60041C4F202414E
:10B1A000086840F480500860FAF71CFA0590FFE741
:10B1B00040F60040C4F202400068800400280CD42D
:10B1C000FFE7FAF70FFA0599401A032804D3FFE7BF
:10B1D00003208DF81F0085E1EAE721E040F60041F9
:10B1E000C4F20241086820F480500860FAF7FAF9C6
:10B1F0000590FFE740F60040C4F20240006880047A
:10B2000000280CD5FFE7FAF7EDF90599401A032855
:10B2100004D3FFE703208DF81F0063E1EAE7FFE7AF
:10B22000FFE70698806A002800F05881FFE704983D
:10B23000182800F0D580FFE70698806A022840F0C1
:10B24000A180FFE740F60041C4F20241086820F007
:10B2500080700860FAF7C6F90590FFE740F60040F5
:10B26000C4F202400068800100280CD5FFE7FAF71D
:10B27000B9F90599401A032804D3FFE703208DF894
:10B280001F002FE1EAE7FFE740F62841C4F2024140
:10B29000086843F603729043069BDA6A1B6B42EA26
:10B2A0000322104308600699486BD1F838C0CB6B75
:10B2B0000A6C01386FF35F204FF60061CFF6FF7123
:10B2C00001EB4C2189B208440021CFF6FF7101EB5C
:10B2D000034101F4FE0108444FF07F4101EB02619C
:10B2E00001F0FE41084440F63441C4F202410860D6
:10B2F000FFE740F62841C4F202410091086820F0BF
:10B30000100008600698C06CC00040F63842C4F2D5
:10B3100002421060086840F010000860086820F0E1
:10B320000C00069A526C10430860086820F0200058
:10B33000069A926C10430860086840F480300860F8
:10B3400040F60041C4F20241086840F08070086095
:10B35000FAF748F90590FFE740F60040C4F20240D2
:10B360000068800100280CD4FFE7FAF73BF9059943
:10B37000401A032804D3FFE703208DF81F00B1E033
:10B38000EAE72CE040F60041C4F20241086820F0F0
:10B3900080700860FAF726F90590FFE740F6004054
:10B3A000C4F202400068800100280CD5FFE7FAF7DC
:10B3B00019F90599401A032804D3FFE703208DF8F3
:10B3C0001F008FE0EAE740F62841C4F20241086816
:10B3D0004FF6FC72CFF6F87210400860FFE77CE091
:10B3E00040F62840C4F202400068029040F6344023
:10B3F000C4F20240006801900698806A012837D0A4
:10B40000FFE7029800F003000699C96A88422FD12D
:10B41000FFE7029800F47C510698006BB0EB112F07
:10B4200026D1FFE701986FF35F200699496B013938
:10B4300088421DD1FFE7BDF804100698806B0138E3
:10B44000B0EB512F14D1FFE7019800F4FE010698EC
:10B45000C06B0138B0EB114F0AD1FFE7019800F043
:10B46000FE410698006C0138B0EB116F04D0FFE785
:10B4700001208DF81F0035E040F63840C4F202404C
:10B48000006881B20698C06CB0EBD10F24D0FFE702
:10B4900040F62841C4F20241086820F0100008601C
:10B4A000FAF7A0F80590FFE7FAF79CF80599401A1B
:10B4B00008B9FFE7F8E70698C06CC00040F63841CD
:10B4C000C4F20241086040F62841C4F20241086813
:10B4D00040F010000860FFE7FFE7FFE700208DF86D
:10B4E0001F00FFE79DF81F0008B080BD82B00190EB
:10B4F00001980090042843D80099DFE801F00C1D62
:10B500002F4103004EF21001CEF20001086840F016
:10B510000400086035E04EF21001CEF20001086828
:10B5200020F00400086040F6E441C4F202410868DB
:10B5300020F00C00086024E04EF21001CEF2000171
:10B54000086820F00400086040F6E441C4F20241BB
:10B550000868012262F38300086012E04EF21001D5
:10B56000CEF20001086820F00400086040F6E441D3
:10B57000C4F202410868022262F38300086000E01E
:10B58000FFE702B07047000081B0009001B0704743
:10B5900081B0009001B0704781B0009001B0704759
:10B5A00081B0009001B0704781B0009001B0704749
:10B5B00081B0009001B0704785B003900291FFE721
:10B5C000039890F83C00012804D1FFE702208DF891
:10B5D0001300F6E00399012081F83C00FFE7FFE744
:10B5E0000399022081F83D000398006840680190AB
:10B5F00003980068806800900398006842F6004154
:10B60000C4F2010188421BD0FFE70398006842F6AC
:10B610000041C5F20101884212D0FFE7039800689B
:10B6200043F20041C4F20101884209D0FFE70398C8
:10B63000006843F20041C5F2010188420AD1FFE7E8
:10B64000019820F470000190029841680198084325
:10B650000190FFE701984FF68F71CFF6FF51084038
:10B66000019002980168019808430190019803999C
:10B67000096848600398006842F60041C4F201017D
:10B68000884200F08280FFE70398006842F600419C
:10B69000C5F20101884278D0FFE703980068B0F155
:10B6A000804F72D0FFE703980068B0F1A04F6CD0D4
:10B6B000FFE70398006840F20041C4F200018842AD
:10B6C00063D0FFE70398006840F20041C5F2000133
:10B6D00088425AD0FFE70398006840F60001C4F2A0
:10B6E0000001884251D0FFE70398006840F600014E
:10B6F000C5F20001884248D0FFE70398006840F691
:10B700000041C4F2000188423FD0FFE7039800687F
:10B7100040F60041C5F20001884236D0FFE70398A9
:10B72000006843F20041C4F2010188422DD0FFE7D6
:10B730000398006843F20041C5F20101884224D019
:10B74000FFE70398006841F60001C4F20001884257
:10B750001BD0FFE70398006841F60001C5F2000125
:10B76000884212D0FFE70398006844F20001C4F257
:10B770000101884209D0FFE70398006844F2000104
:10B78000C5F2010188420ED1FFE7009820F0800049
:10B7900000900298816800980843009000980399EF
:10B7A00009688860FFE70399012081F83D00FFE701
:10B7B0000399002081F83C00FFE700208DF813007A
:10B7C000FFE79DF8130005B07047000081B00090BE
:10B7D00001B0704780B582B00090009820B9FFE7B3
:10B7E00001208DF8070045E0009890F83D0040B931
:10B7F000FFE70099002081F83C00009800F03EF837
:10B80000FFE70099022081F83D00009951F8040BF0
:10B8100002F074FF0099012081F84800FFE70099C9
:10B82000012081F83E00009981F83F00009981F8DD
:10B830004000009981F84100009981F84200009988
:10B8400081F84300FFE7FFE70099012081F84400F9
:10B85000009981F84500009981F84600009981F827
:10B860004700FFE70099012081F83D0000208DF896
:10B870000700FFE79DF8070002B080BD80B58EB0DD
:10B880000D9000200C900B900A90099008900D9854
:10B890000068B0F1804F19D1FFE7FFE740F69C4008
:10B8A000C4F20240016841F001010160006800F04B
:10B8B000010007900798FFE72D2003900022114612
:10B8C000F9F752FF0398F9F745FF5CE00D9800681F
:10B8D00040F20041C4F20001884239D1FFE7FFE79E
:10B8E00040F69C40C4F20240016841F00201016050
:10B8F000006800F0020006900698FFE7FFE740F6B8
:10B900008C40C4F20240016841F00401016000680B
:10B9100000F0040005900598FFE74FF48070089050
:10B9200002200990002101910A910B910C9040F6A0
:10B930000000C4F2022008A9F9F7C8FC019A2E20E1
:10B9400002901146F9F710FF0298F9F703FF19E08A
:10B950000D98006840F60001C4F20001884210D141
:10B96000FFE7FFE740F69C40C4F20240016841F067
:10B9700004010160006800F0040004900498FFE7EF
:10B98000FFE7FFE7FFE70EB080BD000083B0019046
:10B99000019890F83D00012804D0FFE701208DF8C0
:10B9A0000B00B8E00199022081F83D000198016880
:10B9B000C86840F00100C8600198006842F6004184
:10B9C000C4F20101884200F08280FFE7019800681C
:10B9D00042F60041C5F20101884278D0FFE70198A4
:10B9E0000068B0F1804F72D0FFE701980068B0F1B5
:10B9F000A04F6CD0FFE70198006840F20041C4F20C
:10BA00000001884263D0FFE70198006840F20041DE
:10BA1000C5F2000188425AD0FFE70198006840F65D
:10BA20000001C4F20001884251D0FFE7019800688C
:10BA300040F60001C5F20001884248D0FFE70198B6
:10BA4000006840F60041C4F2000188423FD0FFE7A1
:10BA50000198006840F60041C5F20001884236D0E6
:10BA6000FFE70198006843F20041C4F201018842F7
:10BA70002DD0FFE70198006843F20041C5F20101B3
:10BA8000884224D0FFE70198006841F60001C4F223
:10BA9000000188421BD0FFE70198006841F60001D1
:10BAA000C5F20001884212D0FFE70198006844F215
:10BAB0000001C4F20101884209D0FFE70198006843
:10BAC00044F20001C5F20101884219D1FFE7019853
:10BAD000006880680721C0F20101084000900098CA
:10BAE00006280CD0FFE70098B0F5803F07D0FFE7AD
:10BAF00001980168086840F001000860FFE706E06F
:10BB000001980168086840F001000860FFE7002024
:10BB10008DF80B00FFE79DF80B0003B070470000A5
:10BB200080B586B00490039100208DF80B00FFE7EC
:10BB3000049890F83C00012804D1FFE702208DF81A
:10BB40001700EDE00499012081F83C00FFE7FFE7D2
:10BB50000499022081F83D000498006880680190F3
:10BB600001984FF68871CFF6CE7108400190019888
:10BB700020F47F4001900198049909688860039837
:10BB800000680090002800F0B180FFE700981028BE
:10BB900000F0AC80FFE70098202800F0A780FFE7C6
:10BBA0000098302800F0A280FFE70098402800F0BD
:10BBB0009080FFE70098502871D0FFE70098602838
:10BBC0007AD0FFE70098702845D0FFE70098B0F5DD
:10BBD000805F3FD0FFE70098B0F5005F50D0FFE7EF
:10BBE0000098B0F5801F00F08180FFE70098B0F169
:10BBF000101F7BD0FFE700982021C0F2100188427F
:10BC000074D0FFE700983021C0F2100188426DD057
:10BC1000FFE700984021C0F21001884266D0FFE79C
:10BC200000985021C0F2100188425FD0FFE70098D1
:10BC30006021C0F21001884258D0FFE700987021BF
:10BC4000C0F21001884251D0FFE70098B0F5001F04
:10BC50004CD052E055E004980068039B5A689968FC
:10BC6000DB6802F0F9FE0498006880680190019892
:10BC700040F077000190019804990968886040E0DD
:10BC800004980068039B5A689968DB6802F0E4FE38
:10BC900004980168886840F48040886031E0049826
:10BCA0000068039A5168D26803F03EFC049800686B
:10BCB000502102F0EBFE24E004980068039A5168DA
:10BCC000D26803F035FD04980068602102F0DEFEC2
:10BCD00017E004980068039A5168D26803F024FCC6
:10BCE00004980068402102F0D1FE0AE00498006840
:10BCF0000399096802F0CAFE03E001208DF80B00E9
:10BD0000FFE70499012081F83D00FFE70499002036
:10BD100081F83C00FFE79DF80B008DF81700FFE766
:10BD20009DF8170006B080BD80B586B004900391E1
:10BD3000049820B9FFE701208DF817008AE00498E5
:10BD400090F83D0040B9FFE70499002081F83C00DD
:10BD5000049800F083F8FFE70499022081F83D0081
:10BD60000498016888684BF6F872CFF6FE721040AE
:10BD70008860049951F8040B02F0C0FC0498006834
:10BD800080680290049800688069019004980068B7
:10BD9000006A009003980168029808430290019895
:10BDA00040F203318843019003998868896940EA29
:10BDB0000121019808430190019840F60C41884305
:10BDC000019001984FF2F001884301900399C868EF
:10BDD000C96940EA01210198084301900399086963
:10BDE000096A000140EA0131019808430190009876
:10BDF00020F022000090009820F088000090039925
:10BE00004868496940EA0111009808430090029887
:10BE10000499096888600198049909688861009804
:10BE20000499096808620499012081F8480004997E
:10BE300081F83E00049981F83F00049981F844009C
:10BE4000049981F84500049981F83D0000208DF89F
:10BE50001700FFE79DF8170006B080BD80B58AB0D7
:10BE6000099000200890079006900590049009988A
:10BE7000006842F60041C4F20101884230D1FFE778
:10BE8000FFE740F6A440C4F20240016841F40061BB
:10BE90000160006800F4006003900398FFE7FFE78B
:10BEA00040F68C40C4F20240016841F0100101608C
:10BEB000006800F0100002900298FFE74FF4206045
:10BEC0000490022005900020069007900120089021
:10BED00041F20000C4F2022004A9F9F7F7F938E0B2
:10BEE0000998006843F20041C4F2010188422FD151
:10BEF000FFE7FFE740F6A440C4F20240016841F4C6
:10BF000000510160006800F4005001900198FFE7C3
:10BF1000FFE740F68C40C4F20240016841F00401A2
:10BF20000160006800F0040000900098FFE7C02066
:10BF300004900220059000200690079003200890AE
:10BF400040F60000C4F2022004A9F9F7BFF9FFE7A8
:10BF5000FFE70AB080BD000080B584B0039003986D
:10BF6000007F022840F08480FFE742F27020C2F296
:10BF700000000078F0B9FFE70398042100F090FC7E
:10BF800042F26821C2F200010860FFE703980168ED
:10BF9000086A20F0A000086203980168086A40F06F
:10BFA00020000862FFE742F27021C2F20001012086
:10BFB00008705CE00398042100F072FC42F26C21EE
:10BFC000C2F200010860FFE703980168086A20F0E8
:10BFD000A000086203980168086A0862FFE742F25D
:10BFE0007021C2F200010020087042F26C20C2F2FF
:10BFF0000000006842F26821C2F20001096888422C
:10C000000DD9FFE742F26C20C2F20000006842F254
:10C010006821C2F200010968401A01900FE042F263
:10C020006820C2F20000016842F26C20C2F20000F7
:10C030000068401A4FF6FF7108440190FFE701982D
:10C04000029002984CF60931C8F63D51A0FB011050
:10C05000400941F67851C2F20001086042F2E860FE
:10C06000C2F200000121002207F03EF8FFE7FFE7DF
:10C0700004B080BD80B586B0049003910292002088
:10C080008DF80700FFE7049890F83C00012804D1E0
:10C09000FFE702208DF8170080E00499012081F865
:10C0A0003C00FFE7FFE70298B0B9FFE7049800689B
:10C0B000039B19685A68DB6803F05EFA049801680C
:10C0C000886920F00C0088610398826804980168F0
:10C0D00088691043886156E00298042817D1FFE769
:10C0E00004980068039B19685A68DB6803F04AFBF0
:10C0F00004980168886920F4406088610398826828
:10C1000004980168886940EA022088613AE0029850
:10C11000082816D1FFE704980068039B19685A683D
:10C12000DB6803F065FB04980168C86920F00C0027
:10C13000C8610398826804980168C8691043C8619F
:10C140001FE002980C2817D1FFE704980068039BB2
:10C1500019685A68DB6803F081FB04980168C869B4
:10C1600020F44060C8610398826804980168C86937
:10C1700040EA0220C86103E001208DF80700FFE7D4
:10C18000FFE7FFE7FFE7FFE70499002081F83C00A5
:10C19000FFE79DF807008DF81700FFE79DF81700EF
:10C1A00006B080BD80B582B00090009820B9FFE74E
:10C1B00001208DF8070045E0009890F83D0040B957
:10C1C000FFE70099002081F83C00009800F03EF85D
:10C1D000FFE70099022081F83D00009951F8040B17
:10C1E00002F08CFA0099012081F84800FFE70099DD
:10C1F000012081F83E00009981F83F00009981F804
:10C200004000009981F84100009981F842000099AE
:10C2100081F84300FFE7FFE70099012081F844001F
:10C22000009981F84500009981F84600009981F84D
:10C230004700FFE70099012081F83D0000208DF8BC
:10C240000700FFE79DF8070002B080BD81B00090B5
:10C2500001B0704780B584B0039003980068C0684F
:10C26000029003980068006901909DF8040080071F
:10C27000002824D5FFE79DF80800800700281DD579
:10C28000FFE7039801686FF002000861039901203D
:10C290000877039800688069800720B1FFE703985A
:10C2A000FFF75AFE06E0039800F0B0F9039800F09B
:10C2B000E1FAFFE7039900200877FFE7FFE79DF821
:10C2C00004004007002825D5FFE79DF80800400737
:10C2D00000281ED5FFE7039801686FF0040008618D
:10C2E00003990220087703980068806910F4407F62
:10C2F00004D0FFE70398FFF72FFE06E0039800F055
:10C3000085F9039800F0B6FAFFE703990020087753
:10C31000FFE7FFE79DF804000007002824D5FFE7AA
:10C320009DF80800000700281DD5FFE70398016865
:10C330006FF00800086103990420087703980068EB
:10C34000C069800720B1FFE70398FFF705FE06E00C
:10C35000039800F05BF9039800F08CFAFFE703996B
:10C3600000200877FFE7FFE79DF80400C0060028DB
:10C3700025D5FFE79DF80800C00600281ED5FFE779
:10C38000039801686FF0100008610399082008778E
:10C3900003980068C06910F4407F04D0FFE7039859
:10C3A000FFF7DAFD06E0039800F030F9039800F09B
:10C3B00061FAFFE7039900200877FFE7FFE79DF8A0
:10C3C0000400C00778B1FFE79DF80800C00748B136
:10C3D000FFE7039801686FF001000861039800F01F
:10C3E0004DFAFFE7FFE7019800F08000802806D0B3
:10C3F000FFE79DF805008006002810D5FFE79DF8AF
:10C4000008000006002809D5FFE7039801686FF4CB
:10C41000025008610398FFF7BBF8FFE7FFE79DF8BC
:10C420000500C00780B1FFE79DF80800000600285E
:10C4300009D5FFE7039801686FF4807008610398DD
:10C44000FFF7A2F8FFE7FFE79DF804004006002889
:10C4500010D5FFE79DF808004006002809D5FFE742
:10C46000039801686FF040000861039800F044FAF7
:10C47000FFE7FFE79DF804008006002810D5FFE7DE
:10C480009DF808008006002809D5FFE70398016899
:10C490006FF0200008610398FFF77EF8FFE7FFE7E1
:10C4A0009DF80600C006002810D5FFE79DF80A0099
:10C4B000C006002809D5FFE7039801686FF48010D3
:10C4C00008610398FFF770F8FFE7FFE79DF80600A3
:10C4D0008006002810D5FFE79DF80A008006002896
:10C4E00009D5FFE7039801686FF40010086103980D
:10C4F000FFF756F8FFE7FFE79DF806004006002823
:10C5000010D5FFE79DF80A004006002809D5FFE78F
:10C51000039801686FF4800008610398FFF748F8FA
:10C52000FFE7FFE79DF806000006002810D5FFE7AB
:10C530009DF80A000006002809D5FFE70398016866
:10C540006FF4000008610398FFF740F9FFE7FFE789
:10C5500004B080BD80B588B007900020069005909B
:10C560000490039002900798006840F20041C4F2E2
:10C57000000188421ED1FFE7FFE740F68C40C4F27D
:10C580000240016841F002010160006800F0020011
:10C5900001900198FFE7022002900390002104918E
:10C5A0000591069040F20040C4F2022002A9F8F77B
:10C5B0008DFE28E00798006840F60001C4F20001F3
:10C5C00088421FD1FFE7FFE740F68C40C4F20240EB
:10C5D000016841F004010160006800F0040000906F
:10C5E0000098FFE7042002900220039000210491AC
:10C5F0000591069040F60000C4F2022002A9F8F767
:10C6000065FEFFE7FFE708B080BD000081B0009045
:10C6100001B0704780B586B004900391029200206B
:10C620008DF80700FFE7049890F83C00012804D13A
:10C63000FFE702208DF81700C0E00499012081F87F
:10C640003C00FFE7FFE702980090142800F2A78063
:10C650000099DFE801F00BA4A4A424A4A4A43EA4A0
:10C66000A4A457A4A4A471A4A4A48A000498006854
:10C67000039902F023FA04980168886940F00800E1
:10C68000886104980168886920F004008861039833
:10C6900002690498016888691043886183E00498FE
:10C6A0000068039902F004FB04980168886940F46B
:10C6B0000060886104980168886920F4806088615E
:10C6C0000398026904980168886940EA0220886139
:10C6D00069E004980068039902F0F2FB049801688D
:10C6E000C86940F00800C86104980168C86920F072
:10C6F0000400C8610398026904980168C86910437E
:10C70000C86150E004980068039902F0E1FC0498C5
:10C710000168C86940F40060C86104980168C8698C
:10C7200020F48060C8610398026904980168C869B0
:10C7300040EA0220C86136E004980068039902F0DC
:10C74000CFFD04980168086D40F008000865049862
:10C750000168086D20F004000865039802690498D8
:10C760000168086D104308651DE00498006803998E
:10C7700002F048FE04980168086D40F40060086506
:10C7800004980168086D20F48060086503980269C8
:10C7900004980168086D40EA0220086503E0012062
:10C7A0008DF80700FFE7FFE70499002081F83C00BF
:10C7B000FFE79DF807008DF81700FFE79DF81700C9
:10C7C00006B080BD80B582B00090009820B9FFE728
:10C7D00001208DF8070045E0009890F83D0040B931
:10C7E000FFE70099002081F83C00009800F03EF837
:10C7F000FFE70099022081F83D00009951F8040BF1
:10C8000001F07CFF0099012081F84800FFE70099C2
:10C81000012081F83E00009981F83F00009981F8DD
:10C820004000009981F84100009981F84200009988
:10C8300081F84300FFE7FFE70099012081F84400F9
:10C84000009981F84500009981F84600009981F827
:10C850004700FFE70099012081F83D0000208DF896
:10C860000700FFE79DF8070002B080BD81B000908F
:10C8700001B0704781B0009001B0704780B582B0C0
:10C8800001900198006841F20001C4F20001884261
:10C8900003D1FFE7F8F7ACFEFFE702B080BD000070
:10C8A00084B00390029100200190029800900C281F
:10C8B0001DD80099DFE801F0071B1B1B0C1B1B1B7D
:10C8C000111B1B1B160003980068406B01900FE0C2
:10C8D00003980068806B01900AE003980068C06BC1
:10C8E000019005E003980068006C019000E0FFE70C
:10C8F000019804B07047000081B0009001B070470B
:10C9000083B00190FFE7019890F88400012804D1DA
:10C91000FFE702208DF80B002CE00199012081F83F
:10C920008400FFE7FFE701992420C1F888000198FF
:10C9300000680068009001980168086820F0010014
:10C940000860009820F0005000900199002048668F
:10C95000009801990968086001992020C1F88800B1
:10C96000FFE70199002081F88400FFE700208DF89F
:10C970000B00FFE79DF80B0003B0704780B586B051
:10C9800004900391ADF80A2000208DF80900049866
:10C99000D0F88C0020284BD1FFE7039820B1FFE7A7
:10C9A000BDF80A0020B9FFE701208DF8170043E029
:10C9B0000498006880684006002807D5FFE70498BF
:10C9C0000168886820F040008860FFE70499012032
:10C9D000C86604990020086704980399BDF80A20E6
:10C9E00004F0EAF80498C06E012818D1FFE7049813
:10C9F000016810200862FFE7FFE70498006850E82C
:10CA0000000F40F010000190FFE7019904980268C0
:10CA100042E800100028F0D1FFE7FFE703E0012023
:10CA20008DF80900FFE79DF809008DF8170003E075
:10CA300002208DF81700FFE79DF8170006B080BDB3
:10CA400080B584B00390ADF80A100398006844F6EE
:10CA50000041C4F2000188424ED1FFE70020ADF84A
:10CA60000800FFE7BDF80800BDF80A1088422FDA79
:10CA7000FFE7BDF8081042F2A860C2F20000405C77
:10CA80008DF8070040F65401C2F20001B1F8000130
:10CA90000130C0B2ADF80400BDF80400B1F80211D5
:10CAA00088420ED0FFE79DF8070040F65401C2F21D
:10CAB0000001B1F800218854BDF80400A1F800017C
:10CAC000FFE7FFE7BDF808000130ADF80800C9E74F
:10CAD00040F63000C2F200000121002206F004FB03
:10CAE00042F2D410C2F2000042F2A861C2F2000188
:10CAF0004022FFF743FFFFE704B080BD81B0009004
:10CB000001B0704780B584B002900191FFE70298B0
:10CB100090F88400012804D1FFE702208DF80F006F
:10CB200032E00299012081F88400FFE7FFE70299D3
:10CB30002420C1F8880002980068006800900298DC
:10CB40000168086820F001000860029800688068A9
:10CB500020F0606001990843029909688860029892
:10CB600002F0BAFE00980299096808600299202034
:10CB7000C1F88800FFE70299002081F88400FFE7F0
:10CB800000208DF80F00FFE79DF80F0004B080BD76
:10CB900080B584B002900191FFE7029890F884007C
:10CBA000012804D1FFE702208DF80F0032E002993E
:10CBB000012081F88400FFE7FFE702992420C1F8F3
:10CBC0008800029800680068009002980168086870
:10CBD00020F00100086002980068806820F0604042
:10CBE00001990843029909688860029802F074FE6E
:10CBF000009802990968086002992020C1F888000D
:10CC0000FFE70299002081F88400FFE700208DF8FB
:10CC10000F00FFE79DF80F0004B080BD81B00090C9
:10CC200001B0704781B0009001B0704781B00090B2
:10CC300001B0704780B58EB00D900D980068C06946
:10CC40000C900D98006800680B900D980068806843
:10CC50000A900C9840F60F01084009900998E0B935
:10CC6000FFE79DF830008006002815D5FFE79DF806
:10CC70002C008006002806D4FFE79DF82B00C00694
:10CC8000002809D5FFE70D98406F20B1FFE70D9808
:10CC9000416F8847FFE76CE2FFE70998002800F042
:10CCA000F980FFE70A980121C1F20001084209D189
:10CCB000FFE70B9840F22011C0F20041084200F05B
:10CCC000E980FFE79DF83000C00788B1FFE79DF8D5
:10CCD0002D00C00760B1FFE70D98016801200862D0
:10CCE0000D99D1F8900040F00100C1F89000FFE7E5
:10CCF0009DF830008007002811D5FFE79DF8280037
:10CD0000C00760B1FFE70D980168022008620D9925
:10CD1000D1F8900040F00400C1F89000FFE79DF8C2
:10CD200030004007002811D5FFE79DF82800C00714
:10CD300060B1FFE70D980168042008620D99D1F8F1
:10CD4000900040F00200C1F89000FFE79DF830002D
:10CD50000007002819D5FFE79DF82C008006002861
:10CD600007D4FFE70A980121C1F2000108420CD064
:10CD7000FFE70D980168082008620D99D1F890002E
:10CD800040F00800C1F89000FFE79DF8310000076F
:10CD9000002813D5FFE79DF82F00400700280DD588
:10CDA000FFE70D9801684FF4006008620D99D1F813
:10CDB000900040F02000C1F89000FFE70D98D0F8F7
:10CDC0009000002865D0FFE79DF83000800600281D
:10CDD00015D5FFE79DF82C008006002806D4FFE754
:10CDE0009DF82B00C006002809D5FFE70D98406F7D
:10CDF00020B1FFE70D98416F8847FFE7FFE70D98E7
:10CE0000D0F8900008900D980068806800F040000D
:10CE1000402806D0FFE79DF8200010F0280F2FD003
:10CE2000FFE70D9802F06CFF0D98006880684006DF
:10CE3000002820D5FFE70D98D0F88000B0B1FFE7BB
:10CE40000D98D0F880104FF6F530C0F60000C86697
:10CE50000D98D0F88000F7F719FE30B1FFE70D9874
:10CE6000D0F88000C16E8847FFE703E00D98FFF718
:10CE7000DDFEFFE703E00D98FFF7D8FEFFE707E0D0
:10CE80000D98FFF7D3FE0D990020C1F89000FFE741
:10CE9000FFE76EE10D98C06E012840F00B81FFE7BF
:10CEA0009DF83000C006002840F10481FFE79DF89E
:10CEB0002C00C006002840F1FD80FFE70D980168B6
:10CEC000102008620D98006880684006002840F134
:10CED0008F80FFE70D98D0F880000068806CADF877
:10CEE0001E00BDF81E00002867D0FFE7BDF81E0039
:10CEF0000D99B1F85C1088425FDAFFE7BDF81E00BB
:10CF00000D99A1F85E000D98D0F88000006D812881
:10CF100046D0FFE7FFE7FFE70D98006850E8000FF5
:10CF200020F480700690FFE706990D98026842E8A9
:10CF300000100028F0D1FFE7FFE7FFE7FFE70D98BB
:10CF4000006850E8020F20F001000590FFE7059906
:10CF50000D98026842E802100028F0D1FFE7FFE7D1
:10CF60000D992020C1F88C000D990020C866FFE7BC
:10CF7000FFE70D98006850E8000F20F010000490C3
:10CF8000FFE704990D98026842E800100028F0D1EC
:10CF9000FFE7FFE70D98D0F88000F7F7EBFCFFE71D
:10CFA0000D99022008670D98B0F85C10B0F85E206B
:10CFB000891A89B2FFF744FD19E0BDF81E000D99EA
:10CFC000B1F85C10884211D1FFE70D98D0F88000CD
:10CFD000006D812809D1FFE70D99022008670D989F
:10CFE000B0F85C10FFF72CFDFFE7FFE7FFE7C0E0BC
:10CFF0000D99B1F85C00B1F85E10401AADF80E0062
:10D000000D98B0F85E00002853D0FFE7BDF80E0081
:10D0100000284ED0FFE7FFE7FFE70D98006850E8D3
:10D02000000F20F490700290FFE702990D980268BB
:10D0300042E800100028F0D1FFE7FFE7FFE7FFE735
:10D040000D98006850E8020F4FF6FE71CEF6FF71A2
:10D0500008400190FFE701990D98026842E802102C
:10D060000028EDD1FFE7FFE70D992020C1F88C00E3
:10D070000D990020C8660D994867FFE7FFE70D98F6
:10D08000006850E8000F20F010000090FFE70099C2
:10D090000D98026842E800100028F0D1FFE7FFE792
:10D0A0000D99022008670D98BDF80E10FFF7C8FC17
:10D0B000FFE75EE09DF83200C00600280FD5FFE7CD
:10D0C0009DF82A004006002809D5FFE70D98016861
:10D0D0004FF4801008620D98FFF7A4FD49E09DF819
:10D0E00030000006002815D5FFE79DF82C0000064B
:10D0F000002806D4FFE79DF82A000006002809D57D
:10D10000FFE70D98806F20B1FFE70D98816F88478A
:10D11000FFE72EE09DF83000400600280AD5FFE723
:10D120009DF82C004006002804D5FFE70D9802F07A
:10D1300037FE1EE09DF83200000600280AD5FFE702
:10D140009DF82F004006002804D5FFE70D98FFF753
:10D1500065FD0EE09DF83300C00750B1FFE79DF874
:10D160002F000006002804D5FFE70D98FFF7C6FC46
:10D17000FFE70EB080BD000080B582B0009000983F
:10D1800020B9FFE701208DF8070046E0009880698C
:10D1900008B1FFE700E0FFE70098D0F8880040B949
:10D1A000FFE70099002081F88400009800F03AF829
:10D1B000FFE700992420C1F88800009801680868FA
:10D1C00020F0010008600098806A20B1FFE7009815
:10D1D00002F0C8FBFFE7009803F0E2FA012804D14F
:10D1E000FFE701208DF8070017E000980168486804
:10D1F00020F49040486000980168886820F02A0078
:10D20000886000980168086840F001000860009894
:10D2100002F04CFC8DF80700FFE79DF8070002B014
:10D2200080BD000080B5F2B07190002070906F90CA
:10D230006E906D906C9051A86C21F3F7F6FA0EA8E1
:10D240004FF48471F3F7F1FA7198006844F60041E5
:10D25000C4F20001884240F0FF80FFE700200F90F9
:10D2600008210E9128900EA8FBF78EFB18B1FFE75E
:10D27000F6F7CAFEFFE7FFE740F69C40C4F2024023
:10D28000016841F400210160006800F400200D9065
:10D290000D98FFE7FFE740F68C40C4F202400168BA
:10D2A00041F002010160006800F002000C900C984F
:10D2B000FFE74FF440706C9002206D9000200790C3
:10D2C0006E906F900820709040F20040C4F20220EF
:10D2D0006CA9F7F7FBFF0798212151911B2152916F
:10D2E00053905490559056905790589001215A91D0
:10D2F0005B914FF040215C915D905E9062905F90F9
:10D30000609040F2CC11C2F2000151A8F6F798FEED
:10D3100018B1FFE7F6F778FEFFE740F29010C2F28F
:10D32000000040F2CC12C2F200020021F7F778F8B8
:10D3300018B1FFE7F6F768FEFFE740F29010C2F27F
:10D340000000F7F70DFA18B1FFE7F6F75DFEFFE70B
:10D3500041F66C60C2F2000040F2D021C4F202013A
:10D36000016000218163C1634FF4003202644164B3
:10D3700081218164F6F792FE18B1FFE7F6F744FECB
:10D38000FFE741F66C60C2F2000040F29011C2F279
:10D390000001F7F713F918B1FFE7F6F735FEFFE7DD
:10D3A000FFE7719841F66C61C2F20001C0F880108D
:10D3B0007198C865FFE741F66C60C2F20000102169
:10D3C000F7F78EFB18B1FFE7F6F71EFEFFE741F611
:10D3D000F450C2F20000059040F25021C4F2020164
:10D3E00001601C2141600021069181604FF4806240
:10D3F000C2600822026141618161C1610162012252
:10D4000042628262C16201634163F7F70DFD18B1A8
:10D41000FFE7F6F7F9FDFFE7FFE7719841F6F451F2
:10D42000C2F20001C1677198C865FFE741F6F45088
:10D43000C2F200001021F7F753FB18B1FFE7F6F72F
:10D44000E3FDFFE73D20049000221146F8F78CF938
:10D450000498F8F77FF919E17198006844F20041E7
:10D46000C4F20001884240F0BF80FFE700200F9027
:10D4700002210E9126900EA8FBF786FA18B1FFE75D
:10D48000F6F7C2FDFFE7FFE740F69C40C4F202401A
:10D49000016841F400310160006800F400300B9035
:10D4A0000B98FFE7FFE740F68C40C4F202400168AA
:10D4B00041F008010160006800F008000A900A9835
:10D4C000FFE760206C9002206D90002003906E902A
:10D4D0006F900720709040F60040C4F202206CA9C3
:10D4E000F7F7F4FE0398212151911721529153909F
:10D4F0005490559056905790589001215A915B91B5
:10D500005C905D905E9062905F90609040F2A81198
:10D51000C2F2000151A8F6F793FD18B1FFE7F6F744
:10D5200073FDFFE740F27810C2F2000040F2A8124B
:10D53000C2F200020021F6F773FF18B1FFE7F6F719
:10D5400063FDFFE740F27810C2F20000F7F708F938
:10D5500018B1FFE7F6F758FDFFE741F67C50C2F23D
:10D56000000040F2D011C4F2020101600021816389
:10D57000C1630164416481218164F6F78FFD18B1B4
:10D58000FFE7F6F741FDFFE741F67C50C2F20000ED
:10D5900040F27811C2F20001F7F710F818B1FFE776
:10D5A000F6F732FDFFE7FFE7719841F67C51C2F2D2
:10D5B0000001C0F880107198C865FFE741F67C5003
:10D5C000C2F200001021F7F78BFA18B1FFE7F6F767
:10D5D0001BFDFFE73B20029000221146F8F7C4F83C
:10D5E0000298F8F7B7F850E07198006844F6000127
:10D5F000C4F20001884247D1FFE700200F900421C8
:10D600000E9127900EA8FBF7BFF918B1FFE7F6F7C8
:10D61000FBFCFFE7FFE740F69C40C4F202400168D4
:10D6200041F480210160006800F48020099009988D
:10D63000FFE7FFE740F68C40C4F20240016841F08A
:10D6400004010160006800F0040008900898FFE7FA
:10D650004FF440606C9002206D90002000906E901E
:10D660006F900720709040F60000C4F202206CA971
:10D67000F7F72CFE009A3C2001901146F8F774F859
:10D680000198F8F767F8FFE7FFE7FFE772B080BDA2
:10D6900081B0009001B0704780B586B004900391CE
:10D6A000ADF80A20BDF80A00ADF806000498D0F8DD
:10D6B0008800202840F0BA80FFE7039820B1FFE7F8
:10D6C000BDF80A0020B9FFE701208DF81700B1E08E
:10D6D000039804990865BDF80A000499A1F854005C
:10D6E000BDF80A000499A1F8560004990020C1F879
:10D6F000900004992120C1F8880004980168402016
:10D7000008620498C06F002879D0FFE70498C16FC1
:10D710004FF69540C0F6000008660498C16F4FF6BA
:10D72000E940C0F6000048660498C16F4FF6154006
:10D73000C0F6000088660498C16F0020C86604988F
:10D740008068B0F5805F0AD1FFE70498006930B9BE
:10D75000FFE7BDF80A004000ADF80600FFE70498B7
:10D76000C06F90F85000000600282BD5FFE7049802
:10D77000C06F406F08B3FFE70498C06F406F006848
:10D78000D8B1FFE7BDF806000499C96F496F096871
:10D7900088600499086DC96F496F0968C860049969
:10D7A0000868C96F2830496F096808610498C06F1C
:10D7B000F7F73CF88DF8090003E001208DF8090027
:10D7C000FFE70BE004980268016DC06F2832BDF8D6
:10D7D0000630F7F709FD8DF80900FFE79DF809000D
:10D7E00060B1FFE704991020C1F89000049920204F
:10D7F000C1F8880001208DF817001BE0FFE7FFE764
:10D80000FFE70498006850E8020F40F080000090A5
:10D81000FFE700990498026842E802100028F0D15E
:10D82000FFE7FFE700208DF8170003E002208DF8E6
:10D830001700FFE79DF8170006B080BD81B000908B
:10D8400001B0704781B0009001B0704780B586B0DC
:10D85000FFE740F65401C2F20001B1F80201B1F84D
:10D860000011884200F0AC80FFE740F65401C2F29C
:10D870000001B1F80201085C8DF81700B1F802014F
:10D880000130C0B2A1F8020140F2F400C2F200007F
:10D89000006838BBFFE79DF81700232821D1FFE778
:10D8A00040F27001C2F2000101910020086040F2D4
:10D8B000F401C2F200010120086040F27400C2F2DB
:10D8C000000002908021F2F78EFFDDF804C002997B
:10D8D0009DF81700DCF80020531CCCF80030885469
:10D8E000FFE7B6E740F27000C2F2000000687E2851
:10D8F00052D8FFE79DF8170040F27003C2F2000310
:10D900001A68511C196040F27401C2F20001885477
:10D910009DF817000A283ED1FFE740F27000C2F2DE
:10D920000000026840F27400C2F20000002181543D
:10D9300044F64121C0F6010104AA03ABF2F70EFF41
:10D94000022811D1FFE70499039A44F61120C0F68A
:10D95000010000F053F8049841F67051C2F2000142
:10D960000860039848600AE044F62C20C0F60100E5
:10D9700040F27401C2F2000100F040F8FFE740F20B
:10D98000F401C2F200010020086040F27001C2F20E
:10D9900000010860FFE712E040F2F401C2F200016A
:10D9A0000020086040F27001C2F20001086040F2FD
:10D9B0007400C2F200008021F2F715FFFFE748E78C
:10D9C00006B080BD80B542F2D410C2F2000042F22F
:10D9D000A861C2F200014022FEF7D0FF80BD000026
:10D9E00080B540F63000C2F2000044F66721C0F670
:10D9F0000101242205F06AFA80BD000083B080B5E1
:10DA000083B0079306920591029005A801900299B0
:10DA1000019A40F2F800C2F200000090F2F78CFE8A
:10DA20000098F2F7B9FE009982B242F2D410C2F225
:10DA30000000FFF731FE03B0BDE8804003B070473F
:10DA4000FFE7FEE780B586B0FFE740F68840C4F206
:10DA50000240016841F001010160006800F001002E
:10DA600005900598FFE71E200190002203921146C1
:10DA7000F7F77AFE0198F7F76DFE039A1F200290E0
:10DA80001146F7F771FE0298F7F764FE039A20201B
:10DA900004901146F7F768FE0498F7F75BFE06B0AE
:10DAA00080BD000080B596B00020159014901390B2
:10DAB00012901190FFE740F68C40C4F202400168DA
:10DAC00041F080010160006800F080001090109823
:10DAD000FFE7FFE740F68C40C4F20240016841F0E6
:10DAE00004010160006800F004000F900F98FFE748
:10DAF000FFE740F68C40C4F20240016841F00201A9
:10DB00000160006800F002000E900E98FFE7FFE74A
:10DB100040F68C40C4F20240016841F040010160CF
:10DB2000006800F040000D900D98FFE7FFE740F619
:10DB30008C40C4F20240016841F0100101600068AD
:10DB400000F010000C900C98FFE7FFE740F68C40C7
:10DB5000C4F20240016841F001010160006800F078
:10DB600001000B900B98FFE7FFE740F68C40C4F2F2
:10DB70000240016841F008010160006800F00800FF
:10DB80000A900A98FFE741F60000C4F202200290D2
:10DB90000F21019100220692F7F70EFD069A40F63A
:10DBA0000000C4F2022003904FF49051F7F704FDF7
:10DBB000069A40F60040C4F2022007900421099121
:10DBC000F7F7FAFC019A0298069911920122049241
:10DBD00012921391149111A90891F7F777FB03980A
:10DBE000049B069A08994FF4007CCDF844C0129328
:10DBF00013921492F7F76AFB0398049B069A08990C
:10DC00004FF4805CCDF844C0129302230593139324
:10DC10001492F7F75BFBDDF810C0059B069A079896
:10DC20000899DDF824E0CDF844E0CDF848C013931E
:10DC30001492F7F74BFB16B080BD000080B590B092
:10DC400007A801902421F2F7F0FD01990022029229
:10DC500006920592049241F6E460C2F2000003903D
:10DC600042F60043C4F201030360426082604FF653
:10DC7000FF73C360026142618261012307930892CE
:10DC800009930A920B920C920D930E920F92FEF74B
:10DC90004BF818B1FFE7F6F7B7F9FFE7002004905B
:10DCA0000590069041F6E460C2F2000004A9FDF779
:10DCB00083FC18B1FFE7F6F7A7F9FFE710B080BDC6
:10DCC00080B588B0002100910791069105910491DB
:10DCD00003910291019141F63070C2F200004FF0C1
:10DCE00080420260F922426081604FF0FF32C260E0
:10DCF00001618161FDF76EFD18B1FFE7F6F784F968
:10DD0000FFE74FF48050049041F63070C2F20000FB
:10DD100004A9FDF705FF18B1FFE7F6F775F9FFE76E
:10DD200000200190039041F63070C2F2000001A97A
:10DD3000FDF742FC18B1FFE7F6F766F9FFE708B018
:10DD400080BD000080B594B0002101911391129123
:10DD5000119110910F910E910D910C910B910A91CF
:10DD600009910891079106910591049103910291FF
:10DD700041F67C70C2F2000040F20042C4F20002A0
:10DD80000260F922426081604FF6FF72C260016159
:10DD90008161FDF71FFD18B1FFE7F6F735F9FFE7E1
:10DDA0004FF48050109041F67C70C2F2000010A930
:10DDB000FDF7B6FE18B1FFE7F6F726F9FFE741F6E3
:10DDC0007C70C2F20000FEF7EDF918B1FFE7F6F73C
:10DDD0001BF9FFE741F67C70C2F20000FEF7F2FC8F
:10DDE00018B1FFE7F6F710F9FFE700200D900F904C
:10DDF00041F67C70C2F200000DA9FDF7DDFB18B101
:10DE0000FFE7F6F701F9FFE70020099001210A91E9
:10DE10000B900C9041F67C70C2F2000009A9082218
:10DE2000FEF728F918B1FFE7F6F7EEF8FFE76020F4
:10DE30000290002003900490069041F67C70C2F29C
:10DE4000000002A90C22FEF7E5FB18B1FFE7F6F788
:10DE5000DBF8FFE741F67C70C2F20000FEF77AFBC8
:10DE600014B080BD80B590B0002101910F910E914A
:10DE70000D910C910B910A910991089107910691CE
:10DE8000059104910391029141F6C870C2F200001D
:10DE900040F60002C4F200020260416081604FF669
:10DEA000FF72C26001618161FDF794FC18B1FFE768
:10DEB000F6F7AAF8FFE74FF480500C9041F6C870CF
:10DEC000C2F200000CA9FDF72BFE18B1FFE7F6F730
:10DED0009BF8FFE741F6C870C2F20000FEF772FC43
:10DEE00018B1FFE7F6F790F8FFE7002009900B90D4
:10DEF00041F6C870C2F2000009A9FDF75DFB18B138
:10DF0000FFE7F6F781F8FFE760200290002003901A
:10DF10000490069041F6C870C2F2000002A90C22DB
:10DF2000FEF778FB18B1FFE7F6F76EF8FFE741F66A
:10DF3000C870C2F20000FEF70DFB10B080BD0000FB
:10DF400080B590B007A801902421F2F76EFC0199EA
:10DF50000022029206920592049242F26000C2F2FE
:10DF60000000039043F20043C4F2010303604260E7
:10DF700082604FF6FF73C3600261426182610123D8
:10DF80000793089209930A920B920C920D930E92AA
:10DF90000F92FDF7C9FE18B1FFE7F6F735F8FFE776
:10DFA000002004900590069042F26000C2F200004A
:10DFB00004A9FDF701FB18B1FFE7F6F725F8FFE725
:10DFC00010B080BD80B5FFF70BFD03F091FC80BD64
:10DFD00080B582B042F2D410C2F20000009044F644
:10DFE0000041C4F2000101604FF41651416000216C
:10DFF00001918160C16001610C2242618161C16156
:10E00000016241628162FFF7B7F818B1FFE7F5F7E7
:10E01000FBFFFFE742F2D410C2F200000021FEF73E
:10E02000B7FD18B1FFE7F5F7EFFFFFE742F2D410B5
:10E03000C2F200000021FEF765FD18B1FFE7F5F719
:10E04000E3FFFFE742F2D410C2F20000FEF758FCF3
:10E0500018B1FFE7F5F7D8FFFFE702B080BD000079
:10E0600080B582B042F2AC00C2F20000009044F2EF
:10E070000041C4F2000101604FF4165141600021DB
:10E0800001918160C16001610C2242618161C161C5
:10E09000016241628162FFF76FF818B1FFE7F5F79F
:10E0A000B3FFFFE742F2AC00C2F200000021FEF72E
:10E0B0006FFD18B1FFE7F5F7A7FFFFE742F2AC00ED
:10E0C000C2F200000021FEF71DFD18B1FFE7F5F7D1
:10E0D0009BFFFFE742F2AC00C2F20000FEF710FC2B
:10E0E00018B1FFE7F5F790FFFFE702B080BD000031
:10E0F00080B582B042F24010C2F20000009044F6B7
:10E100000001C4F2000101604FF41651416000218A
:10E1100001918160C16001610C2242618161C16134
:10E12000016241628162FFF727F818B1FFE7F5F756
:10E130006BFFFFE742F24010C2F200000021FEF741
:10E1400027FD18B1FFE7F5F75FFFFFE742F2401048
:10E15000C2F200000021FEF7D5FC18B1FFE7F5F789
:10E1600053FFFFE742F24010C2F20000FEF7C8FB87
:10E1700018B1FFE7F5F748FFFFE702B080BD0000E8
:10E18000FFE7FEE7FFE7FEE788B0079006910592FC
:10E19000079800F0070004900498C0F107000528D4
:10E1A00003D3FFE70420019004E00498C0F10700C6
:10E1B0000190FFE70198039004980430062803D8E3
:10E1C000FFE70020009003E0049803380090FFE789
:10E1D0000098029006980399012202FA01F1013990
:10E1E0000840029B984005999A40013A1140084323
:10E1F00008B0704780B584B0029040F60041C4F288
:10E200000241086820F080600860F7F7EBF90190A0
:10E21000FFE740F60040C4F20240006800F00061F1
:10E220000020B0EBD16F0CD0FFE7F7F7DBF90199D5
:10E23000401A032804D3FFE703208DF80F008BE07A
:10E24000E7E7FFE740F62C41C4F20241086843F6D5
:10E2500003729043029B1A685B6842EA03221043F0
:10E26000086002998868D1F80CC00B694A690138C6
:10E270006FF35F204FF60061CFF6FF7101EB4C2189
:10E2800089B208440021CFF6FF7101EB034101F48C
:10E29000FE0108444FF07F4101EB026101F0FE41B5
:10E2A000084440F63C41C4F202410860FFE740F6F2
:10E2B0002C41C4F202410091086820F00C00029A3F
:10E2C000926910430860086820F02000029AD26921
:10E2D000104308600298426A0868104308600868A2
:10E2E00020F01000086040F64042C4F2024210687C
:10E2F0004FF6F8739843029B1B6A40EAC300106014
:10E30000086840F01000086040F60041C4F2024185
:10E31000086840F080600860F7F764F90190FFE753
:10E3200040F60040C4F20240006800F000610020A6
:10E33000B0EBD16F0CD1FFE7F7F754F90199401A10
:10E34000032804D3FFE703208DF80F0004E0E7E77C
:10E3500000208DF80F00FFE79DF80F0004B080BD8E
:10E3600080B584B0029040F60041C4F202410868D2
:10E3700020F080500860F7F735F90190FFE740F68C
:10E380000040C4F20240006800F000510020B0EBF1
:10E39000517F0CD0FFE7F7F725F90199401A0328C0
:10E3A00004D3FFE703208DF80F008BE0E7E7FFE7DA
:10E3B00040F63041C4F20241086843F603729043CC
:10E3C000029B1A685B6842EA0322104308600299C4
:10E3D0008868D1F80CC00B694A6901386FF35F2077
:10E3E0004FF60061CFF6FF7101EB4C2189B2084472
:10E3F0000021CFF6FF7101EB034101F4FE01084457
:10E400004FF07F4101EB026101F0FE41084440F60C
:10E410004441C4F202410860FFE740F63041C4F2D3
:10E4200002410091086820F00C00029A92691043A2
:10E430000860086820F02000029AD2691043086042
:10E440000298426A086810430860086820F01000CB
:10E45000086040F64842C4F2024210684FF6F87372
:10E460009843029B1B6A40EAC3001060086840F0B2
:10E470001000086040F60041C4F20241086840F014
:10E4800080500860F7F7AEF80190FFE740F60040D3
:10E49000C4F20240006800F000510020B0EB517F50
:10E4A0000CD1FFE7F7F79EF80199401A032804D32F
:10E4B000FFE703208DF80F0004E0E7E700208DF868
:10E4C0000F00FFE79DF80F0004B080BD80B59CB041
:10E4D00008A85021F2F7A9F90020079006900590AE
:10E4E000049003900290FFE740F61000C4F202404F
:10E4F000016841F030010160006800F030000190D7
:10E500000198FFE7FFE740F61400C4F202400068FC
:10E5100000F00800082801D0FFE7F4E71020089079
:10E520004FF480700F9020201090022012901390D2
:10E53000012114917D2115911690179018900820B3
:10E54000199000201A901B9008A8FCF7D1FA18B176
:10E55000FFE7F5F759FDFFE71F2002900320039026
:10E560000020049005900690079002A80521FBF773
:10E5700083FE18B1FFE7F5F747FDFFE742F2000120
:10E58000C4F202010868022262F3051008601CB0A0
:10E5900080BD000082B04EF68851CEF200010868BE
:10E5A00040F47000086040F60042C4F202420120CC
:10E5B000106040F61C41C4F2024100200090086047
:10E5C00040F62041C4F20241086011684EF6E32390
:10E5D000CEF6E2231940116040F62841C4F2024110
:10E5E000086040F62C41C4F20241086040F6304118
:10E5F000C4F20241086040F63443C4F2024340F2E0
:10E600008021C0F20111196040F63843C4F2024380
:10E61000186040F63C43C4F20243196040F64043A0
:10E62000C4F20243186040F64443C4F20243196046
:10E6300040F64841C4F202410860116821F480218B
:10E64000116040F65041C4F2024108604EF6085194
:10E65000CEF200014FF00060086042F21800C4F2F0
:10E660000200006800F0604001900198B0F1604F36
:10E6700005D0FFE70198B0F1404F24D1FFE742F207
:10E680001C00C4F202000068C00778B1FFE742F244
:10E690000C01C4F2020142F63B20C0F619000860EA
:10E6A00046F67F60C4F65D400860FFE742F21C0159
:10E6B000C4F20201086840F002000860086840F0F7
:10E6C00001000860FFE702B07047000080B541F626
:10E6D0003070C2F20000FDF7BDFD80BD80B541F68F
:10E6E0007C70C2F20000FDF7B5FD80BD80B542F23E
:10E6F0001400C2F20000FDF7ADFD80BD83B00290B2
:10E700000191029800680090029842F60041C4F21C
:10E710000101884252D0FFE7029842F60041C5F25B
:10E72000010188424AD0FFE70298B0F1804F45D0FE
:10E73000FFE70298B0F1A04F40D0FFE7029840F207
:10E740000041C4F20001884238D0FFE7029840F24D
:10E750000041C5F20001884230D0FFE7029840F640
:10E760000001C4F20001884228D0FFE7029840F679
:10E770000001C5F20001884220D0FFE7029840F670
:10E780000041C4F20001884218D0FFE7029840F629
:10E790000041C5F20001884210D0FFE7029843F221
:10E7A0000041C4F20101884208D0FFE7029843F219
:10E7B0000041C5F2010188420AD1FFE7009820F02C
:10E7C0007000009001984168009808430090FFE7AE
:10E7D000029842F60041C4F20101884200F0BA807A
:10E7E000FFE7029842F60041C5F20101884200F0BD
:10E7F000B180FFE70298B0F1804F00F0AB80FFE7F7
:10E800000298B0F1A04F00F0A580FFE7029840F217
:10E810000041C4F20001884200F09C80FFE70298AA
:10E8200040F20041C5F20001884200F09380FFE70A
:10E83000029840F60001C4F20001884200F08A808C
:10E84000FFE7029840F60001C5F20001884200F09F
:10E850008180FFE7029840F60041C4F2000188423F
:10E8600078D0FFE7029840F60041C5F200018842E7
:10E8700070D0FFE7029843F20041C4F201018842E0
:10E8800068D0FFE7029843F20041C5F201018842D7
:10E8900060D0FFE7029841F60001C4F2000188420F
:10E8A00058D0FFE7029841F60001C5F20001884206
:10E8B00050D0FFE7029841F60041C4F200018842BF
:10E8C00048D0FFE7029841F60041C5F200018842B6
:10E8D00040D0FFE7029842F20001C4F200018842F2
:10E8E00038D0FFE7029842F20001C5F200018842E9
:10E8F00030D0FFE7029844F20001C4F201018842DF
:10E9000028D0FFE7029844F20001C5F201018842D5
:10E9100020D0FFE7029844F20041C4F2010188428E
:10E9200018D0FFE7029844F20041C5F20101884285
:10E9300010D0FFE7029844F60001C4F201018842BA
:10E9400008D0FFE7029844F60001C5F201018842B1
:10E950000AD1FFE7009820F4407000900198C16848
:10E96000009808430090FFE7009820F0800001998C
:10E9700049690843009000980299086001988068EE
:10E980000299C8620198006802998862029842F66A
:10E990000041C4F20101884248D0FFE7029842F6E4
:10E9A0000041C5F20101884240D0FFE7029843F2DE
:10E9B0000041C4F20101884238D0FFE7029843F2D7
:10E9C0000041C5F20101884230D0FFE7029844F2CD
:10E9D0000001C4F20101884228D0FFE7029844F206
:10E9E0000001C5F20101884220D0FFE7029844F2FD
:10E9F0000041C4F20101884218D0FFE7029844F2B6
:10EA00000041C5F20101884210D0FFE7029844F6A8
:10EA10000001C4F20101884208D0FFE7029844F6E1
:10EA20000001C5F20101884205D1FFE701980069A4
:10EA300002990863FFE70299012048610298006982
:10EA4000C00730B1FFE70299086920F001000861B2
:10EA5000FFE703B07047000085B004900391029275
:10EA60000193049880680090009820F47F40009003
:10EA700003980299019A41EA022101430098084350
:10EA8000009000980499886005B0704783B00290A8
:10EA9000019102988068009000984FF68F71CFF630
:10EAA000CF710840009001980099084340F007009A
:10EAB000009000980299886003B0704785B0049078
:10EAC00003910498006A01900499086A20F00100FB
:10EAD0000862049840680090049880690290029847
:10EAE0004FF68F71CFF6FE7108400290029820F029
:10EAF000030002900398016802980843029001986D
:10EB000020F0020001900398816801980843019069
:10EB1000049842F60041C4F20101884248D0FFE760
:10EB2000049842F60041C5F20101884240D0FFE757
:10EB3000049843F20041C4F20101884238D0FFE753
:10EB4000049843F20041C5F20101884230D0FFE74A
:10EB5000049844F20001C4F20101884228D0FFE782
:10EB6000049844F20001C5F20101884220D0FFE779
:10EB7000049844F20041C4F20101884218D0FFE732
:10EB8000049844F20041C5F20101884210D0FFE729
:10EB9000049844F60001C4F20101884208D0FFE75E
:10EBA000049844F60001C5F2010188420ED1FFE746
:10EBB000019820F0080001900398C168019808436B
:10EBC0000190019820F004000190FFE7049842F6BC
:10EBD0000041C4F20101884248D0FFE7049842F6A0
:10EBE0000041C5F20101884240D0FFE7049843F29A
:10EBF0000041C4F20101884238D0FFE7049843F293
:10EC00000041C5F20101884230D0FFE7049844F288
:10EC10000001C4F20101884228D0FFE7049844F2C1
:10EC20000001C5F20101884220D0FFE7049844F2B8
:10EC30000041C4F20101884218D0FFE7049844F271
:10EC40000041C5F20101884210D0FFE7049844F664
:10EC50000001C4F20101884208D0FFE7049844F69D
:10EC60000001C5F20101884213D1FFE7009820F4AA
:10EC700080700090009820F4007000900398416923
:10EC80000098084300900398816900980843009019
:10EC9000FFE70098049948600298049988610398F6
:10ECA00040680499486301980499086205B0704768
:10ECB00085B0049003910498006A01900499086A51
:10ECC00020F0100008620498406800900498806961
:10ECD0000290029848F6FF71CFF6FF61084002905B
:10ECE000029820F44070029003980168029840EA6C
:10ECF00001200290019820F0200001900398816883
:10ED0000019840EA01100190049842F60041C4F2D3
:10ED10000101884251D0FFE7049842F60041C5F254
:10ED20000101884249D0FFE7049843F20041C4F250
:10ED30000101884241D0FFE7049843F20041C5F247
:10ED40000101884239D0FFE7049844F20001C4F27F
:10ED50000101884208D0FFE7049844F20001C5F29F
:10ED60000101884203D1FFE7002030BBFFE7049890
:10ED700044F20041C4F20101884208D0FFE7049840
:10ED800044F20041C5F20101884203D1FFE70020AF
:10ED900098B9FFE7049844F60001C4F201018842E3
:10EDA00008D0FFE7049844F60001C5F2010188424B
:10EDB00012D1FFE7012078B9FFE7019820F0800029
:10EDC00001900398C168019840EA011001900198F0
:10EDD00020F040000190FFE7049842F60041C4F2A1
:10EDE0000101884248D0FFE7049842F60041C5F28D
:10EDF0000101884240D0FFE7049843F20041C4F289
:10EE00000101884238D0FFE7049843F20041C5F27F
:10EE10000101884230D0FFE7049844F20001C4F2B7
:10EE20000101884228D0FFE7049844F20001C5F2AE
:10EE30000101884220D0FFE7049844F20041C4F267
:10EE40000101884218D0FFE7049844F20041C5F25E
:10EE50000101884210D0FFE7049844F60001C4F293
:10EE60000101884208D0FFE7049844F60001C5F28A
:10EE70000101884215D1FFE7009820F480600090DE
:10EE8000009820F40060009003984169009840EADF
:10EE90008100009003988169009840EA8100009009
:10EEA000FFE70098049948600298049988610398E4
:10EEB00040680499886301980499086205B0704716
:10EEC00085B0049003910498006A01900499086A3F
:10EED00020F4807008620498406800900498C0692B
:10EEE000029002984FF68F71CFF6FE7108400290A3
:10EEF000029820F0030002900398016802980843EA
:10EF00000290019820F400700190039881680198A4
:10EF100040EA01200190049842F60041C4F2010148
:10EF2000884251D0FFE7049842F60041C5F2010142
:10EF3000884249D0FFE7049843F20041C4F201013E
:10EF4000884241D0FFE7049843F20041C5F2010135
:10EF5000884239D0FFE7049844F20001C4F201016D
:10EF6000884208D0FFE7049844F20001C5F201018D
:10EF7000884203D1FFE7002030BBFFE7049844F24A
:10EF80000041C4F20101884208D0FFE7049844F22E
:10EF90000041C5F20101884203D1FFE7002098B982
:10EFA000FFE7049844F60001C4F20101884208D04A
:10EFB000FFE7049844F60001C5F20101884212D12E
:10EFC000FFE7012078B9FFE7019820F40060019085
:10EFD0000398C168019840EA01200190019820F44B
:10EFE00080600190FFE7049842F60041C4F20101FD
:10EFF000884248D0FFE7049842F60041C5F201017B
:10F00000884240D0FFE7049843F20041C4F2010176
:10F01000884238D0FFE7049843F20041C5F201016D
:10F02000884230D0FFE7049844F20001C4F20101A5
:10F03000884228D0FFE7049844F20001C5F201019C
:10F04000884220D0FFE7049844F20041C4F2010155
:10F05000884218D0FFE7049844F20041C5F201014C
:10F06000884210D0FFE7049844F60001C4F2010181
:10F07000884208D0FFE7049844F60001C5F2010178
:10F08000884215D1FFE7009820F480500090009846
:10F0900020F40050009003984169009840EA011064
:10F0A000009003988169009840EA01100090FFE702
:10F0B00000980499486002980499C86103984068D0
:10F0C0000499C86301980499086205B0704700006C
:10F0D00085B0049003910498006A01900499086A2D
:10F0E00020F4805008620498406800900498C06939
:10F0F0000290029848F6FF71CFF6FF610840029037
:10F10000029820F44070029003980168029840EA47
:10F1100001200290019820F400500190039881682A
:10F12000019840EA01300190049842F60041C4F28F
:10F130000101884251D0FFE7049842F60041C5F230
:10F140000101884249D0FFE7049843F20041C4F22C
:10F150000101884241D0FFE7049843F20041C5F223
:10F160000101884239D0FFE7049844F20001C4F25B
:10F170000101884208D0FFE7049844F20001C5F27B
:10F180000101884203D1FFE7002030BBFFE704986C
:10F1900044F20041C4F20101884208D0FFE704981C
:10F1A00044F20041C5F20101884203D1FFE700208B
:10F1B00098B9FFE7049844F60001C4F201018842BF
:10F1C00008D0FFE7049844F60001C5F20101884227
:10F1D00012D1FFE7012078B9FFE7019820F4004041
:10F1E00001900398C168019840EA013001900198AC
:10F1F00020F480400190FFE7049842F60041C4F2F9
:10F200000101884248D0FFE7049842F60041C5F268
:10F210000101884240D0FFE7049843F20041C4F264
:10F220000101884238D0FFE7049843F20041C5F25B
:10F230000101884230D0FFE7049844F20001C4F293
:10F240000101884228D0FFE7049844F20001C5F28A
:10F250000101884220D0FFE7049844F20041C4F243
:10F260000101884218D0FFE7049844F20041C5F23A
:10F270000101884210D0FFE7049844F60001C4F26F
:10F280000101884208D0FFE7049844F60001C5F266
:10F290000101884215D1FFE7009820F480400090DA
:10F2A000009820F40040009003984169009840EADB
:10F2B0008110009003988169009840EA81100090C5
:10F2C000FFE700980499486002980499C861039880
:10F2D00040680499086401980499086205B0704771
:10F2E00085B0049003910498006A01900499086A1B
:10F2F00020F4803008620498406800900498006D03
:10F30000029002984FF68F71CFF6FE71084002907E
:10F3100003980168029808430290019820F4003095
:10F32000019003988168019840EA01400190049897
:10F3300042F60041C4F20101884248D0FFE7049838
:10F3400042F60041C5F20101884240D0FFE704982F
:10F3500043F20041C4F20101884238D0FFE704982B
:10F3600043F20041C5F20101884230D0FFE7049822
:10F3700044F20001C4F20101884228D0FFE704985A
:10F3800044F20001C5F20101884220D0FFE7049851
:10F3900044F20041C4F20101884218D0FFE704980A
:10F3A00044F20041C5F20101884210D0FFE7049801
:10F3B00044F60001C4F20101884208D0FFE7049836
:10F3C00044F60001C5F2010188420BD1FFE7009825
:10F3D00020F48030009003984169009840EA0120B1
:10F3E0000090FFE700980499486002980499086526
:10F3F000039840680499886401980499086205B0EC
:10F400007047000085B0049003910498006A019051
:10F410000499086A20F480100862049840680090FB
:10F420000498006D0290029848F6FF71CFF6FF61D4
:10F430000840029003980168029840EA0120029077
:10F44000019820F40010019003988168019840EA27
:10F4500001500190049842F60041C4F20101884233
:10F4600048D0FFE7049842F60041C5F20101884206
:10F4700040D0FFE7049843F20041C4F20101884202
:10F4800038D0FFE7049843F20041C5F201018842F9
:10F4900030D0FFE7049844F20001C4F20101884231
:10F4A00028D0FFE7049844F20001C5F20101884228
:10F4B00020D0FFE7049844F20041C4F201018842E1
:10F4C00018D0FFE7049844F20041C5F201018842D8
:10F4D00010D0FFE7049844F60001C4F2010188420D
:10F4E00008D0FFE7049844F60001C5F20101884204
:10F4F0000BD1FFE7009820F4802000900398416929
:10F50000009840EA81200090FFE700980499486045
:10F51000029804990865039840680499C8640198A2
:10F520000499086205B0704785B004900391029277
:10F530000498006A00900499086A20F001000862AB
:10F54000049880690190019820F0F00001900299E0
:10F55000019840EA01100190009820F00A00009004
:10F5600003990098084300900198049988610098D5
:10F570000499086205B0704787B00690059104921F
:10F5800003930698006A01900699086A20F001002A
:10F5900008620698806902900699012042F60042AE
:10F5A000C4F201029142009000F09480FFE70699B6
:10F5B000012042F60042C5F201029142009000F0A3
:10F5C0008980FFE706990120B1F1804F009000F09B
:10F5D0008180FFE706990120B1F1A04F009079D01A
:10F5E000FFE70699012040F20042C4F20002914276
:10F5F00000906FD0FFE70699012040F20042C5F26B
:10F6000000029142009065D0FFE70699012040F684
:10F610000002C4F20002914200905BD0FFE706991D
:10F62000012040F60002C5F200029142009051D044
:10F63000FFE70699012040F60042C4F20002914221
:10F64000009047D0FFE70699012040F60042C5F23E
:10F650000002914200903DD0FFE70699012043F25D
:10F660000042C4F201029142009033D0FFE70699B4
:10F67000012043F20042C5F201029142009029D0DC
:10F68000FFE70699012041F60002C4F20002914210
:10F6900000901FD0FFE70699012041F60002C5F255
:10F6A00000029142009015D0FFE70699012044F234
:10F6B0000002C4F20102914200900BD0FFE70698CD
:10F6C0004CF20001CAF6FE710844B0FA80F040091D
:10F6D0000090FFE70098C00748B1FFE7029820F0CC
:10F6E00003000290049902980843029004E00298F3
:10F6F00040F001000290FFE7029820F0F000029035
:10F7000003980001C1B2029808430290019820F0CA
:10F710000A000190059800F00A0101980843019041
:10F7200002980699886101980699086207B07047A7
:10F7300085B00490039102920498006A00900499A5
:10F74000086A20F01000086204988069019001980E
:10F7500020F4704001900299019840EA0130019034
:10F76000009820F0A00000900399009840EA011052
:10F77000009001980499886100980499086205B086
:10F780007047000086B0059004910392029305989B
:10F79000006A00900599086A20F010000862059838
:10F7A00080690190019820F44070019003990198BC
:10F7B00040EA01200190019820F4704001900298E5
:10F7C000000381B2019808430190009820F0A00046
:10F7D0000090049800F00A01009840EA011000909F
:10F7E00001980599886100980599086206B07047EC
:10F7F00086B005900491039202930598006A0090E8
:10F800000599086A20F4807008620598C069019023
:10F81000019820F00300019003990198084301909A
:10F82000019820F0F000019002980001C1B2019807
:10F8300008430190009820F420600090049800F0A4
:10F840000A01009840EA0120009001980599C861DA
:10F8500000980599086206B07047000086B00590D0
:10F860000491039202930598006A00900599086A32
:10F8700020F4805008620598C0690190019820F436
:10F88000407001900399019840EA0120019001988D
:10F8900020F4704001900298000381B2019808435F
:10F8A0000190009820F420400090049800F00A0194
:10F8B000009840EA0130009001980599C8610098CD
:10F8C0000599086206B0704780B542F2D410C2F2C2
:10F8D0000000FDF7AFF980BD82B001900198406E45
:10F8E00040B9FFE701990120A1F86A000199A1F848
:10F8F000680034E008208DF803008DF802000198BC
:10F9000000688068C0F342608DF8010001980068CB
:10F910008068400F8DF800009DF802009DF80020DF
:10F9200044F6F403C0F60103995C00FB01F044F6D1
:10F93000EC01C0F601018A5CB0FBF2F0019AA2F87A
:10F940006A009DF803009DF801209B5C00FB03F01A
:10F95000895CB0FBF1F00199A1F86800FFE702B003
:10F960007047000081B00090009890F828000007D0
:10F9700000280BD5FFE700980068406820F400409D
:10F98000009A1168926B10434860FFE7009890F866
:10F990002800C00758B1FFE700980068406820F4CD
:10F9A0000030009A1168D26A10434860FFE700985F
:10F9B00090F82800800700280BD5FFE70098006822
:10F9C000406820F48030009A1168126B1043486040
:10F9D000FFE7009890F82800400700280BD5FFE7C4
:10F9E00000980068406820F48020009A1168526BEB
:10F9F00010434860FFE7009890F82800C0060028F0
:10FA00000BD5FFE700980068806820F48050009ACA
:10FA10001168D26B10438860FFE7009890F82800C7
:10FA2000800600280BD5FFE700980068806820F466
:10FA30000050009A1168126C10438860FFE700982C
:10FA400090F82800400600281CD5FFE700980068C1
:10FA5000406820F48010009A1168526C104348608E
:10FA60000098406CB0F5801F0BD1FFE7009800684C
:10FA7000406820F4C000009A1168926C10434860FE
:10FA8000FFE7FFE7009890F82800000600280BD554
:10FA9000FFE700980068406820F40020009A116891
:10FAA000D26C10434860FFE701B0704780B588B062
:10FAB000069006990020C1F89000F5F793FD059097
:10FAC000069800680068000700282FD5FFE7069811
:10FAD000059B6A466FF07E4111604FF400110022D1
:10FAE00001F07CF908B3FFE7FFE7FFE7069800683D
:10FAF00050E8000F20F080000490FFE7049906987A
:10FB0000026842E800100028F0D1FFE7FFE70699FD
:10FB10002020C1F88800FFE70699002081F88400C2
:10FB2000FFE703208DF81F005FE0FFE706980068FD
:10FB300000684007002842D5FFE70698059B6A4603
:10FB40006FF07E4111604FF48001002201F046F910
:10FB5000A0B3FFE7FFE7FFE70698006850E8000F53
:10FB600020F490700390FFE703990698026842E83A
:10FB700000100028F0D1FFE7FFE7FFE7FFE7069856
:10FB8000006850E8020F20F001000290FFE70299A0
:10FB90000698026842E802100028F0D1FFE7FFE76C
:10FBA00006992020C1F88C00FFE70699002081F813
:10FBB0008400FFE703208DF81F0016E0FFE7069999
:10FBC0002020C1F888000699C1F88C000699002011
:10FBD000C86606990867FFE70699002081F8840047
:10FBE000FFE700208DF81F00FFE79DF81F0008B019
:10FBF00080BD000080B582B001900198C06D00907A
:10FC000000990020A1F85E000098FDF70FF802B0FF
:10FC100080BD000080B584B003900398C06D029051
:10FC20000298D0F8880001900298D0F88C000090DB
:10FC3000029800688068000600280CD5FFE701984C
:10FC4000212808D1FFE702990020A1F85600029868
:10FC500000F0C8F8FFE702980068806840060028B6
:10FC60000CD5FFE70098222808D1FFE70299002071
:10FC7000A1F85E00029800F043F8FFE70299D1F87E
:10FC8000900040F01000C1F890000298FCF7CEFF01
:10FC900004B080BD80B584B003900398C06D02901D
:10FCA0000398006D812818D0FFE702990020A1F881
:10FCB0005600FFE7FFE70298006850E8000F40F0A9
:10FCC00040000190FFE701990298026842E80010A5
:10FCD0000028F0D1FFE7FFE703E00298FDF7AEFD53
:10FCE000FFE704B080BD000080B582B001900198AC
:10FCF000C06D00900098FDF7A5FD02B080BD00002A
:10FD000084B00390FFE7FFE70398006850E8000F16
:10FD100020F490700290FFE702990398026842E88D
:10FD200000100028F0D1FFE7FFE7FFE7FFE70398A7
:10FD3000006850E8020F4FF6FE71CEF6FF710840E2
:10FD40000190FFE701990398026842E80210002839
:10FD5000EDD1FFE7FFE70398C06E012814D1FFE75C
:10FD6000FFE7FFE70398006850E8000F20F010005D
:10FD70000090FFE700990398026842E8001000280D
:10FD8000F0D1FFE7FFE7FFE703992020C1F88C00DF
:10FD900003990020C8660399486704B070470000C3
:10FDA00080B582B00190FFE7FFE70198006850E856
:10FDB000000F20F040000090FFE7009901980268D2
:10FDC00042E800100028F0D1FFE7FFE7019920206A
:10FDD000C1F888000199002088670198FDF72EFD81
:10FDE00002B080BD83B00290FFE7FFE70298006891
:10FDF00050E8000F20F0C0000190FFE70199029841
:10FE0000026842E800100028F0D1FFE7FFE7FFE7B3
:10FE1000FFE70298006850E8020F20F4000000900D
:10FE2000FFE700990298026842E802100028F0D12A
:10FE3000FFE7FFE702992020C1F8880003B0704770
:10FE400080B588B007900798B0F86000ADF816004C
:10FE50000798D0F88C00222840F0B480FFE707987C
:10FE60000068406AADF814000798806D0690BDF8F0
:10FE70001400BDF816100840069908800799886D8F
:10FE8000023088650799B1F85E000138A1F85E007C
:10FE90000798B0F85E00002840F09380FFE7FFE786
:10FEA000FFE70798006850E8000F20F49070049076
:10FEB000FFE704990798026842E800100028F0D193
:10FEC000FFE7FFE7FFE7FFE70798006850E8020F4A
:10FED00020F001000390FFE703990798026842E8C9
:10FEE00002100028F0D1FFE7FFE707992020C1F8B2
:10FEF0008C000799002048670799086707980068F1
:10FF000042F20041C4F20041884225D0FFE7079841
:10FF1000006842F20041C5F2004188421CD0FFE770
:10FF20000798006840680002002814D5FFE7FFE743
:10FF3000FFE70798006850E8000F20F0806002900B
:10FF4000FFE702990798026842E800100028F0D104
:10FF5000FFE7FFE7FFE7FFE70798C06E01282BD117
:10FF6000FFE707990020C866FFE7FFE707980068EA
:10FF700050E8000F20F010000190FFE7019907986A
:10FF8000026842E800100028F0D1FFE7FFE7079879
:10FF90000068C06900F010010120B0EB111F05D10D
:10FFA000FFE70798016810200862FFE70798B0F89C
:10FFB0005C10FCF745FD03E00798FDF769FBFFE7E0
:10FFC000FFE706E007980168886940F0080088614B
:10FFD000FFE708B080BD000080B58EB00D900D9891
:10FFE000B0F86000ADF82E000D980068C069099067
:10FFF0000D980068006808900D9800688068079068
:020000040801F1
:100000000D98D0F88C00222840F06A81FFE70D9807
:10001000B0F86800ADF82A00FFE7BDF82A1000200C
:10002000009031B1FFE79DF82400C0F3401000902C
:10003000FFE70098C007002800F01381FFE70D9844
:100040000068406AADF82C000D98806D0C90BDF8EA
:100050002C00BDF82E1008400C9908800D99886D71
:10006000023088650D99B1F85E000138A1F85E0094
:100070000D980068C06909909DF824004007002889
:1000800052D0FFE79DF82400C00788B1FFE79DF834
:100090002100C00760B1FFE70D98016801200862E8
:1000A0000D99D1F8900040F00100C1F89000FFE7F1
:1000B0009DF824008007002811D5FFE79DF81C005B
:1000C000C00760B1FFE70D980168022008620D9932
:1000D000D1F8900040F00400C1F89000FFE79DF8CF
:1000E00024004007002811D5FFE79DF81C00C00739
:1000F00060B1FFE70D980168042008620D99D1F8FE
:10010000900040F00200C1F89000FFE70D98D0F891
:10011000900040B1FFE70D98FCF788FD0D99002095
:10012000C1F89000FFE7FFE70D98B0F85E000028E7
:1001300040F09680FFE7FFE7FFE70D98006850E882
:10014000000F20F480700690FFE706990D98026872
:1001500042E800100028F0D1FFE7FFE7FFE7FFE7E4
:100160000D98006850E8020F4FF6FE71CEF6FF7151
:1001700008400590FFE705990D98026842E80210D3
:100180000028EDD1FFE7FFE70D992020C1F88C0092
:100190000D99002048670D9908670D98006842F294
:1001A0000041C4F20041884225D0FFE70D98006865
:1001B00042F20041C5F2004188421CD0FFE70D9891
:1001C000006840680002002814D5FFE7FFE7FFE75A
:1001D0000D98006850E8000F20F080600490FFE761
:1001E00004990D98026842E800100028F0D1FFE75A
:1001F000FFE7FFE7FFE70D98C06E01282BD1FFE76F
:100200000D990020C866FFE7FFE70D98006850E8E9
:10021000000F20F010000390FFE703990D9802688B
:1002200042E800100028F0D1FFE7FFE70D980068D2
:10023000C06900F010010120B0EB111F05D1FFE7EC
:100240000D98016810200862FFE70D98B0F85C1067
:10025000FCF7F6FB03E00D98FDF71AFAFFE700E064
:10026000DBE60D98B0F85E00ADF82800BDF8280078
:10027000A8B3FFE7BDF828000D99B1F868108842CF
:100280002DDAFFE7FFE7FFE70D98006850E8020F5F
:1002900020F080500290FFE702990D98026842E832
:1002A00002100028F0D1FFE7FFE70D994FF64160FB
:1002B000C0F600004867FFE7FFE70D98006850E8C8
:1002C000000F40F020000190FFE701990D980268AF
:1002D00042E800100028F0D1FFE7FFE7FFE706E063
:1002E0000D980168886940F008008861FFE70EB04A
:1002F00080BD000080B586B005900598B0F860001C
:10030000ADF812000598D0F88C00222840F0B28099
:10031000FFE705980068406AADF81000BDF81000CE
:100320009DF8121008400599896D08700599886D2F
:10033000013088650599B1F85E000138A1F85E00CA
:100340000598B0F85E00002840F09380FFE7FFE7D3
:10035000FFE70598006850E8000F20F490700390C4
:10036000FFE703990598026842E800100028F0D1E1
:10037000FFE7FFE7FFE7FFE70598006850E8020F97
:1003800020F001000290FFE702990598026842E818
:1003900002100028F0D1FFE7FFE705992020C1F8FF
:1003A0008C00059900204867059908670598006842
:1003B00042F20041C4F20041884225D0FFE705988F
:1003C000006842F20041C5F2004188421CD0FFE7BC
:1003D0000598006840680002002814D5FFE7FFE791
:1003E000FFE70598006850E8000F20F0806001905A
:1003F000FFE701990598026842E800100028F0D153
:10040000FFE7FFE7FFE7FFE70598C06E01282BD164
:10041000FFE705990020C866FFE7FFE70598006839
:1004200050E8000F20F010000090FFE700990598B9
:10043000026842E800100028F0D1FFE7FFE70598C6
:100440000068C06900F010010120B0EB111F05D158
:10045000FFE70598016810200862FFE70598B0F8EB
:100460005C10FCF7EDFA03E00598FDF711F9FFE7E2
:10047000FFE706E005980168886940F00800886198
:10048000FFE706B080BD000080B58EB00D900D98DE
:10049000B0F86000ADF832000D980068C0690A90AD
:1004A0000D980068006809900D98006880680890B1
:1004B0000D98D0F88C00222840F06881FFE70D9855
:1004C000B0F86800ADF82E00FFE7BDF82E10002050
:1004D000019031B1FFE79DF82800C0F34010019072
:1004E000FFE70198C007002800F01181FFE70D9891
:1004F0000068406AADF83000BDF830009DF8321059
:1005000008400D99896D08700D99886D01308865D6
:100510000D99B1F85E000138A1F85E000D980068F1
:10052000C0690A909DF828004007002852D0FFE7D4
:100530009DF82800C00788B1FFE79DF82500C00797
:1005400060B1FFE70D980168012008620D99D1F8AC
:10055000900040F00100C1F89000FFE79DF82800EE
:100560008007002811D5FFE79DF82000C00760B183
:10057000FFE70D980168022008620D99D1F89000FC
:1005800040F00400C1F89000FFE79DF82800400704
:10059000002811D5FFE79DF82000C00760B1FFE7F4
:1005A0000D980168042008620D99D1F8900040F080
:1005B0000200C1F89000FFE70D98D0F8900040B11C
:1005C000FFE70D98FCF732FB0D990020C1F8900071
:1005D000FFE7FFE70D98B0F85E00002840F0968036
:1005E000FFE7FFE7FFE70D98006850E8000F20F4F1
:1005F00080700790FFE707990D98026842E80010A5
:100600000028F0D1FFE7FFE7FFE7FFE70D9800685C
:1006100050E8020F4FF6FE71CEF6FF7108400690CB
:10062000FFE706990D98026842E802100028EDD114
:10063000FFE7FFE70D992020C1F88C000D990020FD
:1006400048670D9908670D98006842F20041C4F2AE
:100650000041884225D0FFE70D98006842F2004132
:10066000C5F2004188421CD0FFE70D980068406841
:100670000002002814D5FFE7FFE7FFE70D980068A8
:1006800050E8000F20F080600590FFE705990D9875
:10069000026842E800100028F0D1FFE7FFE7FFE71B
:1006A000FFE70D98C06E01282BD1FFE70D990020C0
:1006B000C866FFE7FFE70D98006850E8000F20F0DC
:1006C00010000490FFE704990D98026842E80010BA
:1006D0000028F0D1FFE7FFE70D980068C06900F03F
:1006E00010010120B0EB111F05D1FFE70D98016843
:1006F00010200862FFE70D98B0F85C10FCF7A0F935
:1007000003E00D98FCF7C4FFFFE700E0DDE60D987D
:10071000B0F85E00ADF82C00BDF82C00A8B3FFE7E0
:10072000BDF82C000D99B1F8681088422DDAFFE76A
:10073000FFE7FFE70D98006850E8020F20F08050B7
:100740000390FFE703990D98026842E80210002821
:10075000F0D1FFE7FFE70D9940F2F520C0F6010068
:100760004867FFE7FFE70D98006850E8000F40F08A
:1007700020000290FFE702990D98026842E80010FD
:100780000028F0D1FFE7FFE7FFE706E00D980168DA
:10079000886940F008008861FFE70EB080BD000066
:1007A00080B58AB0099000208DF813000998006880
:1007B00042F20041C4F20041884209D0FFE70998A3
:1007C000006842F20041C5F20041884201D1FFE7D2
:1007D00000E0FFE7099988680B694A69C96918430D
:1007E00010430843089009980068006846F6F31122
:1007F000CCF6FF7108400899084309990968086018
:1008000009980068406820F44050099A1168D2683D
:10081000104348600998806908900998006842F27E
:100820000041C4F2004188420FD0FFE709980068F8
:1008300042F20041C5F20041884206D0FFE7099824
:10084000016A089808430890FFE7099800688068E3
:100850004FF2FF41C1F2FF1108400899084309997E
:100860000968886009980068C06A20F00F00099A3A
:100870001168526A1043C862FFE70998006843F69E
:100880000001C4F20101884203D1FFE70120069074
:10089000A3E00998006844F20041C4F200018842D4
:1008A00003D1FFE70220069096E00998006844F61D
:1008B0000001C4F20001884203D1FFE70420069042
:1008C00089E00998006844F60041C4F200018842BA
:1008D00003D1FFE7082006907CE00998006845F204
:1008E0000001C4F20001884203D1FFE71020069006
:1008F0006FE00998006846F20041C4F200018842A6
:1009000003D1FFE72020069062E00998006847F6CF
:100910000001C4F20001884203D1FFE740200690A5
:1009200055E00998006847F60041C4F2000188428A
:1009300003D1FFE78020069048E00998006848F25C
:100940000001C4F20001884204D1FFE74FF4807037
:1009500006903AE00998006846F60001C4F20001EA
:10096000884204D1FFE74FF4007006902CE009980C
:10097000006846F60041C4F20001884204D1FFE756
:100980004FF4806006901EE00998006848F200412C
:10099000C4F20001884204D1FFE74FF400600690E2
:1009A00010E00998006842F20041C4F20041884218
:1009B00004D1FFE74FF48050069002E0002006903B
:1009C000FFE7FFE7FFE7FFE7FFE7FFE7FFE7FFE7F7
:1009D000FFE7FFE7FFE7FFE7FFE7FFE709980068AA
:1009E00042F20041C4F20041884209D0FFE7099871
:1009F000006842F20041C5F2004188425CD1FFE745
:100A000006980021F5F744FB02900298002852D086
:100A1000FFE7029809994A6A44F6FC01C0F6010111
:100A200031F81210B0FBF1F003900398099949686E
:100A300001EB4101884207D3FFE703980999496810
:100A4000B0EB013F04D9FFE701208DF8130031E03E
:100A5000029809994A6800924A6A44F6FC01C0F675
:100A6000010131F81220002301931946EFF7ECFD44
:100A7000009A019B090241EA1061000210EB52004A
:100A800041F10001EFF7E0FD05900598B0F5407FDA
:100A90000BD3FFE705990020B0EB115F05D1FFE70D
:100AA000059809990968C86003E001208DF81300D2
:100AB000FFE7FFE7FFE76FE00998C069B0F5004F77
:100AC0003CD1FFE706980021F5F7E2FA0290029880
:100AD00098B3FFE70298099A5168536A44F6FC02FA
:100AE000C0F6010232F81320B0FBF2F0400000EB38
:100AF0005100B0FBF1F005900598102818D3FFE7DE
:100B0000BDF81600A0B9FFE7059820F00F00ADF87A
:100B10001E00059800F00E01BDF81E0040EA5100CD
:100B2000ADF81E00BDF81E0009990968C86003E011
:100B300001208DF81300FFE7FFE72CE00698002165
:100B4000F5F7A6FA0290029820B3FFE70298099AF7
:100B50005168536A44F6FC02C0F6010232F81320D1
:100B6000B0FBF2F000EB5100B0FBF1F005900598FE
:100B700010280AD3FFE7BDF8160030B9FFE7BDF82B
:100B8000140009990968C86003E001208DF813007A
:100B9000FFE7FFE7FFE7FFE709990120A1F86A00F7
:100BA0000999A1F8680009990020486709998867A0
:100BB0009DF813000AB080BD88B007900691ADF88B
:100BC0001620069807998865BDF816000799A1F8C0
:100BD0005C00BDF816000799A1F85E000799002097
:100BE0004867FFE707988068B0F5805F10D1FFE79E
:100BF0000798006930B9FFE7079940F2FF10A1F8A4
:100C0000600004E00799FF20A1F86000FFE72EE0F4
:100C10000798806878B9FFE70798006928B9FFE767
:100C20000799FF20A1F8600004E007997F20A1F850
:100C30006000FFE71AE007988068B0F1805F0FD18D
:100C4000FFE70798006928B9FFE707997F20A1F817
:100C5000600004E007993F20A1F86000FFE704E08E
:100C600007990020A1F86000FFE7FFE7FFE7FFE733
:100C700007990020C1F8900007992220C1F88C0044
:100C8000FFE7FFE70798006850E8020F40F0010017
:100C90000490FFE704990798026842E802100028D0
:100CA000F0D1FFE7FFE70798406EB0F1005F4CD14D
:100CB000FFE7BDF816000799B1F86810884244DBD9
:100CC000FFE707988068B0F5805F0BD1FFE70798D2
:100CD000006938B9FFE707994FF6D970C0F60000F0
:100CE000486706E0079940F28940C0F6010048676E
:100CF000FFE707980069A0B1FFE7FFE7FFE7079864
:100D0000006850E8000F40F480700390FFE70399FB
:100D10000798026842E800100028F0D1FFE7FFE7DB
:100D2000FFE7FFE7FFE70798006850E8020F40F091
:100D300080500290FFE702990798026842E802108B
:100D40000028F0D1FFE7FFE744E007988068B0F59E
:100D5000805F0BD1FFE70798006938B9FFE7079973
:100D60004FF64160C0F60000486706E0079940F280
:100D7000F520C0F601004867FFE707980069A0B1B9
:100D8000FFE7FFE7FFE70798006850E8000F40F42F
:100D900090700190FFE701990798026842E80010FF
:100DA0000028F0D1FFE7FFE713E0FFE7FFE7079830
:100DB000006850E8000F40F020000090FFE7009925
:100DC0000798026842E800100028F0D1FFE7FFE72B
:100DD000FFE7FFE7002008B07047000080B586B04D
:100DE000DDF820C0049003918DF80B200193FFE7FC
:100DF00004980068C06903990840401AB0FA80F06E
:100E000040099DF80B10884266D1FFE70898013031
:100E1000002860D0FFE7F4F7E5FB0199401A089934
:100E2000884203D8FFE7089820B9FFE703208DF830
:100E3000170055E00498006800684007002849D56D
:100E4000FFE70398802845D0FFE70398402841D06A
:100E5000FFE704980068C06900F008010120B0EBCA
:100E6000D10F16D1FFE704980168082000900862AE
:100E70000498FEF745FF00980499C1F89000FFE739
:100E80000499002081F88400FFE701208DF8170005
:100E900026E004980068C06900F400610120B0EB0E
:100EA000D12F16D1FFE7049801684FF40060086263
:100EB0000498FEF725FF04992020C1F89000FFE771
:100EC0000499002081F88400FFE703208DF81700C3
:100ED00006E0FFE7FFE78BE700208DF81700FFE74C
:100EE0009DF8170006B080BD80B542F2AC00C2F29A
:100EF0000000FBF79FFE80BD80B542F24010C2F2B9
:100F00000000FBF797FE80BDFFE7FEE781B0ADF87C
:100F10000200BDF9020000280ED4FFE7BDF902105F
:100F200001F01F02012090404A094EF20011CEF25A
:100F3000000141F82200FFE701B070474EF60C5067
:100F4000CEF200000068C0F30220704782B0ADF816
:100F500006000091BDF9060000280AD4FFE70098BA
:100F60000001BDF906104EF20042CEF20002885494
:100F70000BE000980001BDF8061001F00F014EF6DD
:100F80001452CEF200028854FFE702B0704700000E
:100F900083B00290029800F0070000904EF60C51CA
:100FA000CEF200010868019001984FF6FF02104050
:100FB00001900198009A40EA02200022C0F2FA5201
:100FC000104301900198086003B0704780B58EB05F
:100FD0000A900991089207930A983421EFF725FCAB
:100FE000079820F00300079009980A99486008982C
:100FF0000A99886107980A99C86108980A9908614E
:1010000008980A994861079808380A9988600A99E7
:101010000220C86008980590059807990844059033
:101020000598043805900A98039005980490039851
:10103000049908600598043805900598049008986C
:1010400004990860089803900398049005980499FF
:101050000860089805900598043005900598009060
:1010600000994EF6EE60CFF6FF7008600A990020F6
:101070000862EFF310800D900D980B9072B60B98EC
:1010800006900A9945F24540C4F25920086040F2A2
:10109000FC10C2F20000006858B9FFE70A9840F25D
:1010A0000021C2F2000108600A98C0620A98006339
:1010B00015E040F20020C2F20000006802900298A1
:1010C000006B01900A98029908630A980199C86216
:1010D00001980A99086302980A99C862FFE740F2EA
:1010E000FC11C2F2000108680130086006980C90FB
:1010F0000C9880F3108800200EB080BD80B58EB0B3
:1011000007900691EFF310800C900C98099072B63E
:10111000099805900798806E41F2FD01C0F6010123
:10112000884276D1FFE706980799D1F8AC1088423B
:101130006ED1FFE70798C06E04900498002866D02F
:10114000FFE70498006844F24E41C4F256418842D9
:101150005CD1FFE704984069002856D0FFE7079963
:101160000020886604984069039004980069029002
:10117000029820B3FFE7039801380390039804997D
:101180004861039820B9FFE704990020086115E041
:101190000798006F01900798406F009000980199A0
:1011A000486701980099086702980799884204D116
:1011B000FFE7019804990861FFE7FFE703E004995E
:1011C0000120C860FFE70798006B07281CD1FFE7E4
:1011D00007990720C1F8840040F24021C2F20001C3
:1011E00008680130086005980B900B9880F3108810
:1011F000079801F065F8EFF310800D900D980890B6
:1012000072B608980590FFE7FFE7FFE7FFE7FFE703
:10121000FFE705980A900A9880F310880EB080BD09
:1012200080B588B00490039104982421EFF7FDFA6B
:10123000039804994860EFF3108007900798059091
:1012400072B605980290049944F24E40C4F256409A
:10125000086040F20420C2F20000006858B9FFE7BD
:10126000049840F20821C2F20001086004988061ED
:101270000498C06115E040F20820C2F20000006846
:1012800001900198C069009004980199C861049880
:101290000099886100980499C8610198049988614F
:1012A000FFE740F20421C2F2000108680130086043
:1012B00002980690069880F31088002008B080BD40
:1012C00080B596B0DDF860C00F900E910D920C9332
:1012D000EFF3108014901498119072B611980B903F
:1012E0000F988068079007980F99096A88430C99AE
:1012F00008600D9800F0020009900F98006A0590B0
:10130000059828B1FFE70798059988430790FFE7FC
:10131000099802280DD1FFE707980E99084006901A
:1013200006980E99884203D0FFE700200690FFE759
:1013300004E007980E9908400690FFE7069850B31E
:10134000FFE70D9800F001000890089801281FD1D0
:10135000FFE7002000900F98406940B1FFE70F9829
:10136000006918B9FFE701200090FFE7FFE7009848
:10137000012806D1FFE70F99086A0E9A1043086208
:1013800005E00F9988680E9A90438860FFE7FFE7B1
:1013900000200A907EE01898002877D0FFE740F2FE
:1013A0004020C2F20000006818B9FFE70E9818B993
:1013B000FFE707200A9068E040F23020C2F2000008
:1013C00000680390039941F2FD00C0F601008866B1
:1013D0000E98039988670D980399C1F880000C98BE
:1013E0000399C8670F980399C8660399D1F8AC00B0
:1013F0000130C1F8AC000F9840690490049840B9DE
:10140000FFE703980F990861039800670398406706
:1014100012E00F98006902900298039908670298F9
:10142000406F0190019803994867039801990867F4
:10143000039802994867FFE70F99486901304861AE
:10144000039907200863039901208863189803997A
:10145000C86440F24021C2F200010868013008600F
:101460000B981390139880F31088039801F04CF8B0
:10147000EFF3108015901598109072B610980B909D
:101480000398D0F884000A90FFE702E007200A9052
:10149000FFE7FFE70B981290129880F310880A98E4
:1014A00016B080BD80B5A6B0159014911392EFF3DD
:1014B0001080219021981A9072B61A9812909DF877
:1014C0004C008007002825D5FFE7002001901598E3
:1014D000406940B1FFE71598006918B9FFE701209E
:1014E0000190FFE7FFE70198012807D1FFE7159971
:1014F000086A149A60EA0200086205E01599886893
:10150000149A10408860FFE712982090209880F38A
:101510001088A5E115998868149A10438860159879
:10152000006A30B1FFE71599086A149A904308627F
:10153000FFE700200290159840690A90159800690D
:10154000002800F07781FFE70A98012861D1FFE7C2
:101550001598006911901598806809901198806F0E
:1015600008901198D0F880000490049800F00200D0
:101570000590059802280DD1FFE7099808990840C1
:10158000079007980899884203D0FFE7002007904A
:10159000FFE704E00998089908400790FFE70798DB
:1015A000B0B3FFE71198C06F0690099806990860DC
:1015B000049800F0010003900398012806D1FFE78A
:1015C00015998868089A90438860FFE7159900206C
:1015D000086115994861119988661199C1F88400CC
:1015E00040F24021C2F20001086801300860129800
:1015F0001F901F9880F31088119800F061FEEFF3A0
:10160000108022902298199072B619981290FFE7D4
:101610000FE1159800690B900B9811901599002017
:1016200008610D900C9015988068099040F2402157
:10163000C2F2000108680130086001200290FFE753
:1016400012981E901E9880F31088EFF3108023905C
:101650002398189072B6189812901598C06870B1B7
:10166000FFE715990020C8600B9811901598406904
:101670000A9009981599896808430990FFE711981D
:10168000006F10901198806F08901198D0F880002A
:101690000490049800F002000590059802280DD1EE
:1016A000FFE7099808990840079007980899884229
:1016B00003D0FFE700200790FFE704E009980899AE
:1016C00008400790FFE71198006B072803D0FFE759
:1016D00001200790FFE70798002857D0FFE71198EF
:1016E000006B07281BD1FFE71198C06F069009987F
:1016F00006990860049800F00100039003980128FF
:1017000006D1FFE715998868089A90438860FFE73B
:101710001199002088661199C1F88400FFE711989B
:10172000016F884203D1FFE700200B9015E011986C
:10173000006F0F901198406F0E900E980F994867A8
:101740000F980E9908670B981199884204D1FFE70A
:101750001198006F0B90FFE7FFE715994869013872
:1017600048610D9840B9FFE711980D9011980C90C1
:1017700011990020086708E011980C9908671199E1
:101780000020086711980C90FFE7FFE71098119070
:101790000A9801380A90FFE70A9800287FF450AFB2
:1017A000FFE70B98159908611598006A48B1FFE7A3
:1017B000159988680A6A9043886015990020086224
:1017C000FFE712981D901D9880F310880D981190D6
:1017D000FFE71198E8B1FFE71198006F1090EFF361
:1017E000108024902498179072B61798129040F2A7
:1017F0004021C2F2000108680130086012981C9074
:101800001C9880F31088119800F05AFD10981190E0
:10181000DFE7EFF3108025902598169072B61698A2
:10182000129040F24021C2F20001086801380860BD
:10183000FFE708E01598406920B1FFE715990120FE
:10184000C860FFE7FFE712981B901B9880F3108891
:101850000298012803D1FFE700F0FAFCFFE7FFE759
:10186000002026B080BD000080B500F067FC01F0CC
:1018700035F840F22421C2F200010020086040F255
:101880002021C2F20001086040F21C21C2F20001D6
:10189000086040F21821C2F20001086040F20821FD
:1018A000C2F20001086040F20421C2F200010860A7
:1018B00040F2F411C2F20001086040F2F011C2F2ED
:1018C0000001086040F20021C2F20001086040F20D
:1018D000FC11C2F20001086040F21421C2F20001C2
:1018E000086040F21021C2F20001086080BD0000D3
:1018F00080B582B040F20400C2F20000006810F12E
:101900000F3F13D0FFE740F20401C2F200014FF095
:10191000F0300860EEF778FDFFF7A6FF40F24021B7
:10192000C2F20001086801300860FFE740F20401DC
:10193000C2F2000101914FF0F030086040F20C203B
:10194000C2F20000006801F0B1FE019900200860B9
:10195000EEF796FD02B080BD80B58EB0079006917F
:10196000EFF310800C900C98099072B609980590CE
:101970000798806E41F65911C0F60101884274D172
:10198000FFE706980799D1F8AC1088426CD1FFE7C1
:101990000798C06E04900498002864D0FFE704986C
:1019A000006844F25551C5F2551188425AD1FFE7FB
:1019B0000498C06A002854D0FFE707990020886681
:1019C0000499C86A0138C8620498C06A03900398F1
:1019D00020B9FFE704990020886216E00798006F9D
:1019E00002900798406F0190019802994867029809
:1019F000019908670498806A0799884204D1FFE733
:101A0000029804998862FFE7FFE70798006B0528B2
:101A100026D1FFE70498006928B1FFE707990B205A
:101A2000C1F8840004E007990A20C1F88400FFE7A8
:101A300040F24021C2F200010868013008600598B8
:101A40000B900B9880F31088079800F039FCEFF3A7
:101A500010800D900D98089072B608980590FFE7D9
:101A6000FFE7FFE7FFE7FFE7FFE705980A900A981F
:101A700080F310880EB080BD80B58CB0DDF838C022
:101A8000089007910692059308983821EEF7CDFE4D
:101A90000798089948600698089988600E980699F2
:101AA0008900B0FBF1F003900398069900FB01F068
:101AB000029005980899886108998869029A00EB54
:101AC0008200C861059808990862059808994862DB
:101AD00003980899486103980899C860EFF310804B
:101AE0000B900B98099072B609980490089944F2EB
:101AF0005550C5F25510086040F21820C2F200009F
:101B0000006858B9FFE7089840F21C21C2F20001B2
:101B10000860089800630898406315E040F21C20B4
:101B2000C2F20000006801900198406B0090089894
:101B300001994863089800990863009808994863D8
:101B4000019808990863FFE740F21821C2F20001EA
:101B500008680130086004980A900A9880F3108899
:101B600000200CB080BD000080B594B00B900A91AD
:101B7000099200200090EFF31080139013980C90BE
:101B800072B60C9808900B98C06A03900B98006985
:101B9000002800F04981FFE7039800283FD1FFE7C4
:101BA0000B98006A06900A9805900B98806804903C
:101BB0000698011D0691006805990A1D05920860A6
:101BC0000498022810D3FFE7FFE704980138049037
:101BD00048B1FFE70698011D0691006805990A1DA6
:101BE00005920860F1E7FFE706980B99C9698842FA
:101BF00004D1FFE70B9880690690FFE706980B99E0
